:020000040800F2
:1000000000C0002049450108E9450108312F0108D9
:10001000E9450108E9450108E9450108000000003B
:10002000000000000000000000000000E945010899
:10003000E945010800000000E9450108D5A50008D0
:10004000E9450108E9450108E9450108E9450108D4
:10005000E9450108E94501089DB2000899B2000888
:10006000E9450108E9450108E9450108E9450108B4
:10007000E9450108E9450108B9B20008E945010868
:1000800061E90008E9450108E9450108E945010879
:10009000E9450108E9450108E945010895B200086C
:1000A000E945010885B00008E945010895B0000858
:1000B00075B0000865B0000855B000083159000857
:1000C00035590008295900082D590008E94501084B
:1000D000E9450108ADB20008A1B20008E9450108F0
:1000E000E5A50008E9450108E9450108E9450108D9
:1000F000E9450108E9450108E9450108E945010824
:10010000E9450108E9450108E9450108E945010813
:10011000E9450108E9450108E9450108E945010803
:10012000E9450108E9450108E9450108E9450108F3
:1001300000000000000000000000000000000000BF
:1001400000000000000000000000000000000000AF
:10015000000000000000000000000000000000009F
:10016000000000000000000000000000000000008F
:10017000000000000000000000000000000000007F
:10018000000000000000000000000000000000006F
:10019000000000000000000000000000000000005F
:1001A000000000000000000000000000000000004F
:1001B000000000000000000000000000000000003F
:1001C000000000000000000000000000000000002F
:1001D000000000000000000000000000000000001F
:0401E0005FF8E0F1F3
:1001E8002DE9F04F684B694FA1B03B6000237B605D
:1001F80011F0BCFA18B911F0DBFA08F041FC08F06C
:1002080005FD634A634C1378634E43F00103137092
:100218000023089309930A934FF4E0130B93236880
:10022800B07B43F480332360A36943F01003A361D8
:10023800236803F400330993089B01330893099B4F
:100248001BB9089BB3F5A06FF2D12368514913F489
:10025800003301D0022315E00A6842F001020A6067
:100268000893236803F002030993089B013308935A
:10027800099B1BB9089BB3F5A06FF2D123689B07B4
:1002880039D501230A93454B45491A6842F01002B3
:100298001A601A6822F003021A601A6842F0020211
:1002A8001A606368636063686360636843F48063CB
:1002B80063603C4B1A68043B22F070425A603A4A29
:1002C8001160616821F47C116160596841F0004156
:1002D8005960D96821F40041D9609B681D0449BF61
:1002E800324B4FF4E01313604FF480130B930A9BC7
:1002F800012B01D117E0FEE7022B18D168B10B9B47
:10030800B3F5801F02D14FF4A01305E00B9BB3F5A2
:10031800E01F02D14FF400130B930B9963680B4352
:1003280043F4803302E0636843F460136360236836
:1003380043F0807323602168164B8901FBD5596807
:1003480021F003015960596841F00201596063685E
:10035800104903F00C03082BF9D14B68DFF85490CF
:1003680003F00C03042B03D0082B03D00C4B29E01B
:10037800136827E04B684868C3F38343C50303F158
:10038800020319D40A4A1CE06F820008C800002042
:100398009430002000100240602500200020024018
:1003A80000127A000410014034000020001BB7003E
:1003B80000093D005000002049681268880348BFC2
:1003C80052085343C9F800306368DFF888A2C3F3C2
:1003D800031353441A7ED9F80030DFF87CC2D340A7
:1003E800C9F80030854A864B20ADD360A3690492D2
:1003F80043F00103A361636ADFF86082BB60636A4C
:10040800604643F080736362A3694FF0000B43F0CA
:100418001C03A3614FF6FF7325F82C3D2946CDF840
:100428000CC08DF856B00EF08DFB404629460EF0F4
:1004380089FB744829460EF085FB734928464B68AA
:1004480043F000734B600FF057FE159B6F49049AF9
:10045800B3FBF1F36E490B606E4B4FF47A71C3F83E
:1004680000B0D9F80030DFF8F891B3FBF1F36A492E
:10047800013B4B60F02382F823300723C1F808B012
:100488000B60B368DFF898B1C9F800300AF12803A7
:100498000FCB85E80F00A369159843F00803A36103
:1004A800A36916A943F00803A3610823C8F810300C
:1004B8001023C8F8103004930EF044FB179818A9BD
:1004C8000EF040FBD9F80020049B12F0080F12D060
:1004D8009BF89221012A0ED850499BF893218968EC
:1004E80011F0805B00F0CB8405E04D4B002283F8CF
:1004F800932108F03DFD64200AF02DF8A022494818
:10050800002116F07CF9E369002243F00703E36158
:10051800A36943F4006343F00C03A3613F4B4FF01E
:10052800000B03F10C0102F801B001320E2AF5D1DB
:10053800FF229A76DA761A775A773B4B3B4A594626
:100548001A603B483022D9F8004016F058F959464D
:10055800C4F380180423374ADFF8D4E0885C0C22FF
:100568004A4302F80E00B8F1000F08D11E380128DE
:100578009FBFFF2003F1FF3302F80E00DBB2013109
:100588000429E8D12C4A96F805B013702B4B2C4956
:1005980083F800B02B4B214A3B62C0330B602A4BD7
:1005A800A10603EBCB035B7848BF0123536200230A
:1005B80040F2DC51254A22F813100133082BF7D1F9
:1005C8000EA800211C2216F01AF914F4007304F482
:1005D800006947D0A2040BD4B9F1000F0AD01C4A15
:1005E80096F88601A2F10C01012808BF0A4602E02C
:1005F800184A00E0164A0492149534E000ED00E031
:100608000005FA05001001400000014040420F00BB
:100618007C1200208012002010E000E0C8000020BA
:100628006025002080150020DC22002050270020B3
:10063800E0220020CDBF0108C910002028090020B1
:100648009C16002074250020E4BC0108341000200A
:10065800DC8D0108D08D010800080140000C014024
:10066800002500200493BBF10E0F04D00BF0EF0B14
:10067800BBF1080F02D101228DF84A200120059311
:1006880009F056FD059B18B14088003018BF0120BD
:10069800C4F340028DF83E20C4F3403200F001005C
:1006A8008DF83820C4F3C0328DF83D008DF84080B5
:1006B8008DF83B20B9F1000F07D096F8869109F123
:1006C800FF3EDEF1000949EB0E09003318BF012394
:1006D8008DF842307B6AB6F84801003318BF012311
:1006E8008DF84330C4F300538DF84430B6F84A31DE
:1006F800E504ADF84830B6F85631ADF84E0048BFBD
:10070800BA48ADF84630C4F3804348BFB0F850014A
:100718008DF83F30B6F8543148BFADF84E00B3F508
:10072800FA7FADF84C3084BF0023ADF84E3096F810
:10073800D631AF4887F82830002387F8293043702E
:100748009DF84A30C4F30042002B8DF8412004F094
:100758000101C4F3C0028DF83C908DF839108DF872
:100768003A200CBF0023022301B902B101330AEB7E
:10077800830ADAF838304FF00008A3F102091A3377
:1007880005934FF6FF7339F802AF9A4500F0788168
:100798009DF83D205FFA8AF31AB19A1E012A40F2A9
:1007A8006B819DF8402032B192491A018958924ACA
:1007B800914200F061819DF8412032B18D491A01C2
:1007C80089588D4A914200F057819DF83E2052B1D8
:1007D800884A039802EB03125168814203D11289B7
:1007E800102A00F049819DF83B2052B1814A0398B4
:1007F80002EB03125168814203D11289022A00F0E8
:100808003B819DF83C2052B17A4A7C4802EB0312A6
:100818005168814203D11289022A00F02D81149A6D
:100828007AB1744C116804EB03146068884208D1EB
:1008380021899088884200F01F81D2888A4200F07E
:100848001B814FEA1A2ABAF1020F02D19DF838200B
:1008580004E0BAF1010F04D19DF83920002A00F014
:100868000B81DFF890B19DF844101F010BEB0704D2
:100878005A4631B19DF84A1019B9043B032B40F28E
:10088800E380BAF1010F5FFA8AF341D15C4D3A4433
:10089800FF23517B85F8703085F87130506802F17C
:1008A800080312890026ADF854208DF8561002224C
:1008B80015A985F87460C5F8804006938DF857200F
:1008C80085F82C602E636E63AE63EE6685F8726001
:1008D80085F873600EF036F9069B5BF80700997887
:1008E80032460DF0E3FF2046314652460AF02AFC14
:1008F800444BC5F88C60C5F88430434B2046C5F896
:10090800883005F1840105F188020AF063FCB3E040
:10091800022B46D15FFA88F21C2101FB02FC384AFF
:10092800002502EB0C06334A4FF0010A3A44517B8A
:10093800506802F1080B128986F875808DF85610F8
:1009480086F8765015A986F87E5086F874A0C6F801
:100958008040CDF818C0ADF854208DF857300EF00F
:10096800F1F8244B9BF80210D8592A460DF09EFF47
:100978002046294652460AF0E5FB244A204BDDF87A
:1009880018C0C6F8842003EB0C01214A8431C6F84C
:100998008820C6F88C5020460A1D0AF01BFCD0445B
:1009A8006AE0032B4ED19DF83F30154D194E3BB1EF
:1009B80095F82A70204608214FF6FF72002335E08B
:1009C800BDF84C2095F82A70B2F5FA7FBDF84E3084
:1009D80026D911492046B1FBF2F2082192B20EF055
:1009E800A5F90E4B46F8270025E000BF602500203A
:1009F800F100002040B0010800040040000C014054
:100A0800C800002021E7000801E80008F1E8000814
:100A1800F9E600084C15002000127A0021E80008C9
:100A280067492046B1FBF2F2012192B20EF07EF93D
:100A3800644B46F82700C36095F82A30013385F8DF
:100A48002A3019E0042B17D1BDF846205C4B5E4DC7
:100A580093FBF2F22046BDF84830012192B295F896
:100A680029600EF063F995F8293005EB8606013305
:100A7800C6F8540185F82930059B99457FF481AE65
:100A8800514D524B95F82920002485F87421504A7D
:100A98001C7017789846A7F11702022A19D82B6AF2
:100AA8000021185903EB040912F0FAFC10B16B6A23
:100AB80063BB26E0474E99E80F00264486E80F00FE
:100AC80098F8003010340133C02C88F80030E6D193
:100AD800EDE7414B13F8376003EBC703D3F804E0A5
:100AE80088F80060BEF1000FE1D0B442DFDA394A7D
:100AF800230103EB020C73440FCB01348CE80F0085
:100B0800F3E7364E3368DC0424D41DE0344B354A11
:100B180013F8370003EBC7035C681070002CF0D0A3
:100B280000238342EDDAC3EBC3016218D2F800C098
:100B3800DFF8BCE0013341F80EC001EB0E069188E6
:100B4800B1809279B271ECE707F0EF03082B264BDE
:100B580025D126E098F80030012BF5D9234C04EB79
:100B6800031303F1100810344445EDD054F8100C69
:100B78004FF07C5112F000FB4FF07C5144F8100C00
:100B880054F8140C12F0F8FA4FF07C5144F8140C95
:100B980054F80C0C12F0F0FA44F80C0CE3E70E2FA2
:100BA80008D11A78182F42F010021A7022D10AF0D0
:100BB80027FF1FE01A78192F22F010021A70F5E7A4
:100BC80040420F0011E80008C80000207C150020F2
:100BD8002809002064080020E4BC01080025002042
:100BE80064960108281600200C1100206C080020CB
:100BF800291600200AF0E8FE3368DFF81CB3580312
:100C08005EBFBA4B01221A70B94A0DF15409137824
:100C1800B84F43F004031370B74B4FF0100A93E832
:100C28000300DBF8183089E8030043F00803CBF829
:100C3800183016A915980DF085FF01200BF09EFFBE
:100C48003468524604F400430393384604F40063BE
:100C58000021059315F0D3FD4FF6FF72ADF834204F
:100C680002224FF0000814408DF836208DF83780A6
:100C78000DD020A921F84CADA0480FF0B1FB0423FA
:100C88003B700124072387F80180BC70FB70039B2D
:100C980073B1022320A921F84C3D98480FF0A0FB1E
:100CA8000123E2183B71BB7107237C71FB71D4B23D
:100CB800059B7BB1022320A921F84C3D90480FF0F9
:100CC8008FFB092301223B73BA73631C07227C73D1
:100CD800FA73DCB2DBF804308A4843F44043CBF8BB
:100CE8000430DBF814304FF0000843F00103CBF870
:100CF8001430DBF81830DFF80CA243F40073CBF89B
:100D080018300FF081F9804B012C15937F4B494621
:100D1800169394BF434680231A934FF480731B9312
:100D28004FF480631C9320231D9350464FF40053C7
:100D380018941E93CDF85C80CDF86480CDF87C8043
:100D48000FF044F9DAF80030714A43F00103CAF8A9
:100D580000305368012C23F4702394BF0021012133
:100D680023F4807343EA012353609168694B013C83
:100D78000B4043F4602343F002039360D36AE4B268
:100D880023F4700343EA0454D462012307EB0802F6
:100D9800917800295CD017F80800591C0928C9B2B5
:100DA800D278DFF86CE111D9A0F10A04DEF80CA0C2
:100DB80004EB44044FF0070C0CFA04FC2AEA0C0C70
:100DC800A2404CEA0202CEF80C200EE0DEF81040F9
:100DD80000EB400C4FF0070A0AFA0CFA24EA0A045E
:100DE80002FA0CF22243CEF81020062B484C0ED8FB
:100DF800013B626B03EB83034FF01F0E0EFA03FEF9
:100E080022EA0E0200FA03F3134363631FE00C2B7C
:100E18000ED8073B226B03EB83034FF01F0E0EFA2D
:100E280003FE22EA0E0200FA03F3134323630EE0E3
:100E3800A3F10D02D4F82CC002EB82021F239340C9
:100E48002CEA030E00FA02F34EEA0303E3620B46B0
:100E580008F10408B8F1100F98D12D4B9A6842F4A4
:100E680080729A609A6842F001029A609A6842F029
:100E780008029A609968264A09074FD5FAE7013AA5
:100E8800092A3FF638ABDAF85400C8F81430294676
:100E98002860039804930DF055FE039B3C201A46E6
:100EA8000823136109F057FB049BC8F81030D84693
:100EB80096F893319845BFF618AB114B4FF0080BD5
:100EC800C3F810B00493039B7820C3F814B009F05A
:100ED80037FB049B7820C3F814B0039B08F1010882
:100EE800C3F810B009F02CFBE2E700BF900D00201A
:100EF800943000203C230020188E0108000801408F
:100F0800000C0140080002404C2401404C23002002
:100F180000240140FDF7F1FF00100240936843F000
:100F280004039360AB4B9A6812F00408FAD1AA4FF5
:100F38009A68B7F85C0142F4A0029A60002841F070
:100F48007682B7F95E31002B41F07182B7F96031D2
:100F5800002B41F06C8233689B031FD5C82009F031
:100F6800FAFAAE200BF005FE08B10EF039F89B4CEA
:100F780085F87501C82009F0EEFA994B00210C227A
:100F88002046C5F8783115F03AFC0223E3700EF0DC
:100F9800C0FA09F0B9FA934B0344A36097F86B3190
:100FA800B7F864410593904B97F863B11B6897F8BD
:100FB8006C61B3F85630B7F80CA00693FB7B8B4FE7
:100FC80000210C228A48039315F019FC00211422F1
:100FD800384615F014FC874B00221A700793C5F8A1
:100FE8007C2104F051FD079BDFF840921A4648B374
:100FF800814BB4F5807F3B60804B7B60804BFB600E
:10100800804B3B61804B01D1002116E0BB2C01D9FC
:10101800012112E0612C01D902210EE0292C01D90D
:1010280003210AE0132C01D9042106E0092C01D977
:10103800052102E0002CE7D0062119700123137066
:10104800022322E00790192009F085FA15AB6820E1
:101058000F21012204F034F99DF85430DDF81CC04A
:10106800D32B40F01683694B4E2C3B60684B7B605A
:10107800684B3B6100F007835D2C00F00883362C39
:1010880000F0FF8289F880C10123634A634F3B70F7
:10109800136843F0010313600022614BBBF1090F91
:1010A80000F2F680DFE81BF01000F40010000E00DC
:1010B80079000C000E000A000A00EA001A70D3E05A
:1010C8001A70BDE01A7019E01A704FF0000920ABD1
:1010D80003F82C2D53204946012204F0F1F868B199
:1010E8009DF85430E52B09D1414B4E4A85F8839140
:1010F8001A604D4A5A60022300F01CBC4B4B002278
:10110800C3F87C2104F0C0FC002847D006210A4619
:1011180015AB682004F0D4F89DF8591001F00102CD
:101128009DF8571001F001014B0043EA82019DF838
:10113800552002F001030B430BD05BB2012B01D108
:10114800002202E0022B0FD10122384B83F88421C0
:1011580011E00DAB68200C21012204F0B1F89DF8D4
:10116800343013F00F0303D1052009F0FEF902E033
:10117800042BE9D1E4E71E4B2D4A1A602D4A5A6028
:101188002A4A92F88421002A0CBF6F226E221A7212
:10119800234B01221A700323CCE31A70002220ABE0
:1011A80003F82C2D1C200D21012204F089F80028B9
:1011B80046D09DF854302A2B01D01A2B40D10C4A26
:1011C8001D4911601D495160184A82F88531042370
:1011D800B0E300BF0024014060250020D8110020A2
:1011E800EA260020404B4C0044100020A0160020A6
:1011F800CC240020B4160020A95700089B540008EE
:101208007554000890C1793D000000207558000809
:1012180073550008325C8F3D081100204C000020F7
:10122800BC300020D1580008F5550008C80000203F
:1012380069510008DB540008155800081B550008C0
:10124800002120AB03F82C1D1820012204F038F8E7
:1012580050B19DF85430FB2B06D1C04BC04A1A60E0
:10126800C04A5A60052365E304F062FB38B1BB4B02
:10127800BD4A1A60BD4A5A6008235BE31A70B74B2F
:10128800BB4A1A60BB4A5A6000221A72092351E30A
:10129800BBF1010F3FF618AF1A70042E00F23B8124
:1012A800DFE816F0050042016700050006010A2084
:1012B80009F051F97720A02101220DAB04F000F8C4
:1012C800002856D01E210122772004F0F1F94FF4AE
:1012D8002F6009F035F90026A6F160010025C9B292
:1012E800022215AB77208DF854508DF8555003F035
:1012F800E7FF9DF854209DF855309F4943EA0223A3
:1013080001F5C372B3520236102EE5D1B1F894211B
:101318002B4602F00F0602F47F42A1F894212946D9
:101328000127954D21F001002844B0F886010028D6
:1013380018BF002711F0010F03D0C0B243400820A6
:1013480002E083EA1023FAE713F4004F18BF83F48E
:10135800C05301384FEA4303F6D101311029E0D1D7
:101368003243A5F8942127B9C3F303339E4200F012
:10137800E882814D95F89631002B41F07880142051
:1013880009F0E9F87720D02101220DAB03F098FF8E
:10139800002800F08D809DF834300322552B85F805
:1013A800AF31A5F8B82140F08380D12101220DABDF
:1013B800772003F085FF9DF83430772003F00F0283
:1013C8001B0985F8B02185F8B131162215ABAA2181
:1013D80003F076FF9DF854209DF8553043EA022328
:1013E800A5F898319DF856209DF8573043EA022316
:1013F800A5F89A319DF858209DF8593043EA022300
:10140800A5F89C319DF85A209DF85B3043EA0223E9
:10141800A5F89E319DF85C209DF85D3043EA0223D3
:10142800A5F8A0319DF85E209DF85F3043EA0223BD
:10143800A5F8A2319DF860209DF8613043EA0223A7
:10144800A5F8A4319DF862209DF8633043EA022391
:10145800A5F8A6319DF864209DF8653043EA02237B
:10146800A5F8A8319DF866209DF8673043EA022365
:10147800A5F8AA319DF868209DF8693043EA02234F
:1014880041F27072A5F8AC31012385F896313B4BD7
:101498001A8046F678125A80394A5A60394A9A6050
:1014A800394ADA60394A1A61394A5A6100F0DFBFAD
:1014B800314D95F8BC61002E40F05482142009F09B
:1014C8004AF805F2BD137620D021012203F0F8FE78
:1014D80095F8BD31582B27D105F5E07388211822DE
:1014E800762003F0EDFE31227620F42104F0E0F8B6
:1014F8000123284A85F8BC31204B9A60264A1E8071
:101508005A6045F6D8125A80244ADA60244A1A6189
:10151800244A5A6126E2012E06D0234B234A9E70A4
:10152800136843F004031360204D2B68980702D515
:101538000A4B1B689847039BE4B20F4E1C4A002BCA
:1015480056D02B68B4BB40F2596113F0020F40F239
:10155800712318BF0B467D2135E000BFCC24002045
:10156800AD580008B1550008E95000081D520008A0
:1015780091FC0008ADFC0008C800002058060020B7
:10158800A15700084D540008895700080D54000859
:101598000D500008095000080B500008815700083A
:1015A800C1530008A54D00084C0000200811002078
:1015B8003C2D0020990759BF4FF47A7319464FF410
:1015C800FA634FF47A719A4505DBBAF57A6FA8BFCA
:1015D8004FF47A6A00E09A464B1E5344B3FBF1F38A
:1015E800013BDBB203FB011186F88231116005E093
:1015F8009DF80C30C2F800A086F88231B84FB94681
:101608003B689847059CB74F0023022C3B7004D0D9
:10161800032C19D0002C40F0A781002220AB03F83E
:101628002C2DC6F8DC211E200A21012203F048FED9
:1016380050B19DF85430482B06D1AB4BAB4A1A60D9
:10164800AB4A5A60022393E14FF0000A20AB03F83B
:101658002CAD0C205146012203F032FE002800F088
:1016680009879DF85430482B08D19F4BA14A1A602E
:10167800A14A5A6007233B70032379E1504600F0E2
:10168800F9BE402300E0802389F88031FCE4C023C0
:10169800FAE795F88171002F56D0984B00221A80EE
:1016A800002F40F09380964A802113886B2023F006
:1016B80040031B041B0C1380138823F038031B04FE
:1016C8001B0C43F03003138013889BB243F0400394
:1016D800138004F0C9F9962008F03DFF0321682023
:1016E80004F0C2F9962008F036FF03216B2004F0BD
:1016F800BBF9012008F024FF10216A2004F0B4F996
:10170800012008F01DFF39466C2004F0ADF90120D6
:1017180008F016FF3946192004F0A6F9012008F050
:101728000FFF10211C2004F09FF9012008F008FF8A
:101738001B20182104F098F9012008F001FF714BD3
:10174800012283F8812141E06D4A6B2013888021B2
:1017580023F040031B041B0C138013884FF0060969
:1017680023F038031B041B0C43F030031380138849
:101778009BB243F04003138004F076F9962008F0FA
:10178800EAFE752015A9012204F016F99DF85430D7
:10179800682B05D009F1FF3919F0FF09EED10FE0E8
:1017A8000C2015A9012204F007F99DF85430142BD8
:1017B80006D3182B7FF671AF543B062B7FF66DAF1F
:1017C80004F0B6F8464B002860D180E0B4F5807F7D
:1017D8000ED0BB2C0ED8612C0ED8292C0ED8132C69
:1017E8000ED8092C0ED8002C14BF062700270AE0B3
:1017F800002708E0012706E0022704E0032702E0AB
:10180800042700E005273E4A1920138823F04003E7
:101818001B041B0C1380138823F038031B041B0CB8
:1018280043F03003138013889BB243F040031380C6
:1018380095F8821104F018F9012008F081FE394664
:101848001A2004F011F9012008F07AFE15A804F016
:10185800D9F89DF95630294A013303D19DF95430FE
:10186800013302D013889BB213B100231380A7E77A
:101878001B4B254A64201A60244A5A60244ADA60BD
:10188800244A1A6108F067FEFFF7FEBB224ABB2C08
:101898001A60224A5A60224ADA601E4A1A61214BAB
:1018A80001D901220EE0612C01D902220AE0292C7B
:1018B80001D9032206E0132C01D9042202E0092CE5
:1018C80003D905225A70FFF7DFBB0622FAE7164A4A
:1018D8001A60164A5A60164A9A600823FFF7D5BB61
:1018E800A0160020B830002034060020D1C9000816
:1018F80061C8000861C90008D5C80008F0240020A4
:1019080000380040C8000020F95000080D5A0008AF
:10191800E959000890C1793D79520008E151000861
:10192800BD5100080000002095FC0008B5FC000827
:1019380093FC00082B4A7B70136843F00203136082
:10194800ABE442F21072284B03261A805A80274AC9
:101958005A60274A9A60274ADA60274A1A61274A52
:101968005A61DAE50426D8E5012C07D91C464AE66F
:10197800234AD3702B6843F008032B60214C94F85A
:1019880058310BB1204A137094F859310BB11F4AE2
:10199800137094F85A3103B13B702B68DFF878A0C4
:1019A80013F0080F3AD0BDF918204FF0640B92FBE2
:1019B800FBF73846059211F08BFB059A03900BFB59
:1019C800172000B211F084FB114911F0D5FB039BDD
:1019D8000146184611F0C8FA0E4911F0CDFBCAF8B5
:1019E80000001EE008110020580600207957000862
:1019F800B153000871570008A1530008E94B0008CB
:101A08004C00002060250020B4160020BC300020C7
:101A18008988883C00002041B41400200023CAF8BB
:101A28000030AD4F10223B784FF00A0B43F0020311
:101A38003B70AA4B5A6108221A610397A74F1920D5
:101A4800FB6883F01003FB60FB6883F00803FB600E
:101A580008F081FD192008F07EFD0BF1FF3313F02B
:101A6800FF0BEBD108234FF0100B3B61C7F810B008
:101A78002B681B0709D59A4BC7F814B01B68984701
:101A8800984B0122C7F810B01A70974B974F1B68F4
:101A9800187B11F01DFB964911F06EFB06F0CCFE89
:101AA8008346388811F014FB594611F065FB15F090
:101AB800B3F8904B1880388811F00AFB01468E481D
:101AC80011F00EFC8D4911F00BFC8D4B8849186004
:101AD800D9F8100011F050FB8A4911F04DFB8A4FDC
:101AE8008A4BFF2118601A22384614F088FE3846BF
:101AF800002139702968864B012211F0020F1A70F3
:101B08001FBF7A7003221A70022218BFBA704F07DB
:101B180041BF1A78551C1D70032548BF855411F024
:101B28000A0F0CD01A7804218154511CC9B205251A
:101B38004554D11C02321970D2B206218154754A1B
:101B480011688D0641BF1A78551C1D70072548BFBE
:101B580085540A0608D51A7809258554951C01323A
:101B68001D70D2B20A2585546579082D01D00E2D35
:101B780008D11A7802F1010E83F800E04FF00B0E3D
:101B880000F802E01A78CF0302F1010E4FF00C0CB6
:101B980048BF5F4F00F802C05FFA8EFE48BF0232AE
:101BA80083F800E041BF3A70574A4FF00E0C02F834
:101BB8000EC04A0748BF1A784FF0120C41BF02F115
:101BC800010E83F800E04FF0100E00F802E01A78DA
:101BD8004F0502F1010E5FFA8EFE83F800E000F86F
:101BE80002C00AD594F814723FB1494F02323A70D4
:101BF800454A4FF0130C02F80EC01A788F0502F10F
:101C0800010E4FF0140C48BF414F00F802C05FFAB4
:101C18008EFE48BF023283F800E041BF3A703A4A6C
:101C28004FF0150C02F80EC0182D13D11A784FF08A
:101C3800160E00F802E002F1010E5FFA8EFE4FF078
:101C4800170C00F80EC002F1030E0232D2B283F86C
:101C580000E085540A0341BF1A78511C19701923F2
:101C680048BF8354002198222B4814F0C8FD0EF079
:101C7800AAF82A4A2A4B2B491A6000234B800B7179
:101C8800B4F8980128490A6081B2284A22F813104A
:101C98000133122BF9D11F490B68894613F4805F71
:101CA80004BFB4F89E1111801B0740F1EC8094F832
:101CB8009251062D00F2E180DFE805F004073C6749
:101CC80082A1A10045F2F05201E042F6F822184B39
:101CD8001A800EF001F9CFE094300020000C01408A
:101CE800340600204C060020481700200E00002073
:101CF80035FA8E3C641700200AE81C4100401C4657
:101D080070070020BD3786350D10002044170020CD
:101D18000C1000200025002038220020EA26002090
:101D2800CC0E00201C0E0020643000203C25002032
:101D3800D007002042F6F822794B1A8011F0C8F932
:101D4800784911F019FA784911F00CF911F000FCF2
:101D58000023764A42F823000133122BF9D1744A42
:101D6800744940201160744A137008F0BBFA0028C7
:101D780000F0838001234FF0070A90F9000040210A
:101D88008DE808046D4A6E4B71E042F6F822644B08
:101D980040201A806B4A664B1A60674B10221A70F3
:101DA80008F0A0FA002868D001234FF0000C90F941
:101DB800000040218DE80810634A4FF4E13356E0F3
:101DC80042F6F822564B40201A80604A584B1A6057
:101DD800594B08221A7008F085FA00284DD00123C3
:101DE8004FF0000E90F9000040218DE80840584A55
:101DF8004FF4E13308F0FDFBC6F8E00139E042F6A4
:101E0800F822474B4FF00C0E1A804B4B5148524961
:101E1800524A83F800E0062D4FF0000303700B7060
:101E280013700BD04E4B1B221A704E4B052283F8B1
:101E380000E04D4B4FF4E1351A7008E0484B212281
:101E48001A70484B83F800E0474B1D70474D484ACD
:101E5800374B40201A6008F045FA70B1012300277B
:101E680090F900008DE888002B46424A402108F08E
:101E7800C0FB003018BF012028B9082006F0CEFDAD
:101E88003D4A2B4B1A60D9F800302B4A13F4804F87
:101E98001FBF082111703948254918BF086042F250
:101EA8000101194099B144F620601D490880990440
:101EB80041BF0821117032481D4948BF0860DF073B
:101EC80041BF0C2111702F48194948BF086011788B
:101ED8001D06A1F10401517040F19380DFF8B8A00C
:101EE8000025C6F8E4A1284E29461522274F284880
:101EF80075707560B56014F082FCAAF10503284678
:101F08003B6008F038FF234B02201B68BB46F36098
:101F180008F0E8F9002841D1802006F07FFD68E04C
:101F2800D0070020CDCCCC3F0000B044742F002057
:101F3800300000209D270108D422002041290108F3
:101F4800A08601008927010895280108752701083E
:101F580049280108603000201122002010220020AA
:101F6800332200205F3000203422002090D003006C
:101F780097FC0008BDFC0008F9270108CD270108D7
:101F8800E9270108D92701088C070020AC070020A1
:101F9800B0020020242500205027002045797378BE
:101FA800BC490C2202FB03125278AA4204D0013326
:101FB800DBB2042BF4D900237370DBF8003072789D
:101FC8001B7890F90000002B4FF00C0303FB021361
:101FD80014BF0325012500225B7800950192022198
:101FE80008F007FBAC4B1860002895D0012008F0DA
:101FF800C2FEAA4B1868AA4B00F5C5721A6008F011
:1020080061FFD9F8003098056CD5A64AA64D049B07
:10201800A6482B6093690DA943F001039361049BC3
:102028001B88ADF8343010238DF8363002238DF834
:1020380037300CF087FD2B689C485B880DA9ADF8FC
:10204800343004238DF836300CF07CFD28680F21DD
:10205800037A03F0030203F0FC0303F1804303F562
:1020680080339D689200914025EA01019960996842
:10207800012505FA02F20A439A6042688C4BD14363
:102088005A611E680E401E605E680E405E601E68E3
:1020980016431E609E680E409E60DE683140D9601F
:1020A800996811439960D9680A43DA60437A15A898
:1020B8008DF8543003238DF8553000238DF85630B1
:1020C8008DF857500FF0AEFE7A4B7B4A1B683C3BAD
:1020D80013607A4A136843F010031360784B4FF08B
:1020E800FF321A60774B784A784D1360784A80330C
:1020F8001360D9F800300026D9032E7040F1B28061
:1021080040F22A3B0EF064FBDFF8F0C1654F4FF058
:10211800010A60465A463146CDF810C085F800A03D
:1021280014F06DFBBB696B4843F00403BB614023AB
:10213800ADF8303018238DF833300CA903238DF80F
:1021480032300EF04DF9FB69634943F00203FB613D
:10215800624B634D1B68A7F69477B3FBF1F32988AC
:10216800013B21F45C710904090C29809BB21D21F3
:10217800A9852B85A5F814A02B8C23F001031B043B
:102188001B0C2B842B8CA888298B23F0020321F0AD
:10219800730109041B04090C1B0C41F0600180B297
:1021A80043EA0A03A8802983AE862B842B8B23F06D
:1021B80008031B041B0C43F008032B83B5F84430B9
:1021C8006FEA43436FEA53439BB2A5F84430D7F80C
:1021D800A83F43EA0A03C7F8A83F38460DF014FFA2
:1021E800404BDDF810C0159380231A934FF4807389
:1021F800CDF858C01B934FF0100C4FF400533846DD
:1022080015A9CDF85CC0CDF810C01E9319961C9680
:102218001D961F96CDF860B00DF0D8FEAB89DDF89D
:1022280010C09BB243F40073AB813B680DA843F028
:1022380002033B608DF834C08DF835A08DF8366008
:102248008DF837A00FF0EEFD274B1A68274B43F89F
:10225800282008F10108B8F1200FF5D10CF094FB03
:102268000CF092FBD9F800305A0540F18E80204ED0
:10227800204BD6F828850420C3F8008008F032F8EF
:102288000421C6F82C0508F009F81B4B86F8300520
:10229800082035E0948E0108D41100204410002055
:1022A800200F00200010024088070020000C014089
:1022B8000004014024250020840700200811002084
:1022C80064100020842700201C120020910D00209B
:1022D800181200200008014000366E01500000204E
:1022E8000004004034040040208E0108920D0020B4
:1022F800C8000020FC10002054110020C502002056
:10230800C3F8008007F0EEFF5E4B0821186007F065
:10231800C5FF5D4D86F83105002128462C2214F0B2
:102328006EFA8E236B704FF07C0BE0234FF07D0A22
:10233800EB7085F800B085F82BA0544D2C220021B5
:10234800284614F05CFA8A236B701020A023EB70E7
:1023580085F800B085F82BA0C6F8348507F0C2FFD1
:102368001021C6F8380507F099FF86F83C052020AB
:10237800C6F8408507F0B6FF2021C6F8440507F0E7
:102388008DFF86F848050CF09BFFD9F80030404ACD
:1023980013F4002318BF0123137008F0B5F83D4B60
:1023A80018606379052B02BF3B4B4FF4C8721A8043
:1023B8003A4B4FF47A721A80394BC8221A80394A3C
:1023C800137843F008031370374A137823F0020395
:1023D800137040F60203D9F8002013406BB133495B
:1023E800334B1960334B03211970334B012119709A
:1023F800324900230B8032490B80930341BF314B94
:1024080004221A71DA7844BF42F00102DA702E4BC6
:1024180001229B68C9F800302C4B1A70039B039A61
:102428001B7863F07F03137021B0BDE8F08F284B51
:1024380000221A7000B210F04BFE264910F09CFEE4
:102448001590B7F95E0110F043FE224910F094FE92
:102458001690B7F9600110F03BFE1E4910F08CFE93
:102468001D491790484606F0F1F9FEF774BD02269B
:10247800FFF753B8012C7FF681AA00243870FFF7C4
:10248800CCB800BFA0110020241100205911002051
:10249800382D0020140E002010170020B630002020
:1024A800B03000200C110020BA300020DC260020BB
:1024B800F41000205811002044000020C00F002014
:1024C800C20F0020D811002060250020900D0020A8
:1024D8003800002035FA8E3C18230020834A2DE965
:1024E800F04F1368824C03F59C4320332360A38884
:1024F80089B00133A3807F4B059219689B4611F47C
:10250800804F05D110F0B6FA10B9237B013323733D
:102518000027794BFDB21E78DFF8F481AE4230D93E
:10252800D8F80030072D98BF595D744B88BF2946ED
:102538001B6871489847032D1ED8D8F8002005F16C
:102548000E0302EB83039988DA88A8B14FF47A73F3
:10255800401A5843531A90FBF3F040F6C90300F5AC
:102568007A70984205DC40F2EE239842B8BF1846CC
:1025780001E040F6CA0080B204EB4505E881013766
:10258800C7E7277B0325B7FBF5F50F2384F832301F
:1025980094F8333005EB4505019394F834307D1BEE
:1025A8000393D8F80030DFF870910293EBB20493EC
:1025B8000025B54254DA524B4FEA450833F815A0C6
:1025C800019B53B910F056FA28B1039B002B08BFA2
:1025D8004FF0000A01E0DDF804A0029B988A5045FC
:1025E80002D8D88A50450ED2E8B210F019FA032D55
:1025F8008246DFBF94F832E00120A8402EEA0000AE
:10260800D8BF84F8320010F035FA18B13D4828F8E0
:1026180000A021E0049B94F87E0029F813A028B9B3
:10262800022F15D9324B012083F87E00B9F800003B
:10263800B9F802300344B9F80400034432489BB2A5
:1026480028F800301BB2032093FBF0F39BB200E0A4
:1026580053462C4828F80030013509F10609A8E747
:1026680094F83250224BA5F10F004542454184F8B9
:1026780098503DB19A8811B21429CCBF143A00225F
:102688009A800BE083F83350B54207DAE8B210F0CD
:10269800C7F91C4B23F815000135F5E7DBF80030C6
:1026A800D90405D5194B1B68DA0701D410F016F8C0
:1026B800059B1F68164B1A68907A78B31149137BEB
:1026C800013831F810001BB1C0F53B60083080B20A
:1026D80000B2A0F57A70B0F57A7FA8BF4FF47A708F
:1026E80020EAE07010F0F4FC0A494DE09C3000202C
:1026F800180E002000250020D422002030000020E1
:10270800260E00203C250020980E002008100020EE
:102718006430002000007A444E0E0020DBF80030C0
:102728001B043AD5D4F89C30A64DFB1A002B34DB99
:1027380007F59C432033C5F89C30A34BD27A5979CE
:10274800A24B33F8113095F8A0109BB293FBF2F32B
:10275800013101F00F0285F8A0202A4482F8A13047
:1027680003469B4A825C0130134410289BB2F8D17F
:102778001BB293FBF0F000B26428A8BF642020EAE3
:10278800E07010F0A5FC934910F0AAFD924910F0F2
:10279800F3FC10F0DDFE914B1880DBF80030904D13
:1027A80013F4807F8F4E7FD08F4B9F4204D9237ABA
:1027B80013B9844B01221A72B4F904E03778BEF1D8
:1027C800140FCCBF4FF0000E4FF0010E7D4BC7F336
:1027D8008007BEF1000F06D04FF0000883F80A808A
:1027E80083F8098001E04FF00308D4F8B430A07AE8
:1027F8000193D4F8B8C0B4F90490617AE3882A88C0
:10280800032847D8DFE800F0020E1B36BEF1000FA0
:1028180002D02A8000222BE0002F40F05C862A801C
:10282800A77239E09CF8000000EB8000814502DCCB
:102838002A8001221CE0012067B300F0BBBE47B12B
:10284800019A4FF00208D2896A80AA80BCF8020077
:10285800E8809CF800A09CF80100504400EB800040
:10286800814500F33B86002F00F038862A8002223B
:10287800A27211E02A800322A2726172E3806FB112
:102888003378002243F0020333704E4B5A720FF034
:1028980025FF03E02A80A0726172E380B8F1000F7F
:1028A80002D0404607F0F6FD504FB7F852010FF03E
:1028B8005CFD0197824668B910F028FB4C4B00225A
:1028C800C3F800A0C3F804A0C3F808A0494B1A60D5
:1028D8005A609A6033785F0737D5DBF80030D8063E
:1028E80033D5454B1B78D9062FD4444B1B789BB165
:1028F800019B93F8DE31BAF1000F15D17BB1404B43
:102908001A68D4F8BC309B1A002B08DA0FF0E6FEE0
:102918002C4B83F8C0A018E0BAF1000F0DD110209D
:1029280007F0B8FD01230EE03BB1354A4FF47A7148
:10293800126801FB0323C4F8BC3094F8C03023B1FB
:1029480007F096FD002384F8C030019B93F8DC91D2
:1029580093F8DD11B3F89A71B3F89CE10023184697
:1029680035F913208008BA42C4BF60F07F00C0B2B6
:1029780001337245B8BF40F04000042BF0D194F801
:10298800C130104A834205D192F8C230F92B04D8DD
:10299800013300E0002382F8C230184A84F8C100ED
:1029A8001078084B174F904600283CD13A68D20758
:1029B8002AD5BAF1000F36D13378DB0733D50FF0BB
:1029C800EDFC30E0180E00203C2300204C230020B2
:1029D800B90E00200000C84200C07F4468100020E3
:1029E8003C250020BA300020404B4C0060250020D8
:1029F800D8140020D01B00200C1100200C0000204F
:102A08002425002008100020327850070BD593F8B1
:102A1800332042B15B7A33B911B10FF05FFE02E0A7
:102A2800BAF1000FF9D094F8C2307B4A142BDFF8C2
:102A380018A240F08F8098F8003019F1000918BFEB
:102A48004FF001096BB392F8C1305F2B11D1337885
:102A580003F0040303F0FF0113B10FF03FFE08E099
:102A68000B200391029207F015FD029A039982F850
:102A7800C210B9F1000F14D094F8C1307D2B10D1D9
:102A8800337803F0040303F0FF0213B10FF026FEBE
:102A980007E00B20029207F0FDFC5F4B029A83F8D7
:102AA800C220337803F0040303F0FF01002B51D157
:102AB80094F8C130584A572B16D1584B4FF47A72B4
:102AC8001A80DBF80030190601D508F04BFA544B90
:102AD8001B685A0742BF534A0A21118013F00803A2
:102AE80038D1514A138035E0DBF80000400716D58D
:102AF8005A2B14D14D4B187820B119704C4B012228
:102B08001A7027E092F8C33083F0010382F8C330CB
:102B18000BB10C2000E00D2007F0BCFC1AE05D2B87
:102B280000F0DF845B2B00F0DE845E2B02D10320F3
:102B380000F0DABC562B03D1029306F019FA029B77
:102B480098F80020002A00F0E5846F2B40F0DC8420
:102B58000FF024FCDBF800305B0732D594F8C33063
:102B6800A3B13378580711D5019BB5F90620B3F8FE
:102B78009A319A420ADD3B6813F0010301BF2D4ADE
:102B880032211180244A08BF82F8C3303B68D90338
:102B98000AD5294B1A782AB9244A127812B9254A33
:102BA8003221118001220BE0204A13784BB133788F
:102BB80003F0040303F0FF011BB91D4B1170012240
:102BC8001A70DAF8008000233B6008F17B0608F1F0
:102BD800CB093278737816F8010C9A420BD2314639
:102BE80007F0E8FB38B116F8022C012303FA02F2C9
:102BF8003B6813433B6004364E45EAD10F4B1B78C4
:102C080023B30F4DDFF818802B680E4F13F0020F17
:102C180040F0408338E300BF180E0020B630002093
:102C280008110020B0300020E41000203D170020DB
:102C38003E170020241700203C170020BB3000203E
:102C480008100020D01100204410002008F1CA0606
:102C580008F589773278737816F8010C9A4225D2EC
:102C6800314607F0A7FB08B396F804E00C21B378C7
:102C780001FB0E41B74A013B03EB43031344D1F870
:102C8800C82096F803809A42B3480FD0C1F8C830DC
:102C9800002390F8F420C1F8CC30012303FA0EF396
:102CA80022EA030381F8C48080F8F4300636BE4275
:102CB800D0D1AA4BDFF8B8921F68A94B4FF0000A91
:102CC8001B68029394F833300393D9F80010002955
:102CD80000F0C48291F80080B8F1000F00F0BE82C5
:102CE800D9F80430029AD31A002B0CDB02F5FA73D8
:102CF800C9F8043094F8F420012303FA0AF322EA0D
:102D0800030384F8F430039B002B00F0A78219F822
:102D1800042C4B780432D2B2002B40F06082914BE5
:102D280035F91200B3F8982102F1C80398428A4B8A
:102D380001DD8E7814E0C83A904202DA89784E4272
:102D48000EE093F8F410012202FA0AF221EA0202D4
:102D580083F8F420029B03F5FA73C9F804307DE286
:102D680093F8F42042FA0AF2D20700F17782002E93
:102D7800CCBF02200120049307F0AEFB08F1FF321C
:102D8800049B132A00F26182DFE812F0140021008C
:102D98002E003E0057005E00C30038019D01CA01A5
:102DA800F9015F023E004D005E00C3003801950046
:102DB8000A016F01397838460E44FA2EA8BFFA2660
:102DC80026EAE6763E7007F0DBFA01201AE0797809
:102DD80038460E44642EA8BF642626EAE6767E703E
:102DE80007F0CEFA02200DE0F97838460E44642E3A
:102DF800A8BF642626EAE676FE70D3F8F81007F036
:102E080077FA03203146B7E179790D2031446429F6
:102E1800A8BF642121EAE171797107F015FBB8F1C7
:102E28000D0F00F0128239790E2031446429A8BFB1
:102E3800642121EAE17139719EE1B97905203144B3
:102E480081F30801B97197E1D3F8FC301A78022AA6
:102E580022D13046049310F03BF9434910F040FA70
:102E6800049B596A059310F07FF80021049010F034
:102E780021FB059B48B9049A3C49104610F038FBE1
:102E8800049A059B10B1394A00E000225A620F20CB
:102E9800114607F0C4FA0AE099780F203144C8298E
:102EA800A8BFC82121EAE171997007F0CDFAB8F1FD
:102EB8000F0F00F0CA81284BD3F8FC8098F8003037
:102EC800022B1AD1304610F003F9274910F008FAFE
:102ED800D8F8201010F048F80021064610F0EAFA59
:102EE80030B93046214910F003FB10B11F4E00E005
:102EF8000026C8F82060122061E198F8011012201D
:102F08003144C829A8BFC82121EAE17188F8011015
:102F180032E1D3F8FC301A78022A32D130460493D1
:102F280010F0D6F8114910F0DBF9049B196B0593E2
:102F380010F01AF80021049010F0BCFA059BC8B9EB
:102F4800049A0A49104610F0D3FA049A059B90B1E6
:102F5800064A10E08C920108180E00206C10002020
:102F68002425002060250020000020410000C842E0
:102F7800E00E002000221A631020114607F04FFAD5
:102F88000AE0197B10203144C829A8BFC82121EACA
:102F9800E171197307F058FAB8F1100F00F0558174
:102FA800B34BD3F8FC8098F80030022B1AD1304686
:102FB80010F08EF8AF4910F093F9D8F82C100FF0F4
:102FC800D3FF0021064610F075FA30B93046A949FA
:102FD80010F08EFA10B1A74E00E00026C8F82C6059
:102FE8001320ECE098F80B1013203144C829A8BF2F
:102FF800C82121EAE17188F80B10BDE0D3F8FC3054
:103008001A78022A22D13046049310F061F89A49BE
:1030180010F066F9049BD96B05930FF0A5FF00210A
:10302800049010F047FA059B48B9049A9149104654
:1030380010F05EFA049A059B10B18E4A00E0002257
:10304800DA631120114607F0EAF90AE0997D1120A8
:103058003144C829A8BFC82121EAE171997507F050
:10306800F3F9B8F1110F00F0F080814BD3F8FC8030
:1030780098F80030022B1AD1304610F029F87E4912
:1030880010F02EF9D8F838100FF06EFF0021064620
:1030980010F010FA30B93046764910F029FA10B11C
:1030A800744E00E00026C8F83860142087E098F8CD
:1030B800151014203144C829A8BFC82121EAE1719C
:1030C80088F8151058E0D3F8FC8098F80030022BE7
:1030D8001AD130460FF0FCFF684910F001F9D8F812
:1030E80028100FF041FF0021064610F0E3F930B92F
:1030F8003046604910F0FCF910B15E4E00E0002641
:10310800C8F8286009205AE098F8031009203144CB
:10311800C829A8BFC82121EAE17188F803102BE06B
:10312800D3F8FC8098F80030022B1AD130460FF003
:10313800CFFF504910F0D4F8D8F834100FF014FF2E
:103148000021064610F0B6F930B93046494910F06A
:10315800CFF910B1474E00E00026C8F834600A20C5
:103168002DE098F80D100A203144C829A8BFC821BD
:1031780021EAE17188F80D1007F066F965E0D3F8E7
:10318800FC8098F80030022B1DD130460FF0A0FFCC
:10319800394910F0A5F8D8F840100FF0E5FE0021E5
:1031A800064610F087F930B93046324910F0A0F9D8
:1031B80010B1304E00E00026C8F840600B203146C0
:1031C80007F02DF941E098F817100B203144C82971
:1031D800A8BFC82121EAE17188F81710CCE7012BB4
:1031E80033D135F912308878B3F5617F05DB40F6C5
:1031F80033029342A8BF134601E04FF46173B8F15C
:103208000C0F22D14FF4966292FBF0F0A3F5617394
:1032180093FBF0F31A4ADEB21378B34215D0042EAA
:1032280034BF334602231370019A08FB0323154A5F
:1032380003F2AE73136005F0C5FC4046314607F053
:1032480003F9701CC0B207F047F90949012391F846
:10325800F42003FA0AF3134381F8F4300AF1010A5F
:10326800BAF1040F09F10C097FF42FADC9E400BFCE
:10327800180E00200000C84200007A4400002041D7
:10328800AC2400206C100020DBF80030DB050FD5E3
:10329800637A6BB1D8F800309E0709D53B8813F0E4
:1032A80001060AD10FF032FE012005F0A7FB04E069
:1032B800012005F092FB012300E000232A68500753
:1032C8000CD55BB1012005F088FB3B88990708D431
:1032D8000FF01CFE022005F091FB02E0022005F031
:1032E8007CFB3B88B64A13F0030F4FF0100114BF64
:1032F80051611161D8F8002012F00A0F23D02A6812
:10330800D20609D55E070AD4042005F077FBAD4B39
:103318001B88A4F8003102E0042005F05EFB2B684E
:10332800980606D53B88590606D4402005F066FB6A
:1033380002E0402005F051FB2B685A0642BFA14B22
:103348001B88A4F80231D8F800309B0608D42B68F3
:103358001F0540F18E804FF4807005F04FFB8CE024
:10336800994B1B789E074FD5984B1B78042B4BD94C
:103378002B68974E13F400780ED03B88DC0637D4C0
:10338800102005F03BFB202005F027FB9148011D8C
:1033980007F052FD022327E03C8804F01004A4B291
:1033A8002CB1102005F019FB012486F804812B6844
:1033B800580512D5D6F8083187495A89B1F900302D
:1033C800002BB8BF5B42934207DAB1F90230002BF9
:1033D800B8BF5B429342C0F20F813B88990608D57B
:1033E800202005F0FAFA002386F80431012400E0D1
:1033F800002496F80C31B3B90E2007F04BF8744B43
:10340800012283F80C210EE03B8803F03003002BE7
:103418009DD0102005F0E1FA202005F0DEFA002307
:1034280084F8043101E0002C91D0002006466B4B53
:10343800002423F816406A4B1A1D03F10A0122F8EA
:1034480016400022425001444C608A6023F816401E
:1034580003F132015A334250C250014403444C60D4
:103468008A605C609A601430002E7FF470AF012689
:10347800DDE74FF4807005F0B0FA5A4B5A791C46D4
:10348800082A01D00E2A02D1402005F0A6FADBF85E
:1034980000305A0540F1C58094F8143223B9524BD4
:1034A8001B7813F0040F02E02B6813F4002F0BD0E5
:1034B8004E4B00221A703C200CF056FD002800F0FC
:1034C800B0800DF059FEF6E70BF0FAFE09B0BDE842
:1034D800F04F0CF078BC0120FFF792B90320FFF7FA
:1034E8008FB9012000E002205FFA80F8019A08F104
:1034F800FF3382F8AC3705F0C3FA05F087FB404686
:1035080006F0EAFFFFF726BBB9F1000F02D07E2BC9
:103518003FF41EAB972B05D1354B4FF4C8721A8078
:10352800FFF718BBA72B06D1274A137843F00403EB
:103538001370FFF70FBB0022BB2B079201D10223A8
:1035480003E0B72B04D14FF6FE73ADF81E3009E047
:10355800BE2B01D1022303E0BD2B1AD14FF6FE7317
:10356800ADF81C30DAF80030BDF81C10B3F858205C
:103578000A44A3F85820BDF81E10B3F85A200A448C
:10358800A3F85A2005F0F4FC002384F8C230FFF7B2
:10359800E1BA792B04D1174AD37823F0010306E066
:1035A8007A2B7FF4D7AA134AD37843F00103D37058
:1035B800FFF7D0BA013301469BB20220FFF720B9CA
:1035C800000C0140E41000200C1100201211002012
:1035D800180E002074100020EC100020B2300020DB
:1035E800260F002060250020BA300020D9220020B4
:1035F80010170020D81100203B889B063FF5F9AE34
:10360800202005F0FBF9084B08481A685B68011D83
:103618004360026007F010FC054B012483F8044165
:10362800E7E609B0BDE8F08F141100207C100020F7
:10363800180E0020B54B2DE9F04FB3F90610B44B26
:1036480085B01F6801937A8991420EDBB1F5FA6F54
:10365800FC79BFBF8B1A6343A2F5FA6493FBF4F4B9
:10366800ACBFC4F16404643400E06424A94BAA4AE2
:10367800B3F898B193F9623112689BB20292154679
:103688000393002240F2E630A04B4FEA420C33F994
:1036980012E0CBEB0E0303F2F316864203D8002B9D
:1036A800B8BF5B4201E04FF4FA73022A2ED0029EA3
:1036B80096F811611EB1B342CCBF9B1B0023642056
:1036C80093FBF0F8954E6FF0630A36F818900AFBF2
:1036D800083A08F1010836F918600FFA89F8C8EBBA
:1036E800060606FB0AF696FBF0F68D484E4420F8CF
:1036F8000C60BE183679642073438A4E93FBF6F348
:1037080064339BB2634393FBF0F02CE0029890F88B
:1037180012611EB1B342CCBF9B1B0023642093FBF4
:10372800F0F0DFF82C926FF0630808FB003A39F9E3
:103738001060013039F91000002BA0EB060000FBE7
:103748000AFA9AFBF8FA0398C6EB0A0A0AFB00FA87
:103758007348B8BF5B42A0F804A0B87943437148E6
:1037680093FBF0F064306B784FF06408434393FBAD
:10377800F8F36D4E022AB354EB7A6C4E00FB03F358
:1037880093FBF8F3B3546B7D654E00FB03F090FB9D
:10379800F8F0674B9854674B0ED1DE4583F80280EA
:1037A8000DDB5C4CB4F89A21914214DBB1F5FA6F49
:1037B800A8BF4FF4FA610FE0DE459C5404DA36F8EE
:1037C8000C305B4226F80C300132032A05F1010562
:1037D8007FF458AFE5E71146891A4FF47A735943D5
:1037E800C2F5FA62B1FBF2F1642391FBF3F2DFF860
:1037F80074E16FF063073EF8120007FB0211013213
:103808003EF9122007B2D21B514391FBF3F3034454
:10381800F380494B424D1B885F063BD5474A484BCE
:1038280010881B88181A00B20FF052FC45490FF097
:10383800A3FC074605F000F88046384604F089FFE7
:103848000746B5F902000FF043FC8146B5F90000C0
:103858000FF03EFC414682460FF08EFC3946834607
:1038680048460FF089FC014658460FF07BFB0FF0E5
:1038780049FE4146288048460FF07EFC394680467E
:1038880050460FF079FC014640460FF06DFB0FF0F3
:1038980039FE68802C4D2B68980740F19E8045F2D0
:1038A80007212A4B2A4F1A687B69D31A8B4240F3A7
:1038B80094807A610CF002FF264BDFF8AC901A78FE
:1038C8009846032AB9F8003050D10A2B58D900235A
:1038D800282088F8003006F03EFE0CF0EFFE1E4B64
:1038E80018880CF0D5FE1D4B1A68D37890FBF3F0BE
:1038F800013008281A4BA8BF08201870537980B2E5
:1039080043433B8313795843788339E03C250020AF
:103918006C10002060250020441000205E1200205A
:10392800EC1000200CFEFFFFDC1B0020B60F00206F
:10393800F01B0020B8140020D01100201A0F00201E
:10394800E410002035FA8E3C002500209C30002031
:10395800A80F00205811002054230020F410002044
:103968004400002046120020F81000200A2B07D837
:103978000323954A88F80030002313703B837B8328
:1039880098F80030914A012B0CD002D3022B1BD09F
:1039980023E03A8BB9F800309A421EDD012388F8FB
:1039A80000300FE0B9F800107B8B8B4202DD022358
:1039B80013700FE0864B1B8B0133994202DD002305
:1039C80013700AE0082006E07B8BB9F80020013369
:1039D8009A42E3DC072006F05DFD2D68290575D5C0
:1039E8007C4B7B4F1A68FB69C3EB020845F207233F
:1039F80098456BDDB6F906304FF47A71A3F57A7BFA
:103A0800754BFA61D3F8009098FBF1F899F80A30F1
:103A1800B4F85201012B714E03D040D3022B1FD0B2
:103A28003FE06F4B386A5A7B6E4B4FF0080E33F805
:103A3800122090FBFEF392B2C01A83183B6293FBEC
:103A4800FEF3BA8440F6E4429BB25343B9F8082027
:103A5800C2EB13334B43B9F9062093FBF2F31FE093
:103A6800614BB9F808A01B78C6F800A05A0718D50A
:103A78000EF07BFC20B915F0100F18BF4FF0000BAB
:103A88000BFB0BF1322391FBF3F3B9F906205B44EE
:103A98005A434FF47A7392FBF3F3534400E0002344
:103AA80033603368D7E90A0103FB08F84FF47A73E7
:103AB80098FBF3F810EB080041EBE8710023C7E925
:103AC8000A014A4A0FF064FD494B1860494E3368B1
:103AD800DB0427D52F0622D5474B1B789D071ED51B
:103AE800464B187804281AD90022454B0521D718C7
:103AF800951C4FF00A0E122AD154E9B287F801E05A
:103B080004D0B0EB510F2A46EFD800E014215A1820
:103B1800322002F8010CFF225A540F2000E00A203C
:103B280006F0B8FC374D2A68002A45D0364B374F87
:103B380018683968984681423ED8354BDFF8DC90E2
:103B480018785168B0B901221A70B9F80030CB5C06
:103B5800D3B1304B1A700EF099FFB9F800309BB909
:103B68002B681B78053B012B0ED806F0CDFC2A4BA1
:103B7800186009E000221A70B9F80030CB5C1BB15C
:103B8800244B1A700EF082FF2B68B9F800205B688E
:103B980022499B5CFE2B02D100230B800CE0FF2BFB
:103BA80002D106F065FC07E0D8F800000A2505FBFD
:103BB800030301323B600A800B4D2B78580731D53F
:103BC800174B08225A616BE044000020581100206E
:103BD800A80F00209C300020F410002000110020C5
:103BE8003C2300204C230020BA300020407E0500F2
:103BF80004110020081000200C11002012110020D0
:103C0800D8240020781200202425002070120020DB
:103C18006C12002068300020F42E0020741200205E
:103C2800000C01403268D1075CBF43F001032B70E0
:103C3800984B1B781F075EBF2B7823F001032B706E
:103C4800D60248BF2B78944A44BF23F001032B7057
:103C5800924B1B6813F0040F02D09149098851B99F
:103C68009049098809B1980705D48F4B1B88003300
:103C780018BF012333B1022313702B7823F00103FB
:103C88002B7004E02978C90758BF0223137006F087
:103C98003BFC864B1B68C01A002801DB0EF0F6FEC1
:103CA8000BF00EFB824B1E789846002E00F0AB807E
:103CB800804E3368002B00F0E286306806F0F6FC90
:103CC800002800F0DC867B4B7B4C186806F0EBFC88
:103CD800092801D03F2850D14FF0000A5746D4F8A0
:103CE8000090764DB9F1000F05D0754829684A460D
:103CF80012F0D2FD10B9AA4607B92F46714B1035FC
:103D08009D42EFD3C7B1D7F800E0DAF800C02368C6
:103D18001EF803501CF80300A8420DD15A1C68492C
:103D280038B92D2B05D8644D2A602025CD548854E8
:103D380002E0CD542260EAE723680BB1574511D061
:103D480061480DF009FB574507D857F8100B0DF0DF
:103D580003FB09200DF0F8FAF5E75C480DF0FCFAD2
:103D68004FF0000923689945A7D2554B13F809006D
:103D78000DF0EAFA09F10109F4E72368002B40F095
:103D88006386042840F0A1864D4803F05DFC00F0EE
:103D980076BED9F80000DFF844A106F087FC40B3EE
:103DA800DAF8000006F07FFCDBF80030024693F8F2
:103DB8004810002935D1242840F09280012283F848
:103DC8004820DBF80030DFF810A193F84820062AD5
:103DD800DFD193F8490001F06DFE8146002800F01C
:103DE800A3803B6898790DF004FA3B68002283F8B9
:103DF8004820374B93F83530002B40F013864C366B
:103E0800982E00F03C86334BF21892F84A1001299C
:103E1800F5D1314FF3583A60304ABB4613609146AA
:103E2800B7E7012904D14D2814BF00220222C6E7B2
:103E3800022904D13C2814BF00220322BFE703292A
:103E48000CD140284FF0000102D983F84810B8E798
:103E580058711971D97198710422B0E7042906D1F3
:103E6800997983F849004A409A710522A7E70529FC
:103E7800A7D1587919798842987906D9504098710C
:103E8800481C18710B441A729BE790420CBF06221B
:103E9800002294E70C11002068300020081100204F
:103EA800B030002010170020B63000206C30002001
:103EB800BB300020C8240020141200205C940108A4
:103EC800E41100200C96010847B401084CB401081D
:103ED800A80F002038220020B0110020B4110020C3
:103EE8002B7858073FF56DAF232ADAF800300ED14A
:103EF800012188F80010CF49CF480B60CF490292C2
:103F08000B630DF029FACE480DF026FA029ACD4B34
:103F18001B681B78934201BFCB4ACC4B1A60CC4A32
:103F280004BFCC4BDA604CE7DAF8002092F849304D
:103F38004C2B00F066845DD8332B00F09D8421D88B
:103F4800292B00F02A8409D8252B00F00184272B7F
:103F580000F00584232B40F0B4852CE22D2B00F0D3
:103F68002D8407D82B2B40F0AC850DF025F9607116
:103F780000F03BBD2F2B00F0EB84312B00F0FD84CB
:103F880000F09FBD3E2B00F0F2801DD8372B00F0CB
:103F9800A78404D8352B00F0478200F092BD392B56
:103FA80000F0EA833C2B40F08C85DFF8AC92D9F81E
:103FB80000A00DF001F98AF80000D9F8003018784F
:103FC80008F048F900F011BD432B00F0668406D8CC
:103FD800412B40F076854FF0000900F052BC442B8D
:103FE80000F0FF844A2B40F06C850DF0EFF8A081BB
:103FF80000F0FBBCD02B00F00D8355D8CA2B00F085
:10400800C08009D8C82B00F0858000F23B834E2B76
:1040180000F0048400F055BDCD2B00F0068304D8D1
:10402800CC2B00F0298200F04CBDCE2B00F006838B
:10403800CF2B40F046850DF0C9F86FF4AF628318B6
:104048009BB2C62B98BFA4F898010DF0BFF8A4F84E
:1040580044010DF0BBF8A4F846010DF0B7F8A4F838
:1040680048010DF0B3F8A4F8DA010DF0A5F884F8CA
:10407800EB010DF0A1F80DF09FF884F8EC010DF0BC
:104088009BF884F887010DF097F884F894010DF0F7
:1040980093F8714BD3F800900DF098F800EB80007E
:1040A8004000A9F8560067E3D62B00F038820AD8FA
:1040B800D22B19D0C0F00D83D32B25D0D42B00F0F0
:1040C800398200F0FEBCEF2B41D005D8D82B40F048
:1040D800F8844FF0000901E1F22B00F07382FA2B0B
:1040E80000F0B58200F0EDBC2B78590700F17D8413
:1040F8000DF062F8022884F8AC0740F29182574B21
:10410800002283F8AC278BE20DF060F8544B18803E
:1041180000F06BBC92F805904FEA5909B9F1120FFB
:1041280003D90BF01DFF00F060BC4FF0000ACA4530
:1041380007D20DF04BF84B4B23F81A000AF1010A8D
:10414800F5E73E4B012283F8342000F04EBCDFF83F
:104158000891D9F800A00DF039F8AAF85A00D9F852
:1041680000900DF033F8A9F8580000F03EBC0DF0AF
:1041780023F884F8DE010DF01FF884F8DD0100F063
:1041880034BC354B1A689A461278022A40F08B8064
:10419800DAF8003009F1080B02930DF00DF80EF073
:1041A80093FF31490FF09CF8029B43F82B00DAF893
:1041B80000B00DF001F809F10A030BEB830B0EF0C8
:1041C80083FF2A490FF08CF8DAF80030CBF80400A6
:1041D80002930CF0F1FF0EF077FF25490FF080F8FD
:1041E80009F10E0B029B09F10109B9F1030F43F81C
:1041F8002B00CDD1B9F1070FDAF800B03AD10CF0A5
:10420800DBFF0EF061FF18490FF06AF8CBF84400A5
:10421800DAF800B00CF0D0FF0EF056FF12490FF09C
:104228005FF8CBF84800DAF800B00CF0C5FF8BF85F
:104238004C0032E0C82400207CB40108A80F0020FC
:104248004CB40108DC220020EFBEADDEF04F0020A8
:104258000400FA0500ED00E044100020602500206D
:10426800180F00203C250020000020410000C84213
:1042780000007A440CF0A0FFCB448BF80100DAF878
:1042880000B00CF099FFCB448BF80B00DAF800B0C3
:104298000CF092FFCB448BF8150009F10109B9F134
:1042A8000A0FA7D1A1E3DAF800B00CF085FFCB44E0
:1042B8008BF80100DAF800B00CF07EFFCB448BF8E5
:1042C8000B00DAF800B00CF077FFCB4409F10109D4
:1042D800B9F10A0F8BF81500E5D186E3DFF890A352
:1042E80009F1080BDAF8003002930CF06FFF0EF0BA
:1042F800EBFED9490EF0F4FF029B43F82B00DAF8E5
:1043080000B00CF063FF09F10A030BEB830B0EF00E
:10431800DBFED1490EF0E4FFDAF80030CBF80400F8
:1043280002930CF053FF0EF0CFFECB490EF0D8FFEE
:1043380009F10E0B029B09F10109B9F1030F43F8CA
:104348002B00CBD1B9F1070FDAF800B01AD10CF075
:104358003DFF0EF0B9FEC0490EF0C2FFCBF8440095
:10436800DAF800B00CF032FF0EF0AEFEBA490EF0EB
:10437800B7FFCBF84800DAF800B00CF027FF8BF84D
:104388004C0012E00CF022FFCB448BF80100DAF865
:1043980000B00CF01BFFCB448BF80B00DAF800B030
:1043A8000CF014FFCB448BF8150009F10109B9F1A1
:1043B8000A0FC7D119E30CF0FFFE132883463FF616
:1043C800B0AEDFF8ACA2DAF800900CF0F5FE0023EE
:1043D800A2490C2202FB0312117A814220D11378E0
:1043E80009EB8B0989F879300CF0E6FE89F87A0038
:1043F8000CF0E2FE89F87B000CF0DEFE984A994B3F
:1044080089F87C001A60DAF80000974B00211860E0
:10441800793005F0F3FF954B80F001001870E4E265
:1044280001331B2BD4D17CE60CF0C6FE0B28824648
:104438003FF677AE8E4BD3F800900CF0BDFE032804
:104448003FF66FAE062303FB0A9989F8CE000CF0FD
:10445800B3FE89F8C9000CF0AFFE89F8CA000CF069
:10446800ABFE89F8CB000CF0A7FE89F8CC000CF065
:10447800A3FE89F8CD00B8E25379092B7FF651AE37
:10448800019BD3F800900CF097FE019B89F800007F
:10449800D3F800900CF090FE89F801000CF08CFE27
:1044A800019B64281B68A8BF642018710CF084FE67
:1044B800019B64281B68A8BF642058710CF07CFE1F
:1044C800019BFF281B68A8BFFF2098710CF074FEA1
:1044D800019B6428D3F8009028BF642089F807005E
:1044E8000CF06AFE019B89F80200D3F800900CF0EA
:1044F80063FE019B89F80300D3F800900CF066FE78
:104508003B68A9F80A005B790A2B40F26E82594B86
:10451800D3F800900CF050FE89F8080065E20CF022
:1045280055FE554B23F8190009F10109B9F1080F97
:10453800F5D15AE253790F2B7FF4F3AD0CF03CFE22
:10454800072881463FF6EDADDFF824A1DAF800B080
:104558000CF03CFE0E2303FB09F9CB44ABF8190120
:10456800DAF800B00CF032FECB44ABF81B01DAF8F5
:1045780000B00CF02BFECB44ABF81D01DAF800B00C
:104588000CF01AFECB448BF81F01DAF800B00CF0DF
:1045980013FECB448BF82001DAF800B00CF00CFEC7
:1045A800CB448BF82101DAF800B00CF005FECB44BF
:1045B8008BF82201DAF800A00CF012FED144C9F8F9
:1045C800230112E20CF0F8FD0F2881463FF6A9AD51
:1045D8000CF0F2FDC9EBC909A14489F8D4000CF02C
:1045E800EBFD89F8D5000CF0E7FD89F8D6000CF052
:1045F800E3FD89F8D7000CF0DFFD89F8D8000CF04E
:10460800DBFD89F8D9000CF0D7FD89F8DA0007F04E
:10461800F7F9EAE12B785B0700F1E7810DF0C8F8BC
:1046280004F02EFA04F0F2FADFE12B78580700F1D3
:10463800DC81124B4FF4C8721A80D6E12B785907E7
:1046480000F1D3810E4A137843F004033FE02B783E
:104658005A07E5D535E200BF00007A44F892010810
:10466800A4260020100F0020140F00200C000020AA
:10467800441000206C100020AE24002010170020E9
:104688000C1100200CF098FDDA4B1A7810B142F0AA
:10469800020201E022F002021A700CF08DFDD64BE6
:1046A800DFF8789318700CF09BFDC9F800000CF047
:1046B80097FDC9F804000CF089FDD04B18800CF068
:1046C80085FDCF4BCF4A1880137843F0020313704F
:1046D8008BE10CF071FD02900CF082FD83460CF02A
:1046E8007FFD82460CF07CFD81460CF06FFD0CF0DE
:1046F8006DFD0CF061FD029BA3B9C34B1020C3F8FC
:1047080000B0C3F804A004F068F9BA4A137843F07B
:1047180001031370B9F1000F00F06781BB4BC3F8B8
:10472800009062E1102B40F06081B94BC3F800B0F3
:10473800C3F804A0B9F1000F02D0B44BC3F800903D
:10474800B348B44B0222011D1A7006F075FB4CE108
:10475800A0600CF045FDA3681843A06045E10CF08B
:1047680035FDA4F85C010CF031FDA4F85E010CF0F5
:104778002DFDA4F8600138E10CF01EFD84F87C01E1
:104788000CF01AFD84F880010CF016FD84F87F0106
:104798000CF012FD84F8810127E10CF017FDA4F854
:1047A80082010CF013FDA4F884010CF005FD84F8D7
:1047B80086010CF00BFDA4F8880116E10CF0FCFC56
:1047C80084F892010CF002FDA4F89C010CF0FEFCA8
:1047D800A4F898010CF0FAFCA4F89A010CF0ECFC8F
:1047E800DAF8003084F893015B79082B40F2FD80F9
:1047F8000CF0ECFCA4F89E010CF0E8FCA4F8A00175
:10480800F3E00CF0D9FC84F8D8010CF0D5FC84F85E
:10481800D9010CF0DBFCA4F8DA01E6E092F8059087
:104828000323B9FBF3F9B9F1120F3FF67AACDFF8BD
:10483800F0A14FF0000BCB4580F0D7800CF0BCFC0A
:104848008AF8A2010CF0C2FC40F2ED23984205DD83
:1048580040F6CA039842A8BF184601E040F2EE208D
:10486800A0F2EE20192390FBF3F00BF1010B8AF86C
:10487800A3010AF1020ADEE70CF09EFC84F8940119
:10488800B3E00CF099FC04EB090309F10109B9F153
:10489800080F83F88A01F4D1A7E00CF08DFCC4F866
:1048A800089060710CF09CFCA3681843A0600CF0A1
:1048B80083FC84F892010CF089FCA4F85C010CF0EC
:1048C80085FCA4F85E010CF081FCA4F860010CF0F2
:1048D8007DFCA4F882010CF079FCA4F8840184E042
:1048E80053794FF0070AB3FBFAF2C2EBC2029A1AE5
:1048F80012F0FF0F7FF415ACB3FBFAFA0AF1FF3A96
:104908005FFA8AFABAF1FF0F6FD00CF055FC5FFA24
:1049180080FB4FFA8BF005F00BFC814600283FF432
:1049280000AC80F800B00CF051FCA9F802000CF0C3
:1049380043FC89F804000CF03FFC89F805000CF0F2
:104948003BFC89F807000CF037FC89F80600D5E72E
:10495800DFF8CC9009F1400A0CF038FCA9F8A40261
:104968000CF02AFC89F8A6020CF026FC09F10409CF
:1049780089F8A302D145EFD137E00CF01DFC1F28C0
:1049880081463FF6CEAB3B685B79082B7FF4C9AB19
:104998000CF01CFC09F1880904EB890900F03F00C0
:1049A800A9F806000CF012FCB9F80630800100F4F2
:1049B800FE501843A9F806000CF0FEFB000189F828
:1049C80004000CF0F9FB99F8043000F00F001843CC
:1049D80089F804000CF0F0FB89F805000BF0F8FEEC
:1049E80003E00D4B012283F8352000200CF030FC49
:1049F800FFF7F7B90C110020121100201011002048
:104A08000E11002072100020741000208410002065
:104A18007C1000201C0F0020A80F0020141100207B
:104A2800602500205B4B985905F02CFE18B9322000
:104A380005F091FDF6E706F0A3FF03F0F7FF564AED
:104A4800564BDA60FFF7DBB90C2840D00A2847D16B
:104A5800534D54480CF080FC2846232111F005FFE3
:104A680008B1401B20602368002B5CD14C48002112
:104A78003022236011F0C3FE98F8003053BB4A4B34
:104A88001B689B0614D5494B49491B688A6B9A1ABF
:104A9800002A0DDB474A1278042A09D903F5123394
:104AA80003F5F873444A8B63D36883F01003D3602B
:104AB800424B9B68002B69D0414805B0BDE8F04FD8
:104AC80018470BF04DFAFFF78CB90C2804D13D4874
:104AD8000CF042FC3C480DE07F2812D1FFF7EDB8FE
:104AE8000D28B5D07F2809D12D4A013B0021374830
:104AF8002360D1540CF030FCFFF7DFB82F2B3FF6C2
:104B0800DCA8A0F12002D2B25E2A3FF6D6A813B9DB
:104B180020283FF4D2A85A1C2260214AD0540CF015
:104B280013FCFFF7CAB85A1EA95C202901D1134605
:104B38009AE71B4A00212360D154254B254DD3F811
:104B480000A0D5F800B0DFF85890584611F09BFE49
:104B5800074659463A46484611F09EFE1E4A28B96D
:104B680019F8073053445B785B0703D0103595423A
:104B7800E7D306E0954204D2781CEB68484498478E
:104B880002E016480CF0E8FB00236FE705B0BDE82B
:104B9800F08F00BF382200200400FA0500ED00E085
:104BA800E411002000C10108081100209C300020F9
:104BB800A80F002012110020000C0140A0160020B0
:104BC800E40F002051B401084CB4010878B401087E
:104BD800580000205C9401080C9601085CB4010898
:104BE8006B4B6C4A2DE9F04F5E8914684FEA062A30
:104BF800B4EB0A0A9C884FF000054FEA04481C8968
:104C08004FF0000BA4FB0A6765EB0B0B04FB0B775B
:104C1800F40944EA476418EB04065C884FF000097D
:104C28004FEAE7154FEAC438DC8849EB050787B037
:104C3800CDE90467A4FB0A6704FB0B77340A44EA4E
:104C4800076418EB04064FEA27259C894FF00009F2
:104C580049EB0507CDE90067AAFB046704FB0B775E
:104C6800F40D44EA472414F5FA664FEAE75545F18E
:104C78000007B6F5FA6F77F10003CDE902679646AB
:104C880066DADDE90489A4FB046704FB05F34FF049
:104C9800050C07EB4307A6FB0C230CFB07335F103F
:104CA8004FEA3206B8EB06084FEA920646EA8376E0
:104CB80069EB07099F10DDE90023921B63EB0703EB
:104CC800CDE90023DDE90267334A4FF0FF3396420E
:104CD80077EB0303CDE9048927DA40F6AC520023C9
:104CE800A4185D4104FB05F3A4FB04456FF006021C
:104CF80005EB4305664202FB0566A4FB0223334429
:104D080018EB020649EB0307CDE904670B26A4FB61
:104D1800062306FB0533DDE900455B104FEA320246
:104D2800A41A65EB0305CDE90045DDE902450AFB58
:104D38000BF3AAFB0AAB0BEB430B4FEADA7242EA1E
:104D48004B02A41A4FEAEB7365EB0305CDE9024564
:104D5800DEF80440009B019DA4FB032304FB0533FC
:104D68004FEA525848EAC3284FEA6359DDE9042359
:104D7800B8EB020269EB03039946D30B43EA4943B4
:104D880000B1036009B1029B0B6007B0BDE8F08F6A
:104D98004E020020E80F002024FAFFFF2DE9F04F13
:104DA800DFF8589285B00746D9F808000E460EF08D
:104DB8008FF98E4C804620880EF086F94FF05C51B2
:104DC800054640460EF0D8F94FF064518246284611
:104DD8000EF0D2F9014650460EF0C4F84FF0625179
:104DE800824640460EF0C8F94FF06A518046284680
:104DF8000EF0C2F9014640460EF0B4F80546B4F983
:104E080002000EF065F9014628460EF0B5F9514644
:104E1800054650460EF0B0F98046B4F904000EF08D
:104E280057F9014640460EF0A7F9014628460EF00C
:104E38009BF880460EF066FB6D490546A06140462A
:104E48000EF04EFAD9F80C308046284601930EF041
:104E58003FF94FF07C510EF08FF966490EF082F859
:104E68000546E389B4F90A0002930EF031F92946A0
:104E78000EF082F929460EF07FF94FF058510EF0E6
:104E88007BF98146B4F90800B4F810B0B4F80CA066
:104E98000EF01EF929460EF06FF9014648460EF04D
:104EA80063F84FF058510EF067F94FF060510EF06B
:104EB80063F94FF07E510EF057F88146E0880EF006
:104EC80003F9014648460EF057F9002181460EF0D5
:104ED800E7FA00287BD1294628460EF04DF90390C1
:104EE8000FFA8BF00EF0F4F8039B014618460EF00B
:104EF80043F94FF060510EF03FF98346BDF90800C1
:104F08000EF0E6F8014628460EF036F901460EF096
:104F18002BF8014658460EF027F84FF07A510EF05C
:104F28002BF9834601980EF0D3F801464FF09340D1
:104F38000EF018F805460FFA8AF00EF0C9F84FF08F
:104F48008F410EF019F9014658460EF00DF84FF052
:104F580066510EF011F9014628460EF003F826496D
:104F68000EF00AF949460EF0BBF90546B4F91600E9
:104F78000EF0AEF829460EF0FFF829460EF0FCF8C0
:104F88004FF040510EF0F8F88146B4F914000EF0D5
:104F98009FF8014628460EF0EFF84FF060510EF0EA
:104FA800EBF8014648460DF0DFFF8146B4F91200E0
:104FB8000EF08EF8014648460DF0D6FF4FF07651B8
:104FC8000EF0DAF8014628460DF0CEFF00E000208A
:104FD80017B10EF097FA38602EB140460EF092FAEB
:104FE80064235843306005B0BDE8F08F8802002084
:104FF8000000A04500007A470050C345E80F002094
:10500800704770472DE9F041324C334D62892B8A45
:10501800B4F904809A1A2389B4F902E05A43B4F91E
:105028001230D613B4F91420DB02324493FBF2F2A7
:1050380032440A26E2615643A2F57A6202FB02F381
:10504800B4F90EC002FB0EFE02FB08F2B4F90C80A4
:105058001B130CFB03FC03FB08F31B1403EB62326A
:105068000232E388921002F5004253434CF2503268
:10507800B4F920704FEAEE2EB4F900400EEBEC2C98
:105088000CEB8404BC406D690234A5EBA4043A41DE
:1050980062434FEAD3384EBFB2FBF8F35400B4FB77
:1050A800F8F340F6DE3448BF5B001A1252436243FD
:1050B8000A4C08365C43241404EB224202F6CF6201
:1050C800361103EB221300B1036001B10E60BDE895
:1050D800F08100BF60020020E80F002043E3FFFFDB
:1050E800024B4FF480521A80704700BF0E00002018
:1050F8007047064A08B5138801339BB21380044BE6
:10510800187807F03BFD002008BD00BF06100020FE
:10511800B01700200F4B13B51A7E1C46C2B90E4BB0
:105128001B68ABB11A681AB10C49886902438A61D5
:105138009A889868ADF8042002228DF80720042286
:105148000DEB02018DF8062009F0FCFC0123237603
:1051580002B010BDE80F00204402002000100240F9
:1051680008B5FFF7D7FF074B1B7813B1012B03D006
:1051780008BD4FF4006201E04FF48052024B1A80E0
:1051880008BD00BF4C0200200E000020F8B50F46F5
:105198001646074C4FF48055656140F080000CF0CE
:1051A8005FFE384631460CF081FE2561F8BD00BF30
:1051B800000C014013B501220DF107010446382007
:1051C800FFF7E4FF052005F0BBF99DF8073003B1B0
:1051D8000123237002B010BD13B50446694643206D
:1051E8000622FFF7D3FF9DF800209DF8013043EA1F
:1051F800022323809DF802209DF8033043EA02230E
:1052080063809DF804209DF8053043EA0223A380BB
:1052180002B010BD13B5044669463B200622FFF7CD
:10522800B5FF9DF800209DF8013043EA0223238052
:105238009DF802209DF8033043EA022363809DF81D
:1052480004209DF8053043EA0223A38002B010BD74
:1052580070B50E46054C4FF4805565610CF000FEA4
:1052680030460CF0FDFD256170BD00BF000C01400B
:1052780008B580216B20FFF7EBFF642005F06BF980
:1052880000216B20FFF7E4FF642005F064F96B2030
:105298000121FFF7DDFF1B201821FFF7D9FF1C2094
:1052A8001021FFF7D5FF054B1A201978FFF7D0FF1B
:1052B800BDE8084019200021CAE700BF010000200E
:1052C80010B54000204CC0B220702048204C01701E
:1052D800204800210170012020701F4C23601F4CC2
:1052E80023601F4B1A701F4A1F4B107019701F49FB
:1052F800086811461A4630B383889C0515D403887C
:10530800DB050DD447F230530488A40502D5013BD0
:10531800FAD112E08BB103889BB243F48073038007
:1053280083889BB243F44073838047F230530878F4
:1053380010B1013BFBD100E013B9BDE81040D8E63D
:10534800107880F0010010BDB6170020B4170020B7
:10535800B2170020BC170020B8170020C017002083
:10536800B5170020C4170020C5170020AC1700206F
:1053780007B5002101AB03227720FFF7A1FF9DF8B5
:1053880005309DF804001B0243EA00439DF806001F
:10539800184303B05DF804FB08B5FFF7E9FF014BBC
:1053A800586008BDE80F002008B5FFF7E1FF014B82
:1053B800186008BDE80F002007B5F7216B460622E4
:1053C8007620FFF77DFF9DF800309DF801101B0344
:1053D80043EA01139DF80210094A43EA1113D36006
:1053E8009DF803309DF804101B0343EA01139DF850
:1053F800051043EA1113936003B05DF804FB00BF86
:10540800E80F002007B5F62101AB03227720FFF74C
:1054180057FF9DF805309DF804201B0243EA02431C
:105428009DF806201343054AB2F92020C2F108026C
:10543800D340034A536103B05DF804FB60020020C7
:10544800E80F002007B5F62101AB02227720FFF70D
:1054580037FF9DF804209DF8053043EA0223024AED
:10546800138203B05DF804FBE80F002013B5012296
:105478000DF107033A2104466820FFF721FF0520B4
:1054880005F05EF89DF8073003B10123237002B0E0
:1054980010BD13B506220446432168206B46FFF76A
:1054A8000FFFA0B19DF800209DF8013043EA0223C8
:1054B80023809DF802209DF8033043EA022363808D
:1054C8009DF804209DF8053043EA0223A38002B02A
:1054D80010BD13B5062204463B2168206B46FFF732
:1054E800EFFEA0B19DF800209DF8013043EA0223A9
:1054F80023809DF802209DF8033043EA022363804D
:105508009DF804209DF8053043EA0223A38002B0E9
:1055180010BD13B5062204466B4601211C20FFF777
:10552800CFFE9DF801309DF80020042143EA0222B5
:1055380042F38D0292FBF1F29DF8023022809DF831
:10554800032042EA032242F38D0292FBF1F29DF816
:10555800043062809DF8052042EA032343F38D035B
:1055680093FBF1F3A38002B010BD13B504466B465C
:10557800A82106226820FFF7A3FE9DF800209DF8C9
:10558800013043EA022323809DF802209DF803306E
:1055980043EA022363809DF804209DF8053043EA1E
:1055A8000223A38002B010BD13B504466B46022146
:1055B80006221820FFF784FE9DF800309DF8012090
:1055C8009B0803EB022323809DF802309DF80320FB
:1055D8009B0803EB022363809DF804309DF80520A7
:1055E8009B0803EB0223A38002B010BD2E4B2DE9CC
:1055F800F3411B780546002B38D000242646274661
:10560800A04608226B4653203221FFF759FE9DF829
:1056180001209DF80030013403EB02231BB29DF8F2
:10562800032098449DF80230E4B203EB02231BB236
:105638001F449DF805209DF80430202C03EB02231D
:105648001BB21E449DF8073003F07F0301D0002BE6
:10565800D7D198FBF4F897FBF4F796FBF4F6134BC5
:10566800A5F800806F80AE805C761AE006226B4653
:1056780053203221FFF724FE9DF801209DF80030C9
:1056880003EB02232B809DF803209DF8023003EBE7
:1056980002236B809DF805209DF8043003EB02235C
:1056A800AB8002B0BDE8F0814B020020E80F00207B
:1056B80013B502AB03F8012D4000214AC0B21070A7
:1056C800204A00201170204901220A701F490870E1
:1056D8001F490B601F490B601F4B20491A700A7045
:1056E8001F4B204A187010681A4630B383889C05EF
:1056F80015D40388DB050DD447F230530488A4057C
:1057080002D5013BFAD112E08BB103889BB243F476
:105718008073038083889BB243F44073838047F28D
:105728003053087810B1013BFBD100E013B9FFF703
:10573800E0FC02E0107880F0010002B010BD00BF6C
:10574800B6170020B4170020BC170020B21700209D
:10575800C0170020B8170020B5170020C417002074
:10576800C5170020AC1700207720482101229FE7A9
:105778007720582101229BE77620F421312297E7F0
:10578800044B772093F82020F4219201343202F060
:10579800FC028DE7600200207720F4212E2287E7A3
:1057A80008B5FFF7B7FC6B2180226820FFF780FF60
:1057B800642004F0D0FE6B2103226820FFF778FFF5
:1057C8000F2004F0C8FE0F4B19211A786820FFF744
:1057D8006FFF0F2004F0BFFE0B4B1A211A786820C8
:1057E800FFF766FF1B2118226820FFF761FF1C21C5
:1057F80010226820FFF75CFFBDE8084068203721C9
:10580800022255E74A0200200000002008B52A219C
:1058180000221C20FFF74CFF0E2102221C20FFF75C
:1058280047FF0F2103221C20FFF742FF2B211222E2
:105838001C20FFF73DFF2C2102221C20FFF738FF18
:105848002D2101221C20FFF733FF2E2100221C20CE
:10585800FFF72EFF05221C202A21FFF729FF024B04
:105868004FF480721A8008BD0E00002008B564202D
:1058780004F071FE68202321F022FFF719FF10B908
:10588800032004F072FE052004F065FE044B682036
:105898001A78202142F00F02BDE8084008E700BF4F
:1058A8004802002008B50F2108221820FFF700FF42
:1058B8000E2218201021FFF7FBFE024B4FF48052F6
:1058C8001A8008BD0E00002008B5134B53201B7822
:1058D8002D2108227BB1FFF7EBFE31210A2253204C
:1058E800FFF7E6FE2C210C225320FFF7E1FE5320A0
:1058F8003821902209E0FFF7DBFE31210A225320EC
:10590800FFF7D6FE53202C210A22FFF7D1FE40F2E2
:105918000912024B1A8008BD4B0200200E0000201D
:1059280007F024BA07F048BB07F020BA07F044BBD9
:1059380073B51D4CA37E53BB1C4A1D4D93694FF490
:10594800805643F00803936110238DF806302846EB
:10595800032301A98DF80730ADF8046009F0F2F8C7
:10596800144A2E61138823F040031B041B0C138078
:10597800138823F038031B041B0C43F0080313801F
:1059880013889BB243F0400313800123A37675204C
:1059980001A90122FFF7FAFB9DF80400A0F17003AA
:1059A8005842584102B070BDE80F00200010024074
:1059B800000C014000380040F8B50F461646074C69
:1059C8004FF48055656140F080000CF049FA384684
:1059D80031460CF06BFA2561F8BD00BF000C0140A0
:1059E80013B501220DF1070104463A20FFF7E4FF41
:1059F800052004F0A5FD9DF8073003B101232370AD
:105A080002B010BD174A13B51388044623F04003AB
:105A18001B041B0C13801388432023F038031B043A
:105A28001B0C1380138869469BB243F04003138014
:105A38000622FFF7C1FF9DF800209DF8013043EAD8
:105A4800022323809DF802209DF8033043EA0223B5
:105A580063809DF804209DF8053043EA0223A38063
:105A680002B010BD0038004070B50E46054C4FF42A
:105A7800805565610CF0F4F930460CF0F1F92561B8
:105A880070BD00BF000C014007B5232004F063FD82
:105A98006820752101220DF10703FFF711FC28B1D9
:105AA8009DF80700A0F168035842584103B05DF81B
:105AB80004FB00BF4D282DE9F047044600F04E8650
:105AC80000F2B980302800F0AE8651D8222800F0C4
:105AD8008A8423D8032800F0FD8114D8012800F017
:105AE800D581022840F0EE8604200BF0B1FB43205C
:105AF8000BF07FFB4C200BF07CFB46200BF079FB76
:105B08004C2000F050BE042800F0ED81052840F03C
:105B1800D9861A200BF09CFB0024F4E1282800F019
:105B2800DC8515D8242800F0C385262840F0CA86CD
:105B3800DC4C06200BF08CFBB4F85C010BF08BFB03
:105B4800B4F85E010BF087FBB4F8600100F0ADBD5E
:105B58002C2800F0D5852E2800F04F862A2840F002
:105B6800B18601200BF074FBCE4B587900F01BBEB8
:105B78003D2800F0F1821ED8362800F025860BD883
:105B8800322800F00A86342840F09C8648200BF022
:105B98005FFB002500F049BC3A2800F0B2823B28A0
:105BA80000F01A84382840F08D8604200BF050FB52
:105BB800BC4C00F083BD452800F0708627D84028EB
:105BC80000F0F485422840F07D86B64C10200BF09A
:105BD8003FFB60790BF00DFBA0680BF045FB94F8D8
:105BE80092010BF006FBB4F85C010BF034FBB4F83F
:105BF8005E010BF030FBB4F860010BF02CFBB4F83D
:105C080082010BF028FBB4F8840100F04EBD49284E
:105C180000F0AD824B2800F09285462840F052866D
:105C28000D200BF015FB00200BF0E3FA00200BF021
:105C38001BFB00F03EBE702800F0EA8200F2D9801B
:105C4800692800F03E8200F2AA80662800F0998157
:105C580000F29A80642800F06F81652840F032864F
:105C6800914C0B200BF0F4FA20880BF0F4FA6088C2
:105C780080B20BF0F0FA8D4B1B68C3F3C000C3F37E
:105C88008002800040EA4200C3F340021043C3F39D
:105C9800401240EAC20003F0100318430BF0DBFA8D
:105CA800834B1A88636812F0010F14BF4FF0020C7F
:105CB8004FF0000C12F0020F02F0080814BF4FF06A
:105CC800040E4FF0000E03F4475912F0040F14BFEE
:105CD8001027002749EA080912F0400F03F480480A
:105CE80014BF2026002649EA080912F0100F03F411
:105CF800004814BF4FF40075002549EA080912F05E
:105D0800200F03F4803814BF4FF48060002049EA64
:105D1800080912F4807F03F4003814BF4FF40061BF
:105D2800002149EA080912F4007F03F48028614A37
:105D380049EA080903F4002849EA0809127803F433
:105D4800801849EA080903F0007349EA0303C2F31B
:105D5800800243EA020343EA0C0343EA0E0E4EEACA
:105D6800070746EA070645EA060540EA050041EA4C
:105D7800000114BF4FF400184FF00008002041EA5A
:105D880008080346217AE7E0672800F0228168289E
:105D980040F0988510200BF05BFA002489E16C280C
:105DA80000F0A28117D86A2800F005846B2840F01B
:105DB800898505200BF04CFA3F4B18880BF04BFAFD
:105DC8003E4B18880BF047FA374B93F86E0000F0FB
:105DD800010000F0E8BC6E28334D00F0988100F215
:105DE800CC8106200BF034FAE86D0BF03DFA344B09
:105DF80085E1782800F0FA8018D8742800F03683F6
:105E08000AD8722800F09783732840F05B85082031
:105E18000BF01EFA0124C7E3762800F0EC8300F2A9
:105E28005E832F200BF014FA264CCDE2A42800F054
:105E3800088414D87B2800F06D82A02840F04285A1
:105E48000C200BF005FA204B18680BF00DFA1F4BCD
:105E580018680BF009FA1E4B186800F02EBDF128DF
:105E680000F00081FE2800F01384F02840F02A8515
:105E78000D4C04200BF0ECF9236CB3F85A000BF02E
:105E8800EAF9236CB3F8580000F00FBC03200BF0BC
:105E9800DFF900200BF0ADF920460BF0AAF90C2031
:105EA80000F081BC602500200410002008110020AB
:105EB800D0110020BA30002086110020881100205F
:105EC800DC100020C7920108E8F7FF1FECF7FF1F5E
:105ED800F0F7FF1F0BF0BCF901200BF08AF90A203C
:105EE8000BF087F9ABE306200BF0B2F945200BF075
:105EF80080F955200BF07DF946200BF07AF9312016
:105F08000BF077F9D0E3B14B185D01340BF071F960
:105F18000B2CF8D10024AE4B185D01340BF069F955
:105F2800082CF8D10024AB4B185D01340BF061F953
:105F3800072CF8D100F0C3BC07200BF089F9E72043
:105F48000BF057F9A44B58790BF053F900200BF0DC
:105F580050F9042000F0B1BC8B420BD29F4A9C5CE4
:105F6800012202FA04F414EA080F1CBF9A401043F5
:105F78000133F1E70BF078F9974B93F8AC0700F091
:105F880012BC12200BF064F9954B00241B88B3F562
:105F9800806F8CBF08250125924B33F9140001341A
:105FA80090FBF5F080B20BF056F9032CF4D18E4C2F
:105FB800A08C0BF050F9E08C0BF04DF9208D0BF014
:105FC8004AF9608D0BF047F9A08D0BF044F9E08D8C
:105FD8006BE310200BF03CF90024844B185D01346E
:105FE8000BF007F9102CF8D100F069BC70200BF009
:105FF8002FF900260E2474437B4D01362B6C234465
:10600800B3F819010BF027F92B6C2344B3F81B01E3
:106018000BF021F92B6C2344B3F81D010BF01BF98D
:106028002B6C234493F81F010BF0E3F82B6C2344EB
:1060380093F820010BF0DDF82B6C234493F8210131
:106048000BF0D7F82B6C234493F822010BF0D1F80E
:106058002B6C1C44D4F823010BF006F9082EC9D187
:1060680000F02DBC70200BF0F3F85B4C04F17005C8
:1060780094F8D4000BF0BDF894F8D5000BF0B9F8FB
:1060880094F8D6000BF0B5F894F8D7000BF0B1F8F7
:1060980094F8D8000BF0ADF894F8D9000BF0A9F8F3
:1060A800073494F8D3000BF0A4F8AC42E0D100F028
:1060B80006BC4F4B185D01340BF09BF8102CF8D13F
:1060C800FDE34C4D00242878400000F0FE000BF062
:1060D800BFF82B789C4280F0F283474B33F81400CA
:1060E8000BF0B9F80134F4E7444C06200BF0B0F893
:1060F80020880BF0B0F860880BF0ADF8404B18889A
:10610800D3E204200BF0A4F8374B186ED5E3072030
:106118000BF09EF83B4B1888FF28A8BFFF20C0B2A1
:106128000BF067F8384B186880F3100080B20BF05A
:1061380092F8B5F864000BF08EF8274B93F8872196
:10614800324B186822B10A23584380F3100001E04B
:1061580000F30F0080B2A8E21F4C02200BF078F881
:1061680094F8DE010BF045F894F8DD011BE30220FA
:106178000BF06EF8184B988997E20B200BF068F833
:10618800AB6E002618780BF034F8AB6E58780BF02D
:1061980030F8AB6E144C3344187901360BF029F8FB
:1061A800032EF6D1A36ED8790BF023F8A36E987856
:1061B8000BF01FF8A36ED8780BF01BF8A36E588964
:1061C8000BF049F8A36E187AEDE200BF78B1010828
:1061D80084B1010859B10108602500200D10002084
:1061E8000E000020D61000200410002034100020DB
:1061F80048100020D42200203C250020F82400204C
:10620800E4100020F81000200411002000110020E4
:10621800C04C1E200BF01CF8236C00251B78022BA9
:1062280065D1236C05F1080253F82200BA490CF035
:10623800A3FF10F0F1FC80F30800C0B20AF0D9FF08
:10624800236CB64903EB8503D86A0CF095FF10F070
:10625800E3FC80F30800C0B20AF0CBFF236C05F121
:106268000E0253F82200AE490CF086FF10F0D4FC61
:1062780080F30800C0B201350AF0BBFF032DD0D16E
:10628800072D236C21D1586CA3490CF075FF10F031
:10629800C3FC80F30800C0B20AF0ABFF236C9E4930
:1062A800986C0CF069FF10F0B7FC80F30800C0B2DE
:1062B8000AF09FFF236C93F84C000CF005FF10F0D8
:1062C800ABFC80F30800C0B20BE02B4458780AF00E
:1062D80090FF236C2B44D87A0AF08BFF236C2B4455
:1062E800587D01350AF085FF0A2DC9D1E7E2236CF4
:1062F8002B4458780AF07DFF236C2B44D87A0AF097
:1063080078FF236C2B44587D01350AF072FF0A2D63
:10631800EDD1D4E23C200AF09BFF00247D4D04F12E
:1063280008022B6C7E4953F822000CF025FF10F070
:1063380073FC80B20AF08FFF2B6C794903EB84035E
:10634800D86A0CF019FF10F067FC80B20AF083FFDE
:106358002B6C04F10E0253F8220071490CF00CFF6B
:1063680010F05AFC013480B20AF075FF032CD5D125
:10637800072C2B6C16D1586C69490CF0FDFE10F0F7
:106388004BFC80B20AF067FF2B6C6549986C0CF0E7
:10639800F3FE10F041FC80B20AF05DFF2B6C93F81D
:1063A8004C000BE0234458780AF055FF2B6C23442B
:1063B800D87A0AF050FF2B6C2344587D01340AF038
:1063C8004AFF0A2CD4D17AE214F8010F002800F011
:1063D80076820AF00EFFF7E701200AF039FF4D4BED
:1063E8001B6C1878DFE150200AF032FF0025494B7A
:1063F8000C211C6C4B4B04EB850494F87920013577
:1064080001FB023393F838000AF0F3FE94F87A009F
:106418000AF0EFFE94F87B000AF0EBFE94F87C009B
:106428000AF0E7FE142DE2D149E23A4B1C6C062330
:1064380003FB054494F8CE000AF0DBFE94F8C9008B
:106448000AF0D7FE94F8CA000AF0D3FE94F8CB00FD
:106458000AF0CFFE94F8CC000AF0CBFE013594F890
:10646800CD000AF0C6FE0C2DDFD128E24FF000085F
:1064780001260027274B1A7A974227DA0933FA5C54
:1064880000240C236343274D05F13001595C9142E8
:1064980007D12B44586B10F0F6F982462EB9B14655
:1064A80005E001341B2CECD10EE080440CE0D14512
:1064B8000ADA0C2303FB04535B6B13F809000AF098
:1064C80098FE09F10109F2E70137D3E7002E00F041
:1064D800F6815FFA88F00AF0BBFE0026C9E70D4D89
:1064E8000024287A0AF0B4FE2B7A9C4280F0E781D7
:1064F8000D4B0021E65C0C2202FB01F3094800F178
:106508003007DA5DB24211D1034493F838000AF03B
:1065180070FE0EE004100020000020410000C84278
:1065280000007A44C89201080D10002001311B298F
:10653800E1D10134D8E7CE4C16200AF089FEB4F830
:1065480098010AF088FEB4F844010AF084FEB4F811
:1065580046010AF080FEB4F848010AF07CFEB4F85F
:10656800DA010AF078FE94F8EB010AF042FE002006
:106578000AF03FFE94F8EC010AF03BFE94F887011C
:106588000AF037FE94F894010AF033FE00200AF06E
:1065980030FEB84B0A201B6CB3F9563093FBF0F071
:1065A80080B20AF058FE89E0E0B201340AF021FE18
:1065B800092CF9D183E110200AF04AFEAE4BAF4C0A
:1065C800187800F002000AF014FEAD4B18780AF0B3
:1065D80010FE20680AF048FE60680AF045FEA94BE4
:1065E80018880AF038FEA84B18880AF034FEA14B28
:1065F800B3F86C0059E00AF0DFFD074612200AF0F4
:1066080027FE9C4C17B9266F656F05E0102F19BF40
:1066180000252E46A66FE56F38460AF0EAFD30469B
:106628000AF022FE28460AF01FFED4F880000AF07D
:106638001BFE00200AF00FFE00200AF00CFE0020CE
:10664800B1E08C4D002495F884002E46800001307E
:10665800C0B20AF0FDFD95F884000AF0CAFD96F86C
:1066680084309C4280F02B81884D285D0AF0C1FD62
:1066780005F11003185D0AF0BCFD05F12003185D53
:1066880030350AF0B6FD285D0AF0B3FD0134E6E7BF
:1066980008200AF0DDFD00200AF0DDFD00200AF0E8
:1066A800DAFD00200AF0D7FD00200AF0D4FD06E14B
:1066B80004200AF0CDFD6E4B9868FEE094F87C014A
:1066C8000AF097FD94F880010AF093FD94F87F0191
:1066D8000AF08FFD94F8810165E0654C07200AF007
:1066E800B7FDB4F882010AF0B6FDB4F884010AF0E7
:1066F800B2FD94F886010AF07CFDB4F88801D4E76D
:106708005B4C0C200AF0A4FD94F892010AF071FD8C
:10671800B4F89C010AF09FFDB4F898010AF09BFDBB
:10672800B4F89A010AF097FD94F893010AF061FD14
:10673800B4F89E010AF08FFDB4F8A001B5E74C4CFF
:1067480004200AF085FD94F8D8010AF052FD94F867
:10675800D9010AF04EFDB4F8DA01A6E74C4C4D4DCC
:106768002078002600EB4000C0B20AF071FD2378C3
:1067780002359E4280F0A38015F8020C0AF039FD1C
:1067880015F8010C013600EB800000EB800000F2E8
:10679800EE2080B20AF05FFDE9E701200AF058FD1B
:1067A800334B93F894010AF024FD88E008200AF09E
:1067B8004FFD00242E4B234493F88A0101340AF03C
:1067C80018FD082CF6D17AE02A4B294C93F8C5001D
:1067D80004F12005C0EBC000C0B20AF039FD94F8FE
:1067E800F20100232C4AD25C90426ED00C33302B3D
:1067F800F8D10834AC42F2D161E040200AF028FD1B
:106808001B4C04F14005B4F8A4020AF024FD94F8E6
:10681800A6020AF0EEFC043494F8A3020AF0E9FC9C
:10682800AC42F0D14BE0E0200AF012FD104C04F12C
:106838008005B4F82602043400F03F000AF00BFD8E
:10684800B4F82202C0F386100AF005FD94F820027D
:1068580000090AF0CEFC94F8200200F00F000AF0BC
:10686800C8FC94F821020AF0C4FCAC42E1D126E04D
:1068780060250020041000200C11002014110020B5
:1068880012110020101100200E1100208910002084
:10689800D422002002270020E022002013200AF042
:1068A800D7FC0024144B185D01340AF0A2FC0B2C11
:1068B800F8D100200AF0D8FC00200AF0D5FC01200D
:1068C800BDE8F0870020BDE8F0870AF092FCB4F834
:1068D800F4010AF0C0FC94F8F6010AF08AFC94F876
:1068E800F7010AF086FC94F8F9010AF082FC94F8A2
:1068F800F8010AF07EFC7CE778B101082DE9FF4732
:10690800C54C07462378C54E002B00F0DA81326863
:106918006368D31A7C2B40F2D481237A62600133F6
:1069280023724FF0000808F12400BB4DC0B208F0F4
:106938007BFC05F10A0333F918000CF0C9FBB84BCE
:10694800814618880CF0C4FB014648460CF0C8FC88
:10695800B4490CF011FC0CF0D5FD08F1010800B2A7
:1069680008F050FCB8F1030FDDD1302008F05CFCD2
:10697800B5F9100008F046FC08F04EFC2B7A9A078F
:106988002CD141F288336A689A4218D9102008F04D
:106998004BFC68694FF0640890FBF8F000B208F00F
:1069A80031FC212008F040FC686990FBF8F308FBF3
:1069B80013000028B8BF404200B208F023FC14209E
:1069C80008F032FCB4F9180008F01CFC1C2008F090
:1069D8002BFC002008F016FC08F01EFC237ADFF8D8
:1069E80038825B0740F04A81022008F01DFCD8F885
:1069F8001C006423323090FBF3F000B208F002FC74
:106A0800B8F926504FF0050A95FBFAF5032008F06F
:106A18000BFC854BADB21B78DFF8209213F0040F06
:106A28000BD038460BF0A1FC28B9D9F8003013F088
:106A3800100F18BF002528B205E0D8F8283098892B
:106A4800B0FBFAF000B208F0DDFBD9F800309F0780
:106A580065D5DFF8EC91A28D99F800304FF0640805
:106A680008FB02325B00B2FBF3F3E78D06203F011F
:106A7800BFB247EA0327BFB2C3F303231F4308F09B
:106A8800D3FB38B208F0BEFBE38D99F80010013350
:106A98009BB293FBF1F201FB1233E385236B5E4D4E
:106AA8009B7B012B05D1392008F0BEFBB5F92C00E2
:106AB80019E0AD8D6E235D43152795FBF7F53A2058
:106AC800AFB208F0B1FBB7FBF8F528B208FB1575B3
:106AD80008F098FB3B2008F0A7FBA8B2451D0A2048
:106AE80095FBF0F000B208F08DFB282008F09CFB25
:106AF800636B0A2093FBF0F000B208F083FB0420DC
:106B080008F092FBA36A9B8913B109F09BFD03E08F
:106B1800414B986B80F3100000B208F073FBE36BF5
:106B28003D4F9D0640F19F8097F8403098071DD54E
:106B3800112008F079FBB7F842004FF4F365684379
:106B48003A4B90FBF3F000B208F05CFB192008F018
:106B58006BFBB7F842004543642095FBF0F595FBC5
:106B6800F0F300FB135000B208F04CFB94F84030EF
:106B7800B4F8445013F0020F08BF0025012008F0B4
:106B880053FB28B208F03EFB092008F04DFB00201B
:106B980008F038FB264B94F846501A88B2F5967FD1
:106BA8000AD91D4B1B7A03F00F03072B04D842F2B6
:106BB8000F75954228BF1546052008F035FB236B55
:106BC8005B7B0BB928B216E0A5F120000CF080FA27
:106BD80018490CF085FB002105460CF06BFC10B938
:106BE8004FF07C5101E04FF03F4128460CF0BCF9D2
:106BF8000CF088FC00B208F005FB94F84020064B26
:106C0800910703D493F84720012A1BD1012384F864
:106C1800473009482EE000BFCC1000202425002072
:106C28000E00002000007A44BA300020A08601003F
:106C3800460000206666E63F14110020002500206B
:106C4800440000201D6BBD4968680CF095FA0CF0F3
:106C580059FCBA490290A8680CF08EFA0CF052FC64
:106C6800039002A806E0B64A02AB92E8030083E864
:106C78000300184608F0E8FA08F0CEFA237A282B21
:106C88001FD1B04B00221A7233684FF47A70B3FBED
:106C9800F0F83C27172008F0C7FAB8FBF7F5B5FB62
:106CA800F7F007FB1050000200B208F0ABFA18200A
:106CB80008F0BAFA07FB158000B208F0A3FA08F04A
:106CC800ABFA94F850309F4D002B00F05A8103F036
:106CD8001BFC6B6D9C4AC31A9342074640F2C28064
:106CE800002385F85A3085F85C30AB8DDAB21B0A80
:106CF80085F8762085F8773085F86C2085F86D3032
:106D0800D5F8842033689A1AD5F88830D97B4FF49F
:106D18007A734B439A420ED38C4B1B68C5F8843068
:106D280095F88C30013B012B9FBF102385F85A3012
:106D3800022385F85C30626B0A20A36B92FBF0F2A9
:106D480093FBF0F384F87420121284F8752084F809
:106D5800783094F840201B1284F8793094F8463043
:106D68009207784984F8A73003D42D2381F8A830F6
:106D780077E0D4F848907648DFF8E0C199FBF0FA5C
:106D88000CFB0A924FF0060E042B0EFB02F28CBF8E
:106D98003323322381F8A8306E4BE66C92FBF3F173
:106DA80096FBF0F003FB1122642592FBF5F20CFB35
:106DB800006C0EFB0CFE84F89920121284F89A20BD
:106DC8009EFBF3F203FB12E393FBF5F30AEB8A0A4B
:106DD8004FFA81F80AEB8A0A08EB8A0189B284F82B
:106DE800971000EB8000090A84F8981000EB8000E7
:106DF80051B201EB800292B284F89C20120A84F806
:106E08009D2084F89E30B4F842201B1284F89F30ED
:106E18002423534393FBF5F5B4F8BA300A2284F8D7
:106E2800A0301B0A84F8A130B4F844304FEAD9796D
:106E3800B3FBF2F303F5FA739BB284F8A2301B0A92
:106E480084F8A330B4F8BC30F60F84F89450C5F336
:106E5800072584F8969084F89B6084F8955084F808
:106E6800A930676594F8BE80364DB8F1000F0DD192
:106E7800D5F8C40003F01AFC012807D90228364EB9
:106E880000F0518202F0E0FD0123B370D4F8C8206D
:106E98002C4D002A75D095F8BE603EB140F6B7314A
:106EA800D5F8D030FB1A8B4219D86AE00123D5F8FF
:106EB800C40085F8BE3003F027F9D5F8D43008218E
:106EC80093F9000002238DE8480032464FF49643B8
:106ED80003F08FFB85F8D860C5F8C4004FE095F83B
:106EE800CC60CEB9D5F8C400C5F8C86085F8BE60D6
:106EF80003F00AF9D5F8D430082193F900000123EA
:106F08008DE8480032464FF4964303F072FBC5F80B
:106F1800C40002F099FD32E0013EF6B285F8CC607B
:106F280095F8D81095F8D930D6B94A1C013385F8A8
:106F3800D82085F8D930D5F8C4001EE08096184BC3
:106F480048940108CC1000203F0D030024250020A0
:106F58008096980040420F000E000020806967FF6D
:106F680012F8016B01337018314685F8D800D5F84E
:106F7800C400C5F8C82085F8D93003F09AFBC4F8D6
:106F8800D07094F8DA309C4DF3B1D5F8DC30DBB131
:106F9800D5F8E030C3B1C5F8E4301B68974AC5F8A6
:106FA800E830D5F8EC301344187AFEF783FDD5F8AD
:106FB800E43098790AF01DF9D5F8EC300133092B43
:106FC80088BF0023C5F8EC308D4D94F8F0202E686A
:106FD800894B002A00F0E181D3F8F420002A00F060
:106FE800DC8193F8F830013B012B00F2D681D4F80C
:106FF800F400814F03F05AFBE0B1D7F8F40003F036
:1070080052FB97F8F93080467E2BD5F800900ED1C8
:1070180002231B2887F8F83009D1D7F8F40003F0C9
:1070280045FB20B90123C7F8FC9087F8003184F8A4
:10703800F980DCE7D7F8FC202B689B1A41F6583218
:1070480093421DD9032387F8F830A6E16D4A32F838
:10705800130010B903464FF403600133B0F5C06F55
:10706800DBB275D01DD9B0F5006F7AD031D9B0F543
:10707800036F3ED184F80131E36B5F4F99063FD42B
:1070880094F8001194F80131002900F049812A6828
:10709800921B012ADAD984F80131002384F80031DF
:1070A8007BE1B0F5007F42D007D8B0F5807F47D0AC
:1070B800B0F5887F00F08380E6E7B0F5806F00F0D8
:1070C800A580B0F5826F00F0EA80B0F5047FDBD1CF
:1070D80023E0B0F5E26F00F08280B0F5E46F00F0D5
:1070E8008380B0F5E06FCFD184F80131B4F90A108C
:1070F8007EE0B0F5046F6BD0B0F5026FC4D1F9E053
:1071080097F840309A07BBD5B7F8421024234B4371
:107118006421123393FBF1F1FCE084F801313A4B1E
:10712800354F1B689B07ABD5BB8D0A21F1E084F86E
:107138000131354B304F1B681905A1D5796BE9E052
:1071480084F80131E36B2C4F5A0799D57969E1E04E
:1071580084F801312C4B284F1B681B0590D5B96B5F
:10716800D8E0E16B244A8F0684F8013188D592F87B
:107178004010880784D5D90710D5D36C192283EA23
:10718800E371A1EBE37101EB5101B1FBF2F1002BCB
:10719800ACBF41F0004141F040410DE0936C192231
:1071A80083EAE371A1EBE37101EB5101B1FBF2F169
:1071B800002BB8BF41F080414FF4006089E084F8AB
:1071C8000131E36B0C4F5B077FF55AAF3969A1E0DA
:1071D80084F80131B4F918306421594379E084F80E
:1071E8000131B4F90C1003E0B4F90E1084F8013140
:1071F8002C2391FBF3F16CE0CC100020489401089B
:107208002425002090B501080025002084F80131CC
:1072180094F80231624A0133DBB2032B88BF0123A1
:1072280082F8023142F2107394F8021159435D4B0F
:107238001B78D80748BF01319A0748BF02315F075A
:10724800B4F8043148BF0431D80748BF0A319A0757
:1072580048BF14311F0648BF2831D80548BF283118
:107268005A0748BF64311F0748BFC831980548BF4F
:1072780001F5C8719A0648BF01F57A71DF0648BF63
:1072880001F5FA61580648BF01F57A614FF480604C
:1072980002F0A6FB424B002283F80021F0E6E16BE6
:1072A800DFF8FC8011F0200784F8013117D098F836
:1072B800402012F0020F14BF4FF47A71002112F02F
:1072C800010F14BF4FF4FA6300230B4494F84610DF
:1072D800194402F085FB002384F80031D0E6324BD4
:1072E8001B6819067FF5CCAE394602F079FB88F8A1
:1072F8000071C5E684F80131E36B294F9A067FF5E2
:10730800BFAE97F840309B077FF5BAAEB7F8443068
:107318006421594302F064FB002387F80031AFE68B
:1073280084F8013139E0B37823B1C5F8C07086F824
:107338000280ABE5D5F8C030FB1AB3F57A6FFFF4DD
:10734800A5AD0123D5F8C400B37003F0ACF9064627
:10735800D5F8C40003F0A7F976067FF497AD8A281C
:1073680002D08E280CD091E5EB6B98067FF58EAD98
:1073780095F8BE30002B7FF489AD05F18D0306E04A
:1073880095F8BE30002B7FF481AD05F15803C5F8A0
:10739800C8302D2385F8CC3078E504B0BDE8F087F7
:1073A800CC100020BA3000200025002038B5002479
:1073B8000B4D6059254409F0CFFF696811B10948A0
:1073C80001F098F9A96811B1074801F093F9074845
:1073D800103409F0C1FFB4F5D87FE9D138BD00BF3A
:1073E8005C940108B0B50108B6B5010800C10108F0
:1073F800F0B585B004460FF046FA082826D1621E7B
:10740800E01D1F4912F8013F09681944497801F045
:107418000301022908BF203B82421370F1D125469F
:1074280004F1080715F8016B164831460FF01DFAEC
:1074380020B1284631460FF018FA10B102F0C0FB0F
:107448001CE0BD42EED1204608F028FD0E4809F0A8
:1074580083FF00230D4A04A91A4492F88A210A449A
:107468000849595C0133082B02F80C1CF2D100239F
:10747800074801A98DF80C3001F03CF905B0F0BDC2
:107488005800002023CC0108BCB501086025002065
:1074980042C001082A4B2B4C1E6880B5206803F0B7
:1074A800F4F8304603F0F1F8206841798D0703D4E9
:1074B80041F0020103F09AF8234B08221A61234D88
:1074C80010221A612B689A0341BF06236371E3797E
:1074D80023F0010344BF43F00203E371206803F083
:1074E800E5F890B1184F08237B61164B186803F034
:1074F800DAF8804603F068F908B109F0C3F93046B4
:10750800414603F0D6F808233B61304603F0CEF835
:1075180078B10D4F4FF01008C7F814803046D4F8F2
:10752800009003F0C0F80146484603F0C2F8C7F8D7
:1075380010802B689B03D1D507F0EBFFCEE700BF87
:10754800C8240020D4110020000C01400025002090
:107558002DE9F04705460FF096F92F4E0446D6F868
:10756800088090B92D4809F0F7FE2D4B53F82410E8
:1075780049B10123A34013EA080F02D0294801F0BA
:10758800B9F80134F1E7284822E02846274922467D
:107598000FF082F958B9264809F0DEFE254C54F858
:1075A800041F0029EFD01F4801F0A4F8F7E72B7853
:1075B8004FF000092D2B03BF013504F1FF344FF0C4
:1075C800010A4FF0000A164B53F8297027B91A48D8
:1075D800BDE8F04709F0C0BE2846394622460FF0FC
:1075E8005BF9A8B9012000FA09F0BAF1000F03D03D
:1075F80001F014FA114803E040EA0800B0601048AE
:1076080009F0AAFE3946BDE8F0470E4801F072B805
:1076180009F10109D7E700BF60250020C2B50108BC
:107628000C960108CCB5010800C10108D0B50108C5
:10763800D5B5010808960108E1B50108F0B50108BB
:10764800F9B5010841C0010810B5084809F084FEE1
:10765800074B00241C741C64064B1C7004F0B4F91E
:107668000AF052F8044B1C6010BD00BF01B60108B7
:10767800D4110020BB300020C824002070B5064675
:1076880000240B4BE518AA8816420AD0E15809488D
:1076980001F030F82846002109F0EFFD064809F00E
:1076A8005BFE40F6944314349C42EAD170BD00BF9F
:1076B8000CA201082DB6010800C10108F0B5047834
:1076C8008BB005460CB1002436E04A4B19680E23EE
:1076D80003FB0411B1F91D51B1F91921B1F91B319D
:1076E800009591F8205101F58C70019591F8215180
:1076F80001F59071029590F90700039091F9021035
:107708003D4804912146013400F0F4FF082CDCD1F7
:107718006DE02D2B14D1072C1BDC28460FF008F93F
:107728000AAB661C03EB440424F8100C15F8013F5F
:10773800303B092BFAD934462B78002BE9D104E0E9
:10774800A3F13002092A09D8E5E7082CBDF818206A
:1077580009D00BB0BDE8F04002F032BA202BF8D1C6
:1077680001352646E7E7072AF3D840F2DC55BDF88D
:107778001A00204BA0F2EE2189B2A9421B68E8D872
:10778800BDF81C10A1F2EE24A4B2AC42E1D8BDF8B9
:107798001E7004B23EB2A642DBDB0DB2AE42D8DCAC
:1077A800A542D6DBBDF92440642CD2D1BDF82660B1
:1077B80034B2112CCDDCBDF82050B42DC9D8BDF899
:1077C8002240B42CC5D812B24FF00E0E0EFB023375
:1077D800A3F81B116421A3F81901A3F81D7183F8FC
:1077E800205183F8214183F81F1183F822610BB0DF
:1077F800F0BD00BF4410002037B60108F0B50446BC
:107808008FB020460FF03FF8C5B21DBBAB4809F05A
:10781800A3FDAB4C94F8D61009B9AA4853E049B275
:1078280094F8D42094F8D530009194F8D710A6484D
:10783800019194F9D8100734029194F9D210039168
:1078480094F8D31004912946013500F053FF102D08
:10785800E0D1E2E720469D4905220FF01DF80546D4
:10786800B8B929469A4870220EF0C9FF2846994BA4
:1078780019680E2303FB001301300022082883F83F
:10788800232183F8242183F8252183F82621F0D1A8
:1078980012E12046904904220EF0FEFF05462046DC
:1078A800002D4AD120210EF0E0FF002800F00481CD
:1078B800461C30460EF0E7FF2C460746874B53F828
:1078C80024502DB986480FB0BDE8F04000F012BF33
:1078D80030462946FAB20EF0DFFF01340028EDD118
:1078E800774A164602F17001002382F8DA3082F8EE
:1078F800D63082F8D53082F8D43007328A42F3D1B4
:10790800784901EBC40191F80822934210DAD1F8C2
:107918000C72C3EBC302B0183A44176800F1D401E3
:10792800C0F8D47090880133888092798A71E7E72B
:1079380029466D4800F0DEFE8FE06C4907220EF004
:10794800ABFF05462046002D49D120210EF08DFFC2
:1079580006460EF098FFC4B26CBB654800F0CAFE3C
:1079680021466448013400F0C5FE0E2CF8D1554874
:1079780000F0C0FE00246048214600F0BBFE002550
:10798800544A012311680E2202FB0412D2F8232163
:10799800AB401342594B5A495A4808BF194601355A
:1079A80000F0A8FE0E2DEBD14648013400F0A2FEEF
:1079B800082CE0D180E0304653490EF0BDFF2C463C
:1079C80000284CD0022C4FD00EF0B2FF06AB43F883
:1079D80024004D4900200EF0AFFF0134F0E74A497A
:1079E8000EF0AAFF002460B1082C38D00EF0A0FFDA
:1079F80006AB43F82400444900200EF09DFF0134F3
:107A0800F1E7082C2BD1069B0F2B28D8DDF81CE0BA
:107A1800BEF1070F23D8089F0D2F20D8099E06F125
:107A28006402C82A1BD80A9DFF2D18D80B98642811
:107A380015D80C99642912D8884210DA0D9C032CA9
:107A48000DD8324AC3EBC303134483F804E05F71D3
:107A58009E71DD71187259729C722D4CD1E60FB06F
:107A6800BDE8F04002F0ACB8069B072B20D8079978
:107A78000D291DD80278722A0DD06E2A18D1154A00
:107A88000E20126800FB032301228A40D3F8231139
:107A980021EA020209E00F4A0E20126800FB0323C4
:107AA80001228A40D3F823110A43C3F8232101E0B5
:107AB80002F086F80D4CA4E60FB0F0BD5FB60108E1
:107AC8006025002000C101088AB60108A6B6010891
:107AD8003426002044100020ACB60108A0AE0108EE
:107AE800E1B501085C940108B1B6010857B6010870
:107AF800BAB50108BDB601087EBF010815C5010861
:107B08005BC40108C2B60108C6B6010830260020C9
:107B18007BB401082DE9F743047805468CB9324D4A
:107B280095F8A712B5F8A42295F8A6322F48009127
:107B38002146013400F0DEFD102C05F10405EFD1DB
:107B48004EE00EF0F5FE0F28044636DC28462021CC
:107B58000EF08BFE264EE4B2D6F84480451CA400F5
:107B6800002728460EF0E4FE5FFA87F9B9F1010F05
:107B780083B208D0B9F1020F0BD0B3F5B47F24D289
:107B8800726C13530AE0FF2B1FD8736C2344987050
:107B980004E0FF2B19D8736C2344D87028462C2195
:107BA8000EF063FE054608B1013502E0B9F1020F97
:107BB8000BD10137032FD4D112E00E4800210F2238
:107BC80003B0BDE8F04301F078BF08EB04000021E2
:107BD80004220EF014FE03B0BDE8F04301F0F0BF3C
:107BE80003B0BDE8F08300BF60250020C8B60108D7
:107BF800D4110020DCB601082DE9F04304788FB0D9
:107C08000546002C59D17C4B0021142209A807AE47
:107C1800D3F848800EF0F3FD0722304600210EF01D
:107C2800EEFD00231A46A70005A8059308EB0705F3
:107C380083807249B5F802E031F813C01CEA0E0FD0
:107C48000AD00E310DF1380C595C02F1010E624474
:107C580002F81C1C5FFA8EF20133072BE9D10021D0
:107C68000B46674AB5F802E011F802C01CEA0E0F8D
:107C78000AD006320DF1380C8A5C03F1010E634418
:107C880003F8242C5FFA8EF301310629E9D118F89C
:107C980007308DE841006A785A49029209A81A0902
:107CA80003F00F0300F011FD2146574809AA0134DB
:107CB80000F020FD202CA6D19BE00EF039FE1F28F5
:107CC800044600F3898028462021E4B20EF0CDFD59
:107CD8001F2C02D901F074FF8BE0474B451C9B6CAD
:107CE800002103EB8404204604220EF088FD0027BF
:107CF800464B09AE304600210A2217F803905FFA76
:107D080087F80EF07CFD002315F8012B32B10A2B01
:107D180004D04A4502D0F2540133F5E74A4561D10F
:107D280008F1FF33032B09D8DFE803F010050242FE
:107D38000DF1230037E00DF123011FE030460EF06E
:107D4800F7FD2378C0B243EA001006E030460EF093
:107D5800EFFD237800F00F001843207034E0013362
:107D6800062B0BD02A4800F2F3269E5D9642F6D1E8
:107D7800034493F8ED2263881343638011F8012FBD
:107D880012B30023EEE70133072B0CD0204A02F28E
:107D9800E6269E5D8E42F6D102EB4303B3F8D82265
:107DA80063881343638010F8011F69B10023EDE76E
:107DB80030460EF0BDFD0F2804DC30460EF0B8FD4D
:107DC800607001E0002363700137052F90D1012412
:107DD80008F0FEFC6CB97DE70E4800211F2201F077
:107DE8006CFE06E02046002104220EF008FD002467
:107DF800EEE70FB0BDE8F083D411002034970108F6
:107E080049970108E2B60108F1B60108559701083B
:107E18005C940108DCB601082DE9F04FAC498BB041
:107E280004460EF0F5FCAB49002820460CBF01259E
:107E380007250EF0EDFCA8490028204608BF0225BA
:107E48000EF0E6FC002808BF0425E90740F1FA8097
:107E5800A24809F081FA002009F08EF8A04CA14848
:107E680009F07AFAA04809F077FA63799F4A013B4A
:107E780052F823109E4800F03DFC9E4800F03AFC62
:107E880026460027D6F81480002140460BF008FB50
:107E980020B1994800F02EFC002669E03946974841
:107EA800D6F818B0D6F81CA0D6F8209000F022FC1E
:107EB800404600210BF0FEFA10B1202009F044FAE8
:107EC80006A9404600F09CFA01468D4800F012FCD5
:107ED800584600210BF0EEFA10B1202009F034FAD0
:107EE80006A9584600F08CFA0146854800F002FCC5
:107EF800504600210BF0DEFA10B1202009F024FAD8
:107F080006A9504600F07CFA01467D4800F0F2FBD5
:107F1800484600210BF0CEFA10B1202009F014FADF
:107F280006A9484600F06CFA01370146754800F08A
:107F3800E1FB0C2F06F11006A4D1AAE749B294F888
:107F4800D42094F8D530009194F8D7106E48019158
:107F580094F9D8100734029194F9D210039194F847
:107F6800D31004913146013600F0C4FB102E03D023
:107F780094F8D6100029E1D100260E277743002473
:107F8800624A0123D26CA3403A44D2F80A20134231
:107F980040F0948001340E2CF2D10136082EECD139
:107FA8005B4809F0D9F94E4B5A4C9F6854F8041FA6
:107FB80019B1594800F09EFBF8E70E46574B53F8A5
:107FC80026404CB10123B3403B4203D054482146DC
:107FD80000F090FB0136F1E7524809F0BDF921465F
:107FE8003F4B0AAA0B4493F88A3113444E4A8A5CE1
:107FF8000131082903F8102CF2D1002306A94B48B7
:108008008DF8203000F076FB494809F0A5F9494879
:1080180002F0A2F8484809F09FF94648FFF7ECFD3E
:10802800464809F099F94348FFF774FD444800F0C1
:1080380061FB4020FFF722FB424809F08DF93D48DB
:1080480001F0DCFFAA0726D53F4809F085F93F482B
:1080580009F082F9374808F0CFFF3D4809F07CF96C
:10806800344801F037FD3B4809F076F9314801F012
:1080780017FF394800F03EFB2E4801F0A7FD3748AE
:1080880009F06AF92B48FFF719FB2D4800F032FB7D
:108098008020FFF7F3FA6B0716D5314809F05CF931
:1080A800304809F059F9234808F080FF244800F0C7
:1080B80021FB4FF48070FFF7E1FA05E031462246D4
:1080C800294800F017FB65E70BB0BDE8F08F00BF4B
:1080D800FDB601080DBB010804B701080AB701087D
:1080E8006025002018B701082AB70108A0AE0108CA
:1080F80036B7010841B701084EB701085BB7010858
:10810800B9B5010842C0010863B70108D4110020BD
:1081180082B701080896010892B701080C96010871
:10812800A0B70108ADB7010823CC0108B9B7010809
:10813800C2B701087BB40108D1B70108DDB701084F
:1081480000C10108EBB70108F8B701080BB801082E
:1081580019B8010823B8010832B8010840B8010865
:108168004CB801085DB801086FB80108F0B50124E2
:10817800B0FBF4F58D4201D34C43F9E70026D4B1A6
:10818800B0FBF4F504FB1500B4FBF1F41EB9002DA7
:1081980001DC002CF3D1092D03F1010EEFB204DD4F
:1081A800002A14BF3725572500E030253D441D70AF
:1081B80001367346E3E71C70F0BDF0B50124B0FB4F
:1081C800F4F58D4201D34C43F9E70026D4B1B0FB56
:1081D800F4F504FB1500B4FBF1F41EB9002D01DC25
:1081E800002CF3D1092D03F1010EEFB204DD002AB2
:1081F80014BF3725572500E030253D441D70013652
:108208007346E3E71C70F0BD03685A1C02601970DE
:1082180070472DE9F843089E002B07468846144608
:10822800334614BF4FF030094FF0200913F8012BE3
:108238000AB9254603E0002CFBDD013CF6E7002DDA
:1082480004DD38464946C047013DF8E7354624EA8B
:10825800E474A01B284415F8011B11B13846C04727
:10826800F7E7BDE8F883024B186802F022BA00BFAE
:10827800D80F0020F8B507460C4648680021154677
:108288001E460BF00DF958B128460AF021FF104997
:108298000AF072FF01464FF07E500BF021F8606043
:1082A800616830460AF060FE014630460BF018F867
:1082B80025680646294638460AF054FE01463046E7
:1082C8000AF05AFF014628460AF04EFE2060F8BD23
:1082D800DB0FC9402DE9F04102780346202A00F15E
:1082E8000100F9D0092AF7D02D2A02D10346414DC1
:1082F80004E02B2A08BF03464FF07E551C46002693
:10830800234614F8012BA2F13007F9B209290DD838
:10831800394930460AF030FF064638460AF0D8FE9A
:10832800014630460AF020FE0646E9E72E2A17D114
:10833800314F234614F8010B3038C2B2092A0FD83E
:108348000AF0C6FE39460AF0CBFF014630460AF06D
:108358000BFE2949064638460AF00EFF0746E8E7AD
:108368001A7802F0DF02452A39D15A782D2A02D12B
:108378000233012704E02B2A14BF013302330027FC
:10838800013B002413F8012F303AD1B2092903D850
:108398000A2101FB0424F5E7B4F59A7F28BF4FF4BE
:1083A8009A74A0464FF07E53B8F1070F07D91846C4
:1083B80012490AF0E1FEA8F108080346F4E704F0C0
:1083C800070434B118460C490AF0D6FE013C0346AE
:1083D800F7E719462FB130460AF082FF04E04FF064
:1083E8007E5130460AF0C8FE014628460AF0C4FE0F
:1083F800BDE8F081000080BF0000204120BCBE4CD9
:1084080030B5054687B00C4603A800210C220EF0B3
:10841800F6F9284600210BF06BF820B128462849C8
:108428000AF0A2FD03E0284625490AF09BFD2549EC
:108438000AF0A2FE0BF066F8054680EAE07069468D
:10844800A0EBE57009F080FF002DACBF20232D23A1
:1084580068468DF80C300EF016FA012807D1302343
:108468008DF80D308DF80E308DF80F300CE00228A5
:1084780005D130238DF80D308DF80E3004E0032837
:1084880004BF30238DF80D30694603A80EF0DEF9DD
:1084980003A80EF0F8F90338C5B22A4603A9204606
:1084A8000EF01CFA00236355204607490EF0CEF95A
:1084B80003AB204659190EF0C9F9204607B030BD64
:1084C8006F12033A00007A447EBC010870B5064674
:1084D800B6FBF2F40846154614B12046FFF7F6FF3E
:1084E80005FB1464024B1B5D00F8013B70BD00BF27
:1084F80080BC01082DE9F04F81468A4616461C4685
:1085080089B000253178002900F0DB80252902D0C8
:108518000136484674E072784FF00008302A0CBFE4
:10852800B278B71CA2F1300312BF4FF0000BF71C52
:108538004FF0010B092B19D8A2F13003D9B2092940
:1085480005D80A2202FB083817F8012BF4E7A2F134
:108558006103052B02D8A2F1570305E0A2F14103FC
:10856800052B03D8A2F137030A2BEADD6C2A30D198
:108578003A787E1C642A00F083800BD8252A3DD0E7
:1085880003D8002A00F09D80BCE7582A0CD0632A43
:1085980019D0B7E7732A22D002D86E2A37D0B1E7AC
:1085A800752A5CD0782AADD1271D2068A2F158041D
:1085B80062424FF01001624155E02CD9582A32D05E
:1085C800632A2AD13E4648462178271DD0470135DF
:1085D8000FE0642A63D00ED9732A14D13E4623686B
:1085E80048460093514642460023FFF712FE271DD6
:1085F80005443C4686E7252ADFD13E4648462521E4
:10860800D04701357EE70AD86E2A06D13E46236850
:1086180004341D6076E7002A53D03E4672E7752A77
:1086280026D0782AF9D1A2F1580304F1040C5A4251
:108638002068CDF80CC04FF010015A4105ABFFF788
:1086480095FDDDF80CC03E46644605AB00934846F0
:10865800514642465B46FFF7DCFD054452E7206879
:10866800271D0A21002205ABFFF7A7FD3C46ECE7D2
:1086780004F1040CCDF80CC020680A210022DDE7C3
:108688002068271D002808DA2D238DF81430404271
:108698000DF115030A210022E6E705ABFAE7206889
:1086A80004F1040C00280ADA2D238DF81430404216
:1086B8000DF11503CDF80CC00A210022BFE705AB68
:1086C800F8E7284609B0BDE8F08F0EB40FB505AB42
:1086D80053F8042B0190064901A80393FFF70AFFFA
:1086E800019B00221A7004B05DF804EB03B07047D8
:1086F800118200080FB413B50B4904AB08680B4985
:1087080053F8042B09680193FFF7F4FE0446084B5D
:10871800186801F0B7FF0028F9D0204602B0BDE87C
:10872800104004B0704700BFCC000020C8000020F3
:10873800D80F002080EAE073A3EBE0738B4206DBDE
:10874800002801DD401A704702D008447047002015
:10875800704770B504460AF0D5FE2030402857D837
:1087680020462C490AF0C4FE28B120462A490AF0BE
:10877800F9FB0446F4E7204628490AF09BFE28B195
:10878800204625490AF0F0FB0446F4E72046244930
:108798000AF0AEFE30B1224920460AF0E3FB01465A
:1087A8001F480AE020461F490AF084FE40B11C49D0
:1087B80020460AF0D9FB01461A480AF0D3FB0446C2
:1087C800214620460AF0D8FC0546204629460AF0EC
:1087D800D3FC1549064628460AF0CEFC13490AF090
:1087E800C1FB014628460AF0C7FC11490AF0BCFB48
:1087F800014628460AF0C0FC0E490AF0B3FB0146C0
:1088080030460AF0B9FC014620460AF0ADFB70BDBF
:10881800002070BDDB0F4940DB0FC940DB0F49C0AA
:10882800DB0FC93FDB0FC9BF9A7C2E36FAAF4F3931
:108838003587083CA4AA2A3E08B503490AF094FBE8
:10884800BDE8084085E700BFDB0FC93F2DE9F04FC1
:10885800056885B0814628460C46FFF7EDFF80463F
:108868002846FFF776FFD9F8045006462846FFF752
:10887800E3FF07462846FFF76CFFD9F8089005463E
:108888004846FFF7D9FF82464846FFF762FF414650
:10889800814650460AF070FC4146834648460AF035
:1088A8006BFC5146019030460AF066FC494602903E
:1088B80030460AF061FC3946039050460AF05CFCE9
:1088C8004946206007F100400AF056FC29466060DE
:1088D800A56002980AF050FC014601980AF044FB92
:1088E8002946E06003980AF047FC014658460AF01A
:1088F80039FB3946206106F100400AF03DFC294663
:10890800606158460AF038FC014603980AF02AFBD1
:108918002946A06101980AF02FFC014602980AF046
:1089280023FB4146E06138460AF026FC206205B088
:10893800BDE8F08F2DE9F04107688AB04668856880
:108948000446084601A9FFF781FF019938460AF055
:1089580013FC0499804630460AF00EFC0146404656
:108968000AF002FB0799804628460AF005FC0146F2
:1089780040460AF0F9FA0299206038460AF0FCFBF2
:108988000599804630460AF0F7FB014640460AF052
:10899800EBFA0899804628460AF0EEFB0146404665
:1089A8000AF0E2FA0399606038460AF0E5FB069996
:1089B800074630460AF0E0FB014638460AF0D4FA8A
:1089C8000999064628460AF0D7FB014630460AF0C0
:1089D800CBFAA0600AB0BDE8F081074B10B51A8841
:1089E8001C4622EA00009042188002D0012001F0C3
:1089F80073FD208810BD00BFD0110020064B10B5B4
:108A08001A881C4610439042188002D0012001F0B9
:108A180063FD208810BD00BFD0110020024A936872
:108A280023EA0000906070476025002008B5104BCD
:108A38001A780023D9B2914207D20E49002051F882
:108A48002310013309680880F4E7322001F083FD20
:108A5800094B1B685A0309D5084B9B685B0305D46F
:108A6800BDE8084040F2DC5001F075BD08BD00BF0C
:108A78007C1500204C1500200025002060250020D2
:108A88004B4A69232DE9F34113704FF4FB6353807C
:108A9800BE231371EF2382F8D537002319461646F3
:108AA80082F8D637F25C0133B3F5FB6F81EA020135
:108AB800F8D13F4B3F4A83F8D6173F4B04275A60FB
:108AC80002F188325A600020013F17F0FF075ED09C
:108AD800394B3422DA60002454B100234FF400509B
:108AE80056F80480019307F057FB0428ECD11DE0E9
:108AF8004FF4302007F050FB0428E5D12E4D4FF4F9
:108B080030202B6943F002032B612C4B6B612B69DE
:108B180043F040032B6107F03FFB41F6FD732A69E0
:108B2800042803EA02032B61D7D0CDE7224D1FFAB0
:108B380088F22B694FF4005043F001032B6104F1D4
:108B4800006303F57E331A8007F026FB042814D14E
:108B58001B4B4FEA184823440193019B4FF40050E4
:108B6800A3F8008007F018FB41F6FE732A69042871
:108B780003EA02032B6106D0A6E741F6FE732A69D1
:108B880013402B61A0E70434B4F5FB6FA4D10A4A63
:108B98000428136943F08003136102D108F0E6FD4D
:108BA80010B90A2001F0E1FC02B0BDE8F08100BF75
:108BB80060250020230167450020024000F80308D3
:108BC80002F8030810B50E4C206801F0D9FB2068A4
:108BD8000022047A02FB02F3193B634303F6C41331
:108BE8005343192193FBF1F3064921F8123001325E
:108BF800072AEFD1BDE81040034901F079BB00BF57
:108C08006C100020A80F0020A42600202DE9F041B8
:108C180008F0ACFD10B90A2001F0A7FCAF4CB04930
:108C28004FF4FB6220460DF0DFFD94F8AC374FF4AB
:108C3800CC71022B84BF002384F8AC3794F8AC279E
:108C4800A84D01FB02F3E01800F5397023442860B1
:108C580093F8380301FB0242022803F54C7384BFE2
:108C68000020187292F838339F4A13700C2202FBC6
:108C780003439E4A03F2AE73136046F20902A368E7
:108C88001A401AB9954A43F400539360A368DE0763
:108C980003D54FF40050FFF7C1FEA368580409D567
:108CA8000820FFF7BBFE4FF40050FFF7B7FE012086
:108CB800FFF7B4FEA368190706D54FF40050FFF775
:108CC800ADFE0120FFF7AAFEA3689A0413D54FF45E
:108CD8000040FFF7A3FE814B93F88631012B03D1A7
:108CE8004FF40060FFF79AFE4FF48030FFF796FECE
:108CF8004020FFF793FEA3685B0603D54FF480304E
:108D0800FFF78CFE94F8DC21744B2AB193F8E0212C
:108D180012B1002283F8E0214FF0000C6746744E30
:108D2800744B1E6004EB0C03B3F8F4E14FEA5E01E8
:108D380001F077314FEA9E0303F03333C1EB0E00A5
:108D4800C11A4FEADE0303F01133CB1A03EB2313E6
:108D580003F00F32FF2392FBF3F31EF00108C3EB7D
:108D6800032318BF0137A2EB030318BFFFB2012B7F
:108D78000ADD022B40F0AE80B8F1000F00F0AA80A7
:108D88001EF0BC0F00F0A6800CF1080CBCF1200FFF
:108D9800C8D1013F012F00F29D80FFF713FF302259
:108DA800002155480DF02BFD544F554BD5F8008048
:108DB8001F60544B002108F17900C3F8008001F0CE
:108DC8001DFB514B80F001001870504B07F1260233
:108DD8001A604F4B07F1D0021A6098F8000003F0B0
:108DE80039FA28684B4B00F5C5721A6002F06AF828
:108DF800494B07F194021A60484B00221A809A7175
:108E0800474B2D6807F12C021A60464B05F21912E0
:108E18001A60454B05F289121A60444B07F10802A3
:108E28001A60434BDFF844811F60424B07F19C02F4
:108E38001A6007F1A603C8F800303F4BB4F8660182
:108E48001E600AF041F9C8F80800B4F868010AF091
:108E58003BF995F85C3008F1040288F8043095F87D
:108E68007830C8F80C0088F8053094F8DF31286E9F
:108E780088F81030314BC8F814501A60304B05F19F
:108E880064021A602F490AF077F901464FF07C50C6
:108E98000AF026FAB5F816412B4B186020460AF05E
:108EA80017F9014629480AF01BFA29490AF064F91A
:108EB800284A294B1560294A186005F16803136090
:108EC800274A05F211151560264A1760264A1360CD
:108ED800BDE8F08106F0B8FF5FE700BF602500201D
:108EE80000F8030844100020AC2400206C10002077
:108EF800EA26002064300020DC0E0020A426002092
:108F0800100F0020140F00200C000020B8160020BD
:108F1800F0050020200F0020D00E00201C0E00209D
:108F280014170020201200204C09002020160020D1
:108F3800241600206008002024090020481700207B
:108F480080170020DB0F49407C1700200000614497
:108F58004C3D0F44800700205C0800207407002067
:108F68004C080020540800207C0600202412002011
:108F780008B5FFF785FDFFF749FEBDE80840012069
:108F880001F0AABA344B354A1B68126810B51A604A
:108F9800334A11685960516892689960DA60314AB9
:108FA800116819615168926859619A612E4A11686D
:108FB800D9615168926819625A622C4A11881985D8
:108FC800518859859188D2889985DA85284A1188E7
:108FD80019865188598692889A86264A1188D98690
:108FE800518892881987194621F83A2F224A107811
:108FF8000022824206DA214C34F81240013221F86C
:10900800024FF6E71E4A1288A3F864201D4A128808
:10901800A3F866201C4A1188A3F86C10518892881E
:10902800A3F86E10A3F87020184A3B2112689A66BC
:10903800174A126892FBF1F2B2F5967FC8BF4FF05B
:10904800FF325A67134A1288A3F87820124A5289C5
:10905800A3F85E2010BD00BF5C2D00209C300020CE
:10906800281500203415002040150020EC100020A1
:1090780028100020D61000207C1500204810002061
:1090880054230020CC0F00202E100020E0100020D8
:109098000400002068100020341000202DE9F84357
:1090A80005460E460D4B002493E88003B44213DABC
:1090B8007B1933F9140008EB050333F9142009EB85
:1090C800050333F9143001341344022293FBF2F3FD
:1090D800C01A08F0A1FEE9E7BDE8F8835C2D00207E
:1090E80070B5472008F0E8FD174B1B681B0307D530
:1090F800164B174A5B6810681B68C01A08F07DFE9B
:10910800144E154C154D307808F077FE2368286802
:10911800C01A08F081FE63686868C01A08F07CFE0F
:109128000F4B188808F069FE0E4B188808F065FE8A
:109138000D4B188808F061FE337823742B68A36000
:109148006B68E36070BD00BFE02E00205C2D00203E
:109158009C30002012110020482D002014110020FE
:10916800101100200E110020701000207FB5254C32
:10917800254E264D2649274A274B20B127480088E7
:10918800B0F5805F30D2308889791278ADF8040064
:1091980028781C4D1B788DF806008DF807108DF87F
:1091A800082001A8294606228DF809300DF00CFB8D
:1091B80028B30198BDF808302860AB80532008F028
:1091C8007BFD208808F019FEA07808F016FEE378E9
:1091D80001A80193237902936379039308F074FD3E
:1091E8000E4B00221A800AE0308889792080127894
:1091F80028781B78A070E17022716371DEE704B0F3
:1092080070BD00BF3C120020D01100200C110020BE
:109218001C0E00204B0E0020B00E0020002F002056
:10922800A0F17D03012B70B504460D460A4E05D802
:1092380030687D2101F03DFA84F020043068214631
:1092480001F037FA35B12B881C4404EB142404F0E0
:10925800FF042C8070BD00BFC01100200A4A13888B
:1092680001331380094A136801331360084A1388CD
:1092780001339BB2202B01BF00231380054A1388BA
:1092880008BF013313807047002F0020E82E00200C
:10929800EC2E0020EE2E002038B53A4B05461B7800
:1092A8000C46083B012B6BD8452008F005FD2846E5
:1092B80008F002FD0C2D23D004D80A2D0AD014D8AA
:1092C80035B138BD0E2D4BD02ED3FF2D50D038BD23
:1092D800206849E0207808F0EFFC62796378002A7A
:1092E80014BF80200020184300E0207808F0E4FC38
:1092F800A07808F0E1FCE07808F0DEFC20793BE09B
:10930800B4F9000008F06FFDA07808F0D5FCE0780B
:1093180008F0D2FCB4F9040008F065FDB4F90600C1
:10932800BDE8384008F05FBD637820788BB180F0E5
:10933800800008F0C1FCA468E0B208F0BDFCC4F3EA
:10934800072008F0B9FCC4F3074008F0B5FC200E6C
:1093580012E008F0B1FC6068BDE8384008F05CBD78
:10936800206808F04AFD6068BDE8384008F045BD4F
:10937800054808F07FFC0020BDE8384008F09CBC98
:1093880038BD00BF382D0020A5BC01082DE9F04FDD
:10939800BE4B8BB01A880193BD4F002A40F0A980BC
:1093A80042F20103B7F8D207BA4EC21A50425041EE
:1093B800FFF7DCFEFFF7E6FD34684920254608F094
:1093C8007BFCB54B04F11C09186808F016FD55F82C
:1093D800040B08F012FD284606F0E8FC04F1100022
:1093E80006F0E4FC4FF01008AC4D01232A6803FA9C
:1093F80008F3134203D0D9F8000008F00DFD08F176
:109408000108B8F1130F09F10409EDD104F128009E
:1094180006F0BCFCB7F84431B4F92E00C01A08F0C5
:10942800ECFC2B68DB0408D59D4BB4F864001B8862
:10943800181AC0F30D0008F0E0FC2B68980403D557
:10944800B4F8660008F0D9FC2B68590503D504F177
:109458006C0006F09BFC2B681A0502D5A06E08F07C
:10946800DBFC2B685B0402D5606F08F0D5FC2B6829
:10947800180403D5B4F8780008F0BFFCA04604F13E
:10948800300006F083FC04F1360006F07FFCB7F8E4
:10949800443138F93C0F0127C01A08F0AEFC814B63
:1094A8001B789F4208DA38F9020FB4F93C300137CB
:1094B800C01A08F0B1FCF2E72B68990505D5B4F994
:1094C8005E00A0F2DC5008F0A7FC326876487260B3
:1094D800B260121A9110754A4A43531C032293FB37
:1094E800F2F202EB42029A1A7C2303FB0203336076
:1094F800D6E16F4B6F4A1B6811688B4206D00AA9E8
:1095080041F8203D00201360FFF7C6FE019B97F845
:10951800D2171B8897F8D3070B44013BB3FBF0F233
:1095280000FB12338B4280F086815A4F0120FFF7EF
:109538001DFEFFF727FD50203E687D6808F0BCFB44
:10954800BA683B6810681B687A680344106806F1BB
:109558001C0BA3EB400008F05FFC6A68736802A864
:109568009B1A0293AA68B36805F11C089B1A039317
:10957800EA68F36810249B1A049306F017FC2A691A
:10958800336902A89B1A02936A6973699B1A039349
:10959800B369AA699B1A049308F096FB3F49012214
:1095A8000B68A2401A428A4606D0DBF80000D8F8B9
:1095B8000030C01A08F030FC0134132C0BF1040BF6
:1095C80008F10408EAD106F1260005F12601002376
:1095D80031F9024F30F9022F121B02AC44F8232054
:1095E8000133042BF4D103214FF000094FEA89031A
:1095F8005FFA83F902AB53F821206AB102F108003F
:109608000F2802D849F0010906E08032FF2A94BFEA
:1096180049F0020949F0030911F1FF31E6D2484641
:10962800002408F049FBA0460DF1080B09F00302DD
:10963800022A16D0032A1DD0012A4ED1B8F1000FF4
:1096480005D1DBF8004090462401E4B245E0DBF8A0
:1096580000004FF0000800F00F00204308F02CFB3A
:109668003BE0B8F1000F0CD0DBF80000C0F30310AA
:1096780020432CE0B8F1000F1ED19BF8010008F040
:109688001BFB9BF8000008F017FB26E0EC2E0020DF
:10969800602500205C2D0020E82E0020E02E002010
:1096A800DC2E00207C150020682D0020DF7BEFBD1C
:1096B800F42E0020F02E0020DBF80000C0F3033069
:1096C800204308F0F9FADBF80000C0F3071008F0AF
:1096D800F3FADBF800402401E4B20BF1040B06AB0B
:1096E8009B454FEA9909A1D1B8F1010F02D1204653
:1096F80008F0E2FADAF8003013F480541FBFB6F825
:109708006420B5F864100124521A18BF02929A0412
:109718000AD50AAA02EB8401B5F86600B6F86620F5
:109728000134121A41F8202C580513D502AA02EB6D
:10973800840C06F16A0E05F16A0000223EF9021F48
:1097480030F9028FC8EB01014CF822100132032ACC
:10975800F4D10334190508D50AAA02EB8400A96ECE
:10976800B26E0134521A40F8202C5A0408D50AAABD
:1097780002EB8400696F726F0134521A40F8202C92
:1097880018040BD50AAB03EB8402B5F87810B6F8C9
:10979800783001345B1A42F8203C00E0FCB1012C1F
:1097A80003D1029808F038FB19E0631E002002AAD2
:1097B80052F823204000C0B20AB140F00100013B3A
:1097C800F5D508F079FA4FF0000802AB53F82800F5
:1097D80008B108F021FB08F10108A045F5DB3020AD
:1097E8000321FFF75BFC36200321FFF757FC2F4BC3
:1097F8003C201978FFF752FCDAF80030990506D5B5
:10980800B6F95E00B5F95E30C01A08F005FB3A6893
:1098180027487B687A60121A9110264ABB604A432F
:10982800531C032293FBF2F202EB42029A1A7C23A6
:1098380003FB02033B60204B1B681A0630D51F4C04
:109848001F4D22682B689A420BD162686B689A4256
:1098580007D1019B1B88102B11D11A4B1B885B0663
:109868000DD1482008F028FA206808F0D5FA606879
:1098780008F0D2FA23682B6063686B600EE0124A26
:109888000F4B11782A7C914208D1104A99681068C8
:10989800884203D15268DB689A4201D0FFF720FC66
:1098A80008F0DAF90BB0BDE8F08F00BF7C15002096
:1098B800682D0020DF7BEFBD0025002074100020FC
:1098C800482D0020EE2E0020121100201411002037
:1098D8002DE9F84F0C9EC2EB030B394C0B9B00296A
:1098E80014BF4FF0060A4FF0040AF61A63680546DB
:1098F8000133904613D1236853455ED2314A032B76
:1099080098BF294652F823202F4808F0C3F9636806
:109918000022013363602D4B05469A7113E0002540
:1099280011E02B4A1278954240DA0B9BE3B109FB10
:1099380006F2995C01228A40264909680A4213D135
:10994800636801336360D4F804900A9B1C4F9945FF
:10995800E7DB2BD10A2008F0AFF93B6801333B6005
:109968004FF0FF337B6021E0184A917921B12C2018
:1099780008F0A2F9013501E00121917109FB0BF30F
:10998800226808EB030752B958F8030008F072F987
:1099980097F9041005444B1CD2D00F4802E03A4412
:1099A8000E48117908F076F90544C9E72068504552
:1099B8002CBF00200120BDE8F88F0020BDE8F88FFB
:1099C800F82E002018980108B0BC01083C120020AD
:1099D80054000020E02E0020BFBC01087EBF010813
:1099E80030B585B004AC002524F8025D0091ADF8CF
:1099F800060021461020FFF713FC9DF806002146BB
:109A0800FFF70EFC9DF807002146FFF709FC9DF8BB
:109A180000002146FFF704FC9DF801002146FFF7EE
:109A2800FFFB9DF802002146FFF7FAFB9DF80300B3
:109A38002146FFF7F5FB9DF80E002946C043C0B24A
:109A4800FFF7EEFB05B030BD10B5054C206800F0FF
:109A58002DFE18B1206800F026FEF6E710BD00BF05
:109A680090110020F8B504460E46174600252046FA
:109A780020210CF0FAFE0446D0B1013420460CF047
:109A880057FFB0F5617F05DB40F634039842A8BF65
:109A9800184601E04FF46170A0F56170192390FB3E
:109AA800F3F00DB9307000E070703B7801333B7013
:109AB8000DB90125DBE72046F8BD30B505460C4653
:109AC800134629462246BDE830400148FEF712BE3B
:109AD800B4BD01087FB504780646E4B9354B1921B1
:109AE800186800EB840090F87B5090F879204D437B
:109AF80005F5617590F87A30009590F87C0041433F
:109B080001F5617101912C4821460134FEF7F2FDFF
:109B1800142CE3D14BE00CF00BFF1328054641DC75
:109B2800244B701C1C68202100238DF80F300CF08A
:109B38009CFE1E35064670B1013630460CF0F8FE24
:109B480019289FBF04EB850358709DF80F30013327
:109B580098BF8DF80F30304620210CF086FE06465F
:109B680070B1013630460CF0E3FE0D289FBF04EBC0
:109B7800850398709DF80F30013398BF8DF80F302A
:109B880004EB85043046E11C0DF10F02FFF76AFF74
:109B98009DF80F30042B0AD0601C002104220CF021
:109BA8002EFE04E0054800211322FFF786FF04B0CB
:109BB80070BD00BF44100020D3BD0108DCB6010809
:109BC800014807F0C9BB00BFE8BD0108F8B5047833
:109BD800064674B9304D2146B5F8C621B5F8C831E6
:109BE8002E480134FEF786FD042C05F10405F2D158
:109BF800F8BD2B490CF00CFEA8B9274B4FF47A712D
:109C08004FF4FA62A3F8C611A3F8C821A3F8CA1141
:109C1800A3F8CC21A3F8CE11A3F8D021A3F8D21130
:109C2800A3F8D421F8BD30460CF082FE032805467F
:109C38002BD8304620210CF018FE044630B10134F0
:109C480020460CF075FE0126074600E00646204631
:109C580020210CF00AFE10B9BDE8F840B0E7013049
:109C68000CF066FE012EF7D140F2DC53A7F2EE228B
:109C78009A42F1D8A0F2EE229A42EDD8064B7035FE
:109C880003EB8503DF801881F8BD06480021032215
:109C9800BDE8F84011E700BF60250020F6BD0108C7
:109CA800A6B6010828C301082DE9FF410478054636
:109CB800002C34D16D4807F04FFB6D4D68690021C9
:109CC80009F0EEFB002840F0CE8021466948FEF7F7
:109CD80011FD68696946FEF793FB01466648FEF781
:109CE80009FDA8696946FEF78BFB01466248FEF745
:109CF80001FDE8696946FEF783FB01465E48FEF709
:109D0800F9FC286A6946FEF77BFB013401465B488B
:109D1800FEF7F0FC0C2C05F11005CFD1A3E0584953
:109D280005220CF0B9FD38B9514B0022034410301C
:109D3800C0285A61F8D196E02846524904220CF00E
:109D4800ABFD04462846002C3FD120210CF08DFDA8
:109D5800002800F08880451C28460CF094FD074632
:109D6800494B53F824601EB9484807F0F5FA7AE0E1
:109D780028463146FAB20CF08FFD01340028EFD1A5
:109D88003B4B0021C2181030C02851619E46F7D1C4
:109D98003F4B03EBC402D2F804C09846BCF1000F55
:109DA80004D131463B48FEF7A5FC53E0002718F8DC
:109DB80034309F42F5DA3B010EEB0305143563445A
:109DC8000FCB013785E80F00F1E70CF0B1FD0B2848
:109DD800064643DC284620210CF047FD054648B1DD
:109DE80001352846FEF776FA214B012403EB0613CA
:109DF800586100E00446284620210CF036FD05464F
:109E080040B101352846FEF765FA194B013403EBDA
:109E180006139861284620210CF027FD054640B11D
:109E280001352846FEF756FA114B013403EB0613A9
:109E3800D861284620210CF018FD10B9FFF7C0FEA4
:109E480011E00130FEF746FA094B032C03EB061626
:109E58003062F3D11048FFF727FF04E00F480121D3
:109E68000C22FFF72AFE04B0BDE8F08109BE010804
:109E78006025002024BE01082ABE010842C001084E
:109E8800A6B60108ACB60108A0AE0108E1B5010804
:109E9800E4BC0108B1B601087BB40108DCB60108CE
:109EA800F0B5047887B0064614BB514B19201968E1
:109EB800062303FB041191F8CA5091F8CE204543BC
:109EC80005F5617591F8C930009591F8CB50C83106
:109ED800684300F561700190087902904979454816
:109EE800039121460134FEF705FC0C2CDDD17CE002
:109EF8000CF01EFD0B28044672DC3D4B701C1D68DF
:109F0800202100238DF817300CF0AFFC064680B1F5
:109F1800013630460CF00CFD03289FBF062303FBD7
:109F2800045383F8CE009DF817309CBF01338DF899
:109F38001730304620210CF098FC074680B10137D5
:109F480038460CF0F5FC0D289FBF062303FB04538D
:109F580083F8C9009DF817309CBF01338DF817307E
:109F680006266643A9193846CA310DF11702FFF7CC
:109F780079FD20210CF079FC074670B1013738468D
:109F88000CF0D6FC14289FBF9DF8173076190133C2
:109F980086F8CC0098BF8DF81730384620210CF091
:109FA80064FC78B101300CF0C3FC0D289FBF062378
:109FB80003FB045383F8CD009DF817309CBF013391
:109FC8008DF817309DF81730062B0ED0062202FBAD
:109FD80004500021C9300CF012FCFFF7F1FD04E039
:109FE800054800210B22FFF768FD07B0F0BD00BF50
:109FF800441000202EBE0108DCB601082DE9F3410B
:10A00800047880464CB9204601A908F09DF901342E
:10A01800FFF7F4FF122CF6D168E00CF089FCC6B209
:10A02800112E5ED8334C06F1D00704EB470308F134
:10A03800010020219D780CF018FC18B9AA1E554281
:10A04800554139E04378682B06D0732B07D0612B34
:10A0580013D14FF0000804E04FF0010801E04FF081
:10A068000208A8F102035D4200F101004FF020014F
:10A078005D410CF0FAFBD8B115B9FFF7A1FD35E049
:10A0880001300CF055FC40F2ED2380B2984205DD1A
:10A0980040F6CA039842A8BF184601E040F2EE20F5
:10A0A800A0F2EE20192290FBF2F004EB4703D870DF
:10A0B80004EB470383F8028004EB4704A3780E4AB5
:10A0C800D25C4DB1E17819234B430C48314603F279
:10A0D800EE23FEF70FFB09E031460948FEF70AFBBD
:10A0E80004E0084800211122FFF7E7FC02B0BDE8B0
:10A0F800F08100BF60250020309801084EBE01089D
:10A1080060BE010828C30108002208490C2303FB8C
:10A1180002135968814204D10022C2621A725A603D
:10A1280070470132042AF0D1704700BFE0220020B6
:10A1380010B5084B0022196801EBC20393F90240DD
:10A14800844201D1981C10BD0132042AF4D10020A8
:10A1580010BD00BFDC220020F0B5027887B08AB9B4
:10A168004A4C04F1200694F8F2210023484950B2E1
:10A17800595681426DD00C33302BF7D10834B44294
:10A18800F1D180E0002204920592451C0CF0D0FB2E
:10A19800C4B260B2FFF7CCFF074618B18DF8104083
:10A1A800012400E00446284620210CF05EFB054609
:10A1B80038B1013528460CF0BBFB0134ADF812006C
:10A1C800E4B20026284620210CF04FFBB0B3451C12
:10A1D80028460CF0ADFB00222E495FFA82FE51F8AA
:10A1E8002230834204D00132082AF5D1002300E04E
:10A1F800734651F82320824220D1022E0FD0032E1D
:10A2080012D05A1E012ED2B204D0042A13D88DF8C7
:10A2180014300EE0042A0ED88DF8153009E0052B0D
:10A2280009D88DF8173004E09A1E052A03D88DF84E
:10A2380016300134E4B20136042EC3D1052C03D8FC
:10A2480007B0BDE8F040BBE404AB03CB38607960ED
:10A2580019E094F8F7010F4B94F8F65153F82000E1
:10A26800B4F8F421009094F8F90153F82000019013
:10A2780094F8F80153F8200053F825300290064866
:10A28800FEF738FA7AE707B0F0BD00BF6025002076
:10A29800E022002038A001086FBE010838B14388C9
:10A2A80011EA030003D08B420CBF01200220704743
:10A2B80030B50A4B0A491C680A78032A0AD813469B
:10A2C800551C04EBC303EAB29D882842F5D00A70F6
:10A2D800981C30BD0A70002030BD00BFDC22002071
:10A2E80044120020014B00221A70E1E744120020BA
:10A2F8002DE9F047877890F803C0BBB2C7F1640E28
:10A3080003EB83065C42C3F178001C4D5FFA8EFEB6
:10A318007600CCF16408A4B280B2A3B20FFA83F934
:10A32800B9F1000F04DC002B14BF3B46012300E009
:10A33800734609FB09F25B4302FB0CF292FBF3F351
:10A34800434403FB09F30A2293FBF2F333449BB221
:10A3580025F8023FB1F800904A880A34C9EB020A8E
:10A368001AB202FB0AF24FF47A7392FBF3F3A4B227
:10A378004B4484422B80D0D1BDE8F08744120020A2
:10A3880010B544780078002240F6C41102FB02F3AD
:10A39800193B634303F6C4135343434393FBF1F35D
:10A3A800034921F812300132072AEDD110BD00BF50
:10A3B8005E120020104B043033F91000B0F5617FB5
:10A3C80005DB40F633039842A8BF184601E04FF476
:10A3D80061700A7819235A4302F28332824208DAFA
:10A3E8004A78534303F283338342B4BF00200120E9
:10A3F80070470020704700BF3C25002010B500F1D1
:10A40800500302788A4203D18478C278944204D3F4
:10A4180004309842F5D1002010BD012010BD1FB5B1
:10A42800084B1B681B0309D58DF804000391012311
:10A438000D2001A98DF80530FEF72EFF05B05DF857
:10A4480004FB00BF002500201FB5084B1B681B0339
:10A4580009D58DF80400029100230D2001A98DF87B
:10A468000530FEF719FF05B05DF804FB0025002054
:10A4780010B5064B00241C7008F008FB044B83F849
:10A488002840DC621C865C6310BD00BF6830002079
:10A498004412002010B510B9BDE81040E8E70023C9
:10A4A8000C225A430A4C1119125D824203D001331F
:10A4B800102BF5D110BD074B586B18B14A7840786E
:10A4C800824203D2002259631A86DA6210BD00BFA5
:10A4D8006CA001084412002010B540001428A8BF41
:10A4E80014200023074A022199540B449918142474
:10A4F800834201F8014CF5DBFF21D1540F20BDE860
:10A508001040C7E7D824002010B50A4A0A4B116842
:10A518009B6800BF12689142F7D1084A4FF47A70DD
:10A52800946B00FB04F2D31AB3FBF4F300FB013085
:10A5380010BD00BF2425002010E000E044120020D8
:10A5480038B50446FFF7E0FF0546FFF7DDFF401B7F
:10A55800A042FAD338BD10B504462CB14FF47A7036
:10A56800FFF7EEFF013CF8E710BD38B540F2DB1508
:10A578006843114B10225A6108221A61851E0B2468
:10A58800013C14F0FF040FD00B4B2846DA6882F028
:10A598001002DA60DA6882F00802DA60FFF7DBFF9F
:10A5A8001920FFF7D8FFEBE7044A054B1A60054A64
:10A5B800054BDA6038BD00BF000C0140EFBEADDED0
:10A5C800F04F00200400FA0500ED00E0024A13688D
:10A5D80001331360704700BF24250020024BDB6B5A
:10A5E80003B11847704700BF4412002003685B6935
:10A5F80018472DE9F743064689469DF828801146F5
:10A608001A469DF82C3000250C2068431A4FC419AF
:10A61800C057B04202D1207A20B126E00135042D7E
:10A62800F2D122E0012E0AD003DCF6B900931348D8
:10A6380007E01E2E0AD01F2E17D1012006E0104871
:10A648000093434602F045FF044605E004F0ACFAE7
:10A6580041460446FFF7CAFF4CB10C2303FB0575BE
:10A66800267185F808906C6001E0002000E0204623
:10A6780003B0BDE8F08300BFE022002000380140AD
:10A688000044004003681B69184710B5044620467B
:10A69800FFF7F8FF18B90A20FFF75DFFF7E710BDCD
:10A6A8000368DB68184703689B68184703685B689A
:10A6B800184703681B68184710B508F009FD002102
:10A6C800044608F015FF08B1204601E004F10040F7
:10A6D800054908F005FE054908F04EFDFEF7ACF8FF
:10A6E800034B186010BD00BF8096184B35FA8E3C9E
:10A6F8003C0000202DE9F04105460E46078A838973
:10A708009BB21F40002F37D0B7FA87F24FF00043B3
:10A71800D340DB4399B21F40A2F11B032982042BCB
:10A72800F0D8DFE803F0221F1C190300746A24B173
:10A73800013C0023A4B2736201E0AC8DA4B2D6F848
:10A748002080B8F1000FDDD0D8F80030404621460F
:10A758009847D8F80480F4E73068A98E08E0706854
:10A76800298F05E0B068A98F02E0F068B5F84010BD
:10A77800036889B29847C5E7BDE8F08138B50D4B45
:10A788000D4D99680D4B1A681C465288114203D02A
:10A79800FFF7BAFE286007E0FFF7B6FE2B6898427D
:10A7A80082BFC01A064B186023685A68054B5A6165
:10A7B80038BD00BF000C014084120020880700202B
:10A7C8000400002000040140F8B59C4B04461B68B7
:10A7D800187818B1012800F06A819AE2242C984D63
:10A7E8000CD006D80A2C00F0D9800D2C00F0D680A9
:10A7F80048E12A2C06D02C2C04D043E1287168713A
:10A80800A87150E18F4B69792F7900208C4A5854F0
:10A818002FBB1978D771472921D1597850291ED1D2
:10A828009978472907D1D978472904D11979412935
:10A8380001D10121D1719978824A522903D1D17865
:10A848004D2900F0688299787E4A472907D1D17846
:10A85800532904D11279562A04BF0322EA71EA79EE
:10A86800774E022A39D0032A4CD0012A40F085803D
:10A87800BA1E072A00F28180DFE802F004080F13ED
:10A888001A257F2A07F0B4FCA86076E01B78532BC2
:10A8980073D1AB685B42AB606FE007F0A9FCE8607E
:10A8A8006BE01B78572B68D1EB685B42EB6064E088
:10A8B8001B78302B644B1A788CBF42F0020222F0CE
:10A8C80002021A7059E0002007F0F2FC287454E0E4
:10A8D800002007F0EDFC68824FE0072F06D0082F14
:10A8E8004BD1012007F0E4FCF08246E0012007F09C
:10A8F800DFFC41F2184358434FF47A73B0FBF3F08E
:10A90800B0823AE0022F07D0032F0AD1002007F0C7
:10A91800CFFC4E4B187030E0002007F0C9FC3076B1
:10A928002BE02AD93A1F9210337E0132D2B2013B72
:10A9380002EB8303DBB2102B1FD8F91EC2F1010210
:10A9480001EB8202D2B2012A0BD0042A11D10020D5
:10A958005E1E07F0ADFC3E4B002298553D4B9A55C4
:10A9680007E03D4A5E1E0020935507F0A1FC3B4BD3
:10A9780098553B4A136801331360314B2A2C18BF92
:10A988009A7907F101074FF000000CBF01225440EB
:10A998002F7168710CBF5A769C7184E0687E00281C
:10A9A80048D0304B13F8012D2F495A708B42F9D1FA
:10A9B800244A234C13785278402B85BF373B1B0120
:10A9C8001B01DBB298BF03F0F003402A8CBF373A73
:10A9D800303AD2B21344AA79DBB29A4227D1212362
:10A9E8000B702249E0790B68012803F101031E4A24
:10A9F8000B600AD002281CD172231370A28A1C4B48
:10AA08001A80E28A1B4B1A8013E0672313700E4BDF
:10AA18001B789F070ED5184BA2681A60E2685A6027
:10AA2800227C164B1A70628A154B1A8002E03F236B
:10AA38000B70002000236B7635E000BFAC070020C8
:10AA4800841200202C2500200C11002088100020E2
:10AA5800B9100020A91000208910002099100020AA
:10AA6800D8210020C4020020B0020020E4210020E8
:10AA78000E11002070100020141100201211002067
:10AA8800101100206B79687E0E2B9FBFA54A591CB8
:10AA98005171A54A98BFD454A24A18B993795C4019
:10AAA800947100E00020003018BF0120F8BD9D4BD4
:10AAB8000022997E082900F22C81DFE801F0050BBD
:10AAC8000F15202B475D6700B52C40F02281DA7600
:10AAD800012239E0622C08BF022235E003229A766F
:10AAE8001C775C779C7714E104229A765A7F997FC9
:10AAF8002244D2B25A770A449A77DC7709E10522D0
:10AB08009A765A7F997F2244D2B25A770A449A7722
:10AB18001C84FEE006229A765A7F997F2244D2B29C
:10AB28005A770A449A771A8C02EB0424A4B2B4F533
:10AB3800AC7F82BF7B4A0121D17600221C845A84D3
:10AB4800002C40F0E68007229A76E2E05A7F997F4F
:10AB58002244D2B25A770A449A775A8CB2F5AC7F1B
:10AB68003EBF7049891881F824400132198C92B28D
:10AB780091425A84E7D9CCE008229A765B7FA342B7
:10AB880000F0C780674B0122DA760DE0674D9A76B0
:10AB980015F8012D6A70664A9542F9D1997F614A84
:10ABA800A14206D03F232B70624A53680133536099
:10ABB800AFE06148016801310160D07E10B13E23E9
:10ABC8002B70A6E021212970D17F062941D004D815
:10ABD800022907D0032923D0F8BD122959D03029DA
:10ABE80067D0F8BD5021946A297054494C60D46AE2
:10ABF8000C60516B4FF47A7491FBF4F1504C218046
:10AC080092F87C114F4A19B1117841F0020102E023
:10AC1800117821F002011170012283F87D2169E089
:10AC28005321297092F82910CE0705D592F82820CB
:10AC3800D51E6A426A4100E0024602F0010183F82B
:10AC48007C11002A56D13F490A7822F002020A7084
:10AC580050E04F21297092F82F10CC0705D592F8B3
:10AC68002E20D11E4A424A4100E0024602F001016C
:10AC780083F87C1122B933490A7822F002020A705B
:10AC880093F85310304A1170B3F850102F4A1180BE
:10AC980030E05621946B29702D490C8042F21074D3
:10ACA800D16B91FBF4F12B4C2180012182F87E11AC
:10ACB80020E04921297092F82810274A102988BFD6
:10ACC80010211170254914780022A2420ED20E7A62
:10ACD800234D56554E7A234D5655CE7A224D56550C
:10ACE80011F80C6F214D56550132EEE720490A68DC
:10ACF80001320A6093F87D310A4A002B3AD092F863
:10AD08007E31BBB3002182F87D1182F87E1118468E
:10AD1800F8BD0020F8BD1279432A7FF494AD0222D1
:10AD2800EA7190E5841200202C250020C40200203E
:10AD3800B00200208C070020E4210020141100201C
:10AD4800101100200C1100201211002046000020D4
:10AD58000E1100207010002088100020A81200207A
:10AD68008910002099100020A9100020B910002097
:10AD7800D8210020F8BD0449044B09680022187046
:10AD88005A6199611A777047242500208C070020A2
:10AD9800F8B5101A0D461F4608F09AF90446781BB4
:10ADA80008F096F9174B079E196808F0E5F921464F
:10ADB8000546204608F0E0F929460746284608F0E7
:10ADC800DBF90146384608F0CFF80CF089F90E494E
:10ADD80008F0D2F908F0BCFB069B2946186004F17C
:10ADE80000400BF0F1FF094908F0C6F9084908F0DE
:10ADF800BBF808F087FB0028BCBF00F50C40A0306A
:10AE08003060F8BD3C0000202C7D8E3FA00CB3457F
:10AE180000A00C4644F25063984203DDA0F50C40B4
:10AE2800A0387047034B9842BCBF00F50C40A030D7
:10AE3800704700BFB0B9FFFFF7B50368174C184D4E
:10AE480023600B68174E63600068FFF735FC95E8D0
:10AE58000300154B0196009394E80C00FFF798FF48
:10AE68003668124B60681E606B68114FC01A08F094
:10AE78002FF9104B196808F07FF908F043FB2A688E
:10AE8800236878609B1A3B600B4B1E600B4B1B685A
:10AE9800DA880B4B1A8003B0F0BD00BF4C240020A9
:10AEA8001411002058240020542400209424002049
:10AEB8005C2400203C0000208C240020200F00206F
:10AEC8008824002070B50446407908F0FDF81E4932
:10AED80008F006FA1D4D1E4E2860E07B08F0F4F8D5
:10AEE800194908F0FDF9EE606860A07908F0ECF8FF
:10AEF800184908F0F5F9184D2860207C08F0E4F8A6
:10AF0800114908F0EDF96860A07E08F0DDF81349F2
:10AF180008F0E6F9EE60A860E07908F0D5F80D4988
:10AF280008F0DEF90E4D2860607C08F0CDF806497F
:10AF380008F0D6F96860E07E08F0C6F8074908F01E
:10AF4800CFF9EE60A86070BD0000C84264240020FC
:10AF58000000FA44000020417424002000007A44D4
:10AF68009824002010B50C4C23789B0713D50B4B65
:10AF78001B78042B0FD90A4A0A4B106852681860CC
:10AF88005A60FFF799FB084B1A88084B1A802378F8
:10AF980043F00103237010BD0C1100201211002092
:10AFA8001411002074100020E4100020A8240020B0
:10AFB800164B13B51B681B0325D5154B154C1B7871
:10AFC80015498DF80030154B20681B788DF8013035
:10AFD80008F0D2F808F0BCFA11498DF80200606850
:10AFE80008F0CAF808F0B4FA8DF80300A06808F071
:10AFF800AFFA0C4B8DF804001B780A2069468DF8CF
:10B008000530FEF749F902B010BD00BF0025002049
:10B01800F2240020142500200000204110250020E3
:10B0280000007A44F6240020054A137883F00103CF
:10B038001370044A00231360034A1360B8E700BF83
:10B04800F62400200C25002008250020014802498C
:10B05800FFF750BB00080040F815002001480249DE
:10B06800FFF748BB00040040D01500204FF0804097
:10B078000149FFF73FBB00BFA8150020014802495E
:10B08800FFF738BB002C0140801500200148024919
:10B09800FFF730BB002C014080150020254B10B570
:10B0A8005A43254B254C1B680139B3FBF2F2038840
:10B0B800013AA04289B292B29BB212D004F5006460
:10B0C800A0420ED0B0F1804F0BD0A4F59834A04226
:10B0D80007D004F58064A04203D004F58064A04240
:10B0E80002D123F070039BB2154CA04206D004F5A0
:10B0F8008064A0421CBF23F440739BB203800F4BB3
:10B108008185984202850FD003F5006398420BD0E1
:10B1180003F54063984207D003F58063984203D053
:10B1280003F58063984201D10023038601238382BB
:10B1380010BD00BF40420F0050000020002C01400D
:10B148000010004073B505460068FFF7A7FF2A689E
:10B158000124138800269BB243F001031380EB7A85
:10B1680001A88DF804308DF805408DF806608DF83B
:10B17800074006F057FEEB7A1B2B0BD1192301A8C9
:10B188008DF804308DF805408DF806608DF807407D
:10B1980006F048FE02B070BD0C4B800A98420CD0F5
:10B1A80004D8B0F5801F0CD101207047084B984295
:10B1B80005D04933984206D003E0022070470320A7
:10B1C8007047FE2070470020704700BF0100100044
:10B1D800020010002DE9F843046807462046884617
:10B1E8009146FFF7D9FF03284BD8BA7A9108B8F1EE
:10B1F800000F06D1A589AEB202258D4026EA0505C5
:10B20800A5810A2303FB00131F4A42F82380043355
:10B2180042F82390B8F1000F07D0BD7AA189AD0894
:10B228000223AB400B439BB2A3812823434303F182
:10B2380020011144EFF31286502585F3128803F19B
:10B248000C051C331544134455F8047F17B10F60DF
:10B25800296804319D42F7D100230B60F3B283F3D0
:10B268001188282303FB0020036A23B1A3899BB21A
:10B2780043F0010304E0A38923F001031B041B0C22
:10B28800A381BDE8F88300BF80150020FFF776BAD8
:10B29800FFF774BAFFF772BA014802F0B7B800BFF7
:10B2A80004140020014802F0B1B800BF581400206F
:10B2B8000C4B4FF400525A604FF6FE730A48D0F810
:10B2C800082211680B401360D0F8F821D0F8FC313F
:10B2D8009A4203D000F5EA7002F0CAB8012380F858
:10B2E8001832704700000240841200202DE9F74F01
:10B2F8002F4C054627683846FDF79EFA064638461D
:10B30800FDF727FA676881463846FDF795FA0190F8
:10B318003846FDF71EFAD5F804A0074631465046D0
:10B3280007F02AFFD5F8088083464946404607F0CB
:10B3380023FF0146584607F015FE019B29688346FE
:10B34800184607F019FF49460546504607F014FF0E
:10B35800394607F011FF0146284607F005FE394631
:10B368000546404607F008FF314607F005FF01464D
:10B37800284607F0F9FD014658460BF025FD0D4912
:10B3880007F0FAFE0C4907F0ABFFA16807F0ECFDE7
:10B398000A4907F0A5FF0BF03FFC83B21A0444BF2B
:10B3A80000F5B47083B218B203B0BDE8F08F00BFE7
:10B3B800AC1400200000E144DB0F494000002041AC
:10B3C8002DE9F04F89B00593A24B80461B88049263
:10B3D800980737D540F2E632129B9F48DC89B0F9CE
:10B3E80000301B1B03F2F315954203D8002BB8BF9E
:10B3F8005B4201E04FF4FA73B0F9022040F2E63004
:10B40800121B02F2F314844203D8002AB8BF524236
:10B4180001E04FF4FA729342B8BF13460522C3F510
:10B42800FA7393FBF2F30A22643B534398F81C2007
:10B43800D2105343642293FBF2F3134423EAE373D9
:10B44800DBB200E06423C1460193CB1C03930024C4
:10B45800039B022C13F8016F804F03934FEA440AB1
:10B4680005D1B7F904301B365E4376114AE07C4BB0
:10B4780037F9142033F9143003EB4202049B5B4282
:10B488009A4203DB049B9342A8BF1346754A32F9DC
:10B498000A50059A5B1B32F9145003EB050B07F0B1
:10B4A80019FB88B1704A5846155D07F011FE6F49BF
:10B4B80007F016FF0146284606F028FD6B4907F0FD
:10B4C8005BFE08F01FF88346624A1288D10714D43D
:10B4D80037F90A501B366E4393074FEA261611D5E3
:10B4E80098F812509DF9042005FB0BF3534364228E
:10B4F80093FBF2F306EB231604E098F8085005FBDB
:10B508000BF52E115A4B042533F90A30594F93FB8A
:10B51800F5F5751B99F8016007F10C036E43E35CC0
:10B5280098F851B05E430293642396FBF3F6F61144
:10B53800BBF1000F1CD0022C30460CD107F0C8FD1F
:10B548005FEA5B0304D05B45A8BF5B461A4600E090
:10B558000122494906E007F0BBFD5A4607F11001F0
:10B5680001EBC401BB6AFCF785FE07F0CBFF06467A
:10B57800424B99F80B7019883E4B01FB05F203F119
:10B588002C0E5EF82400D21207FB02073C4AB7F5DE
:10B59800001FA8BF4FF40017974203F13800B8BF47
:10B5A800174650F8242040F824504FF6FF70090938
:10B5B800B0FBF1F1AA1A4A4303F1440103F1500523
:10B5C8004EF8247051F824E055F8240045F824E09A
:10B5D80098F85050921170444FEA840C7F1310442D
:10B5E80041F824208DB1CDF818C0079307F070FDFD
:10B5F800079B2A4603F15C0101EBC4019B6AFCF737
:10B6080039FE07F07FFFDDF818C099F81530F219F8
:10B618005843029B013443431846642390FBF3F0DC
:10B62800184B0012024423F80A2003F108024CF8D0
:10B638000260032C03F1140203F120034CF802709A
:10B648004CF8030009F101097FF402AF09B0BDE825
:10B65800F08F00BFD01100203C250020EC10002006
:10B66800B2300020F8240020F49C0108000020419A
:10B6780028100020AC140020CC1400200410002056
:10B688000000E0FF20150020B0F902302DE9F74F47
:10B6980093421CBF0023037090F800A004460E4696
:10B6A8009146BAF1000F40F0AB80104607F010FD4C
:10B6B800864907F061FD864907F05EFD4FF07C5131
:10B6C80007F05AFD0BF008FB0146054607F054FD4C
:10B6D80080498346284607F04FFD034658461946D9
:10B6E800019307F041FC4FF07E5107F03DFC014605
:10B6F8004FF07E5007F0F4FD2946804607F03CFDE8
:10B70800294607F039FD07460146606007F02CFC22
:10B71800E7604FF07E572946A0602761284607F06A
:10B7280023FC294607F028FD4FF0804107F01AFC5A
:10B738000146404607F020FD019B606119465846C6
:10B7480007F010FC394607F00FFC0146404607F0A9
:10B7580013FD40F2DC53A046274655466365102387
:10B76800A4F852301823A061A4F850304FF0974144
:10B77800D8F8100007F000FD0021824607F09AFE75
:10B7880028B150464FF07C5107F0ECFB04E05046DE
:10B798004FF07C5107F0E8FB07F016FFC7E90E01F0
:10B7A8004FF09741D8F8040007F0E6FC00218246E4
:10B7B80007F080FE28B150464FF07C5107F0D2FBCD
:10B7C80004E050464FF07C5107F0CEFB07F0FCFE3A
:10B7D8000135032DC7E9080108F1040807F1080736
:10B7E800C4D1A6F2DC531B042367E3676367C4F87C
:10B7F8008030A367C4F884300123A4F80290237032
:10B80800D4F85490B4F95280C9EB0606636A06FA74
:10B8180008F67343276A4FEAE67B206F07FB0B3372
:10B828002667A7FB0667E26F1F44636CD4F840C025
:10B8380053434FEAE27B0CFB0B3ED4F88010C4F86C
:10B848008020ACFB02237344B61A67EB0307E36A54
:10B85800A26A43434FEAE07B02FB0B3EA2FB0023B4
:10B868007344B6185F41E36C656F4B436067A06C27
:10B878004FEAE17B00FB0B33C4F88410A0FB010105
:10B888001944636B361A05FB03F3206B4FEAE57B1B
:10B8980000FB0B3367EB0107A0FB05018019194476
:10B8A8007941B4F95020A56707F04AFB08F1FF3247
:10B8B80001239340E067C01841EBE371424607F06B
:10B8C8003FFB484403B0BDE8F08F00BF6F12833AD6
:10B8D800DB0F4940F404B53F2DE9F8430024254B1C
:10B8E800E0B293F8D060B0420DD203EB8003224A55
:10B8F800D3F8A03032F810101BB10B2801D8DB6840
:10B9080098470134EBE71D4B1B685B032FD50024D8
:10B918002346E2B2B2422AD2DFF858904FEA8408AE
:10B9280009F1A00757F8242055689D4217D02846EA
:10B93800FFF732FCEFF31283502282F3128828219A
:10B94800AA8C01FB009092B20132C0F8F820AA8AB2
:10B95800DBB292B242F00102AA8283F3118857F84F
:10B96800083000221B6801341A802B46D1E7BDE855
:10B97800F88300BFAC1400204810002000250020E8
:10B9880008B50E4B1B6813F4805F0D4B14BFD3F83A
:10B998007421D3F8782193F8D01092880023D8B274
:10B9A800884204D2074820F813200133F7E7FFF74D
:10B9B80093FFBDE808403220FEF7CDBD00250020EA
:10B9C800AC140020481000200A4B30B51A680A4B06
:10B9D80002F48052D3F87441D3F8785100230AB1A5
:10B9E800A18800E0A988054820F8131001330C2B22
:10B9F800F5D130BD00250020AC140020AE24002075
:10BA080070B5124D0024214605F27D10702285F88C
:10BA18007C410AF0F4FE2146D5F8F0310B4A0B447C
:10BA280093F9020088B11E6802F27D140E510819BC
:10BA38009C88073184809B797029837192F87C31C6
:10BA480003F1010382F87C31E6D170BDAC1400200B
:10BA5800094B1A680E2303FB0020437AFF2B07D0FB
:10BA6800064A12789A4203D9054A32F8130000E0D0
:10BA7800808800B2704700BF20120020D422002026
:10BA88003C2500202DE9F04F974C91B0D4F8F831BF
:10BA98000546964898479548954F014694F80822D8
:10BAA80004F012FD3B880197002B79D0D4F80C32B2
:10BAB80004F504781B7804F5077702934FF0000922
:10BAC800019B4FEA490A1E88B6F57A7F02BF002219
:10BAD800C8F800203A61854A32F91900D8F80020E0
:10BAE8000244C8F8002007F0F3FA3A690132012A43
:10BAF8003A6104D1002278603860BA6028E03B6877
:10BB0800059219460393049007F02CFA059A834688
:10BB1800104607F0DDFA0146584607F0E1FB039BA3
:10BB28000146184607F020FA0246DDF810C0114613
:10BB380078606046039207F015FA0146584607F008
:10BB48001BFBB96807F010FA039AF8603A60B8600E
:10BB58006649DFF8B8B10022012E2AF801202AF838
:10BB68000B2029D13869012807DD013807F0B0FA20
:10BB78000146F86807F0B4FB00E000200BF0B0FACB
:10BB8800029B7BB10390184607F0A2FA039A01467C
:10BB9800104607F0ADFC28B1019A4FF47A73138070
:10BBA80000231CE0D8F800204FF47A7102F5FA72ED
:10BBB80092FBF1F22BF80A2009F10109B9F1030F00
:10BBC80008F1040807F114077FF47AAF012E02D1B7
:10BBD8003046FEF75FFC019B013E1E80E0E7424EC7
:10BBE800424906F5167031F8132030F81300121A7E
:10BBF80021F813200133032BF1D13E4B1B6813F0BE
:10BC0800020300F00B833C4B06F25E205B6898470A
:10BC18003A4B06F25E201A78014604F055FCB6F855
:10BC2800643206F25E27002B42D0D6F86802002361
:10BC3800B4F864224FEA830CB2F5C87F304A04BFD7
:10BC4800002142F8231037F913E052F80C10264E61
:10BC5800714442F80C10002127F8131020F8131033
:10BC68000133032BE4D1B6F86432012B1BD1D6F88B
:10BC78006C324FF4C87E03F1C80292FBFEF20280D8
:10BC8800D6F87022C83292FBFEF24280D6F874329F
:10BC98001C4AC83393FBFEF312889B1A83802980C1
:10BCA8006980FDF765F9B4F86432013BA4F86432A1
:10BCB800154B1B685A0740F18D80B4F878220A4B5F
:10BCC800322A25D1D3F868221188A3F87A1251882C
:10BCD8009288A3F87C12A3F87E222A88A3F88022EF
:10BCE8006A88A3F8822215E0AC14002028100020EE
:10BCF800B630002008110020CC240020BC300020E1
:10BD0800181700200E00002000250020041700202E
:10BD1800002A3FD0D4F868820023B4F878224FEA8A
:10BD2800830E322AC24A04BF002142F8231037F991
:10BD3800130052F80E10BF4E014442F80E100022B4
:10BD480027F8132028F813200133032B1146E4D1D8
:10BD5800B6F87832012B18D10C2086F8913286F883
:10BD68009022FEF797FBB6F87A32A8F80030B6F8BA
:10BD78007C32A8F80230B6F87E32A8F80430B6F85B
:10BD880080322B80B6F882326B80B4F87832013B6F
:10BD9800A4F8783294F89232A64ADBB1D2F8843209
:10BDA800322693FBF6F3D2F86802002182F8921249
:10BDB8000380D2F8883293FBF6F34380D2F88C32B2
:10BDC8009D4A93FBF6F312889B1A83802980698029
:10BDD800FDF7CEF8D4F86822B4F85E3211884FF037
:10BDE80000085B1AA4F85E325188B4F860325B1A16
:10BDF800A4F860329288B4F862329B1AA4F86232CE
:10BE0800FEF782FBD4F894620546831B184601931B
:10BE180007F05AF9D4F89812029007F0ADF9C4F86F
:10BE280094524546D4F89C72844E97F800B003901B
:10BE3800834A0DF11C0A32F9150007F049F90399F4
:10BE480007F09AF94AF82500BBF1000F2BD05846A5
:10BE580007F03EF901464FF07E5007F041FA0246DE
:10BE6800DFF8049211464FF07E50059207F07AF8F9
:10BE780059F8251007F080F9A9F14201049031F929
:10BE8800150007F025F9059A114607F075F9DDF850
:10BE980010C00146604607F067F849F8250007F02A
:10BEA80031FB708003E0674A32F81520728036F95A
:10BEB800022F0135032D02FB0288B9D1642303FB4D
:10BEC80008F85D4B60481B8807A95B4398FBF3F8AB
:10BED800A8F149081FFA88F8FCF72CFDB8F13B0FC8
:10BEE8007D6810D9534BB3F9B802D3F8B45207F0B0
:10BEF800EFF80146284607F0FBFA544B68B31A7866
:10BF080042F008022CE04FF07E51284607F02CF84A
:10BF180001464FF07E5007F0E3F981464FF00008E4
:10BF2800DFF824B128465BF8281007F025F9484ABD
:10BF3800039032F9180007F0CBF8039B0146184626
:10BF480007F012F8494607F017F94BF8280008F1EE
:10BF58000108B8F1030FE3D1C4E71A7822F0080208
:10BF68002946D4F8B0021A700AF02EFF81462060E4
:10BF7800D4F8AC02D4F8B4B200F10045D4F8B00259
:10BF8800014607F0F9F859468046584607F0F4F894
:10BF98000146404606F0E8FF0BF0A2F801462846A5
:10BFA8000AF012FF2B4980466060484607F0E4F823
:10BFB8000AF032FE284D27492880404607F0DCF871
:10BFC8000AF02AFE254B68801B681B074ED52448BB
:10BFD80007A9FCF7AFFCBD684FF07E51284606F074
:10BFE800C3FF01464FF07E5007F07AF982464FF0C2
:10BFF800000B1B4B284653F82B10049307F0BCF892
:10C008001849039031F91B0007F062F8039A0146BA
:10C01800104606F0A9FF514607F0AEF8049B43F816
:10C028002B000BF1010BBBF1030FE2D1184654E0D2
:10C0380030170020AC1400200E000020D41000207F
:10C04800281000200A170020581700200C11002083
:10C05800D61000204C3D0F44F82400200811002081
:10C06800681700202E1000204C170020704D5146F4
:10C078002846FCF75FFC28686B680146039307F0C5
:10C088007BF8039B82461946184607F075F8014667
:10C09800504606F069FFD5F808B08246594658461A
:10C0A80007F06AF80146504606F05EFF0BF018F8F4
:10C0B8000021824607F0F4F970B92868514607F064
:10C0C8000FF951462860686807F00AF95146686018
:10C0D800A86807F005F9A8605548FFF707F9554B18
:10C0E80055491880029807F047F8524B08F1004864
:10C0F800054609F10049B3F90000CDF82C80CDF8C8
:10C10800289006F0E5FF4D4900F1004007F034F8AB
:10C11800DFF83C810C90B8F9000006F0D9FF0D90CB
:10C12800B8F9020006F0D4FF0E90B8F9040006F042
:10C13800CFFF0AA90F900DA8FCF7FCFB7B78012B19
:10C148001AD13F4B3F4F1B7813F0040F0ED1D7F88D
:10C15800C802402390FBF3F3C01A06F0B9FF0F9909
:10C1680006F002FF07F0CEF9C7F8C802D7F8C802F0
:10C17800402390FBF3F001E0334B188806F0A8FF4A
:10C1880001460F9806F0EEFED4F8D0120F9028461C
:10C1980006F0EAFE0146284607F0A2F8D4F8CC7269
:10C1A800054639460F9806F0DDFE0146284606F09A
:10C1B800E3FF0146384606F0D7FE0746C4F8CC022E
:10C1C8000D980AF029FDD4F8D4522978FCF7B2FA70
:10C1D800D4F8D8321844C4F8D8020E980AF01CFDD6
:10C1E8002978FCF7A7FAD4F8DC321844C4F8DC0242
:10C1F80038460AF011FD6978FCF79CFAD4F8E03269
:10C20800124A184401991368C4F8E0021944D4F892
:10C21800E43211600133C4F8E43205E0A6F85E3276
:10C22800A6F86032A6F8623211B0BDE8F08F00BF00
:10C2380014000020E4100020BD37863535FA8E3C06
:10C24800BA300020AC1400200E000020A0300020DE
:10C25800D610002001380A4B042804D8DFE800F083
:10C268000507090B0D00074A08E0074A06E0074AD8
:10C2780004E0074A02E0074A00E0074A1A607047EC
:10C2880048000020DDE30008C9B30008012B0108BD
:10C29800A3E0000811DD000865D7000808B50848C4
:10C2A8000AF0F1FAC0B209280246054B04DC013055
:10C2B8002021C0B29954F6E700221A5408BD00BFE5
:10C2C800C121002008B507480AF0DDFAC0B21428D9
:10C2D800044B04D8421C20211954D0B2F7E700229D
:10C2E8001A5408BDC12100202DE9F74FFEF70CF9BB
:10C2F800A64C804626686568A768861BF643451BDA
:10C30800C71BED43FF43F60FED0FFF0F2EB93FB9E3
:10C31800002D00F08782B9462CE04FF0000929E093
:10C32800B14627E003EB8A0BBBF802301A050ED49E
:10C3380013F4805F1DBF964A9BF801101268954A56
:10C34800954B14BF52F82120126843F82A20BBF8F5
:10C358000230D80516D499050AD5904B1B7813F0EE
:10C36800040F0CBF8E4A8F4A8B4B126843F82A2061
:10C3780009F10109207B5FFA89FA8B4982450B682C
:10C38800D0D326E0894A5046594604F0B1F9884B83
:10C398001B885A0603D550465946864A16E0580760
:10C3A80003D550465946844A10E0190703D550462C
:10C3B8005946824A0AE09A0703D550465946804AA8
:10C3C80004E0DB07D4D5504659467E4A04F090F97C
:10C3D800CEE7DFF808E20093BEF906307822A3F52D
:10C3E8007A7353434FF47A7293FBF2F3F34603F2F2
:10C3F8002B13019300225FFA82FE864517D2009B19
:10C4080003EB820EBEF802E01EF4806F0DD040F2FE
:10C41800671ADFF88491019B39F822E09E449EFB5D
:10C42800FAFC0AFB1CEE29F822E00132E3E74DB3DF
:10C4380008F5C333A0336360637B544A13BB93731B
:10C44800614B1B6813F0020F0AD0DFF894E19EF8E5
:10C4580000E0BEF1000F03D04FF0010E82F80EE0AD
:10C46800DA0506D5594B5B791BB1A37B43F0020370
:10C47800A3734A4B1B7813F0050F02BFA37B43F04D
:10C488000403A37394F80EE0BEF1000F03D13F4BF1
:10C498005B7B002B4FD094F80DC01CF0010FACF162
:10C4A8000C031DD1BCF1030F07D8DFF8E8901EF08C
:10C4B800040F3B4A08BF4A4600E0364AACF1040C78
:10C4C800BCF1070F05D8DFF81CC11EF0010F18BF1B
:10C4D8006246DBB2032B0ED81EF0020F3C4B06E07F
:10C4E800DBB2032B06D82F4B2A4A1EF0020F18BFC7
:10C4F8001A4600E0274A4FF0000C5FFA8CF383429B
:10C508000DD20B6803EB8C035B881B0642BFD2F885
:10C518000090214B43F82C900CF1010CEDE785B10C
:10C52800BEF1000F08D0637B184A0133DBB2142B2D
:10C5380006D1002304E025B1637B002BF3D100E092
:10C548005373002E52D0234A3223B2F90250B2F963
:10C558000020002DB8BF6D42002AB8BF524295FB9B
:10C56800F3F592FBF3F2EDB2D3B2AB4238BF2B46F0
:10C57800194A13B192FBF3F300E0134643442360D6
:10C58800E37B024A83BB01232FE000BF94170020FE
:10C598001812002020B10108920D0020BA300020A6
:10C5A80028B0010818B001081C120020F69C0108E8
:10C5B800D0110020FC9C0108029D0108089D01087B
:10C5C8000E9D0108149D0108002500201C0E002066
:10C5D80030B00108EC100020400D03003C2500207D
:10C5E8005811002038B001080023D3738F4D904BA9
:10C5F8002D78E27BADB9002F00F00F818D4B267BA3
:10C608001A788D4B02F0040293F800C08B4BD2B21B
:10C61800D3F800E00B680021894D03EB86060F462E
:10C62800B5E01AB9874A1A61002508E0864AFAE790
:10C638000A68AB00D6187688760604D40135EBB2C2
:10C648008342F5D3D7E7814EB6F90060192E25DD70
:10C6580012F803E094F814C00EF00F09E1452669BA
:10C668000CDCDFF8CCC19CF815C0BCEB1E1FDEBF8C
:10C67800D6F800C0DFF8D8E143F80EC012F803E09E
:10C6880094F816C00EF00F09E14533DBDFF8A0C1BE
:10C698009CF815C0BCEB1E1F2CDC26E0193629DAE5
:10C6A80012F803E094F814C00EF00F09E14526696A
:10C6B8000CDCDFF87CC19CF817C0BCEB1E1FA2BFC6
:10C6C800D6F800C0DFF888E143F80EC012F803E09E
:10C6D80094F816C00EF00F09E1450BDBDFF850C1E6
:10C6E8009CF817C0BCEB1E1F04DBD6F800E0584EC0
:10C6F80043F806E0554EB6F90260192E1BDD12F814
:10C7080003C094F814E00CF00F09F14526690CDC1D
:10C71800DFF81C9199F81590B9EB1C1FDEBFD6F80D
:10C728000090DFF82CC143F80C90D25C02F00F0C9B
:10C73800F4451EDD82E7193680DA12F803C094F852
:10C7480016E00CF00F09F14526690CDBDFF8E090E4
:10C7580099F81590B9EB1C1FDEBFD6F80090DFF8EA
:10C76800F0C043F80C90D25C02F00F0CF445FFF6D1
:10C7780065AF94F817E0BEEB121FA2BF3668344AC3
:10C788009E505BE75888000504D404330435B3424F
:10C79800F8D122E04AB101EB0C0A06209AFBF0F925
:10C7A80000FB19A001280DDC01E057B9012793F817
:10C7B80001900EEB89003EF829A090F80290C0780D
:10C7C80003E01746002081468246013125F802AC75
:10C7D80085F800906870C9B2D7E7174A1378013B0B
:10C7E80013F0FF0308BF06231370124B1B785B0777
:10C7F80041BFBBF906304FF47A72A3F57A7303EBA5
:10C80800C30348BF93FBF2F3124A46BF0133DBB2BE
:10C81800012392FBF3F34344A36003B0BDE8F04F58
:10C8280002F0B2B803B0BDE8F08F00BF4B0E002095
:10C8380094170020BA300020200000201812002091
:10C84800940D002034B0010820B10108EC1000203C
:10C85800920D0020400D030037B50622044603213F
:10C868006B461E20F8F72CFD9DF801309DF800005E
:10C87800154D43EA002000B206F02AFC296806F0AC
:10C888007BFC06F03FFE9DF8033020809DF80200F7
:10C8980043EA002000B206F01BFCA96806F06CFC15
:10C8A80006F030FE9DF80530A0809DF8040043EAAC
:10C8B800002000B206F00CFC696806F05DFC06F08A
:10C8C80021FE608003B030BD240000201FB504465F
:10C8D80002210C2001220DF10703F8F7F1FCC8B37F
:10C8E8009DF80730DB0735D50321062202AB0C2063
:10C8F800F8F7E6FC0C20092101220DF10703F8F7EF
:10C90800DFFC38B39DF8073013F00C0F22D19DF8E7
:10C9180009209DF808300C2043EA0223C3EB833337
:10C928009B009DF80B2023809DF80A300A2143EADA
:10C938000223C3EB83339B009DF80D2063809DF891
:10C948000C3043EA0223C3EB83339B00A38001220C
:10C95800F8F7AEFE04B010BD07B50A2100220C207E
:10C96800F8F7A6FE1420FDF7F6FD0A210F220C2089
:10C97800F8F79EFE0A20FDF7EEFD01AB1021032219
:10C988000C20F8F79DFC0A20FDF7E5FD0A2100229E
:10C998000C20F8F78DFE0A20FDF7DDFD0DF10303ED
:10C9A800022101220C20F8F78BFC0DF10303092169
:10C9B80001220C20F8F784FC0A2101220C20F8F748
:10C9C80077FE03B05DF804FB2DE9FF41604B1B685F
:10C9D8009BB11A681AB15F49886902438A619A88CB
:10C9E8009868ADF8042002228DF8072004220DEB88
:10C9F80002018DF8062002F0A5F83220FDF7ABFD04
:10CA0800002111221E20F8F753FE012160221E206A
:10CA1800F8F74EFE6420FDF79EFD002402A8FFF7FC
:10CA28001BFF274626460A25022101221E20F8F769
:10CA38003FFE3220FDF78FFD02A8FFF70DFFBDF97D
:10CA48000820BDF90A1014448A42A8BF0A46BDF955
:10CA58000C300F4493421E44A8BF134613F5805F61
:10CA680009DD3D4A013DD36883F01003D360DBD173
:10CA78004FF0010801E04FF000081E2000211222AB
:10CA8800F8F716FE0A25022101221E20F8F710FEEB
:10CA98003220FDF760FD02A8FFF7DEFEBDF9082091
:10CAA800BDF90A10A41A8A42A8BF0A46BDF90C307B
:10CAB8007F1A9342A6EB0306A8BF134613F5805FBF
:10CAC80007DD254A013DD36883F01003D360DAD12E
:10CAD80001E04FF00008204606F0FAFA01461F4828
:10CAE80006F0FEFB1E4D20F000402860384606F098
:10CAF800EFFA0146194806F0F3FB20F000406860A1
:10CB0800304606F0E5FA0146164806F0E9FB20F043
:10CB18000040A860002170221E20F8F7C9FD0121FD
:10CB280020221E20F8F7C4FD1E2002210022F8F75B
:10CB3800BFFD6420FDF70FFDB8F1000F04D14FF0E1
:10CB48007E532B606B60AB6004B0BDE8F08100BF22
:10CB5800A402002000100240000C014000406F4673
:10CB68002400002001C05E46024640213C20F8F720
:10CB78009FBD024680213C20F8F79ABD012828BFB6
:10CB880001202DE9F04F0646142000FB06F3704FF4
:10CB980089B0F918FC586F4B0A691C601E716E4BFE
:10CBA800B1F80880DD69B1F80AA02A43DA61A288E1
:10CBB8004D6822F440721204120C4AEA0809A28055
:10CBC80003A9C5F8109002228DF80E00284601939B
:10CBD800ADF80C908DF80F2001F0B4FF019B009781
:10CBE8001F464FF0080BAA6818EA020F03D10A2063
:10CBF800FDF7A6FCF7E70A20C5F81480FDF7A0FCAE
:10CC0800C5F810800A20FDF79BFCBBF1010BEAD1A7
:10CC1800C5F814A00A20FDF793FCC5F814800A2073
:10CC2800FDF78EFCC5F810800A20FDF789FC02226A
:10CC3800C5F810A0284603A98DF80F201C228DF8EE
:10CC48000E20ADF80C9001F07DFF444A03A89442F1
:10CC58003A690BBF42F4001242F480023A613A6129
:10CC68000BBF3A693A6922F4001222F480023A6151
:10CC7800A38823F440731B041B0CA38023889BB256
:10CC880043F001032380A58803F036FA0599344B55
:10CC980025F03F05B1FBF3F32D042D0C1D43ADB278
:10CCA800A5802288002522F001021204120C22809D
:10CCB8002C4A03A8B1FBF2F100298AB208BF01226D
:10CCC80042F400414FF4967253434FF47A7293FB47
:10CCD800F2F301339BB22384A1832388009A9BB289
:10CCE80043F001032380238823F4816323F00203A4
:10CCF8001B041B0C23804FF480432381142303FB64
:10CD08000626737B01248DF80C308DF80D508DF8B4
:10CD18000E508DF80F4005F085F8337B9DF80F20F5
:10CD28008DF80C308DF80D508DF80E501AB103A8FF
:10CD380005F078F808E05A0903F01F039C4002F157
:10CD48002003094A42F8234009B0BDE8F08F00BF2C
:10CD58001C9D0108AC170020001002400054004040
:10CD680040420F00804F120000E100E0914B70B587
:10CD78001A68908A80B2C1B2CE072ED5118821F4E4
:10CD880000610904090C1180118889B241F480619D
:10CD9800118000215971997999B1D97911B9197A04
:10CDA800FF290ED10121D971597A022901BF1188B1
:10CDB80089B241F400611180997A41F00101118230
:10CDC800E2E0997A01F0FE0111821A7AFF2A00F056
:10CDD800DB80784AFF215171D6E08D073AD5BFF341
:10CDE8005F8F587AC0B2012813D1997989B1D9795E
:10CDF80079B1118821F480610904090C1180BFF30D
:10CE08005F8F118B1188D87289B241F4007111803B
:10CE18001BE0118BBFF35F8F587A664902280AD14D
:10CE2800887940B1C97931B1118821F48061090448
:10CE3800090C1180A2E0587A5E49032805D1887947
:10CE480018B1C979002940F09980918889B241F4D4
:10CE5800806198E04C0757D50121D972997900294A
:10CE680038D0D979002935D0597A108802295979CA
:10CE78001ED920F480600004000C1080148ADD683C
:10CE8800C8B2E4B249B26C541188DC6889B241F482
:10CE9800007111801968821C5A710A8A0130D2B255
:10CEA80040B222548A8892B242F480628A8026E094
:10CEB80080B240F400701080148ADD68C8B2E4B211
:10CEC80049B26C54128A411C49B2D2B203306A5436
:10CED800587114E0D979374809B9017C41B11188F2
:10CEE80089B241F4007111805A7901325A7106E011
:10CEF800118889B241F4807111800122C2711968C8
:10CF08000A88D205FCD43FE001F0400101F0FF049B
:10CF1800E1B15879168ADD68C4B2611C40B2F6B234
:10CF28002E54C9B25D7A597149B2C81C854201BFF5
:10CF3800908820F480600004000C08BF90805A7A22
:10CF48008A4221D11B4A023454711DE006061BD5C2
:10CF5800597948B2451C0AD05C690131205CC9B2D4
:10CF68001082587A597149B288420DD106E0197A6F
:10CF78005C711182997909B9597A29B9918821F492
:10CF880080610904090C9180597A93F905000131EF
:10CF98008842084A0CD10021D171D17A31B1116887
:10CFA8008A8822F440721204120C8A8000221A76AF
:10CFB80070BD00BFAC17002010B5204C2368998ABB
:10CFC80089B211F4706F1CBF0122627611F4E06F10
:10CFD8002AD01A8B9A88890522F480624FEA024285
:10CFE8004FEA12429A801FD41A8892051CD41A88D4
:10CFF800D0050ED51A88D105FCD41A8892B242F40D
:10D0080000721A801A889205FCD42079FFF7B6FDC1
:10D018000AE01A8892B242F400721A809A8822F4BE
:10D0280040721204120C9A802268938A23F4706367
:10D038001B041B0C93820023237610BDAC17002021
:10D04800026B0346C16810B5406942B11A6C8C1A6C
:10D05800013A08BF0A46005D1A64C0B210BD1A6AD8
:10D06800805C01328A4228BF0022C0B21A6210BD19
:10D07800436B13B190F844007047836A406A1B1AE7
:10D08800584258417047036B13B15B68016C01E06B
:10D09800C369016A8B423CBFC2689B18581AC0B268
:10D0A8007047426A806A131A584258417047417162
:10D0B800704743799B070AD5436A8269D154436A0A
:10D0C80001690133B3FBF1F201FB1233436270478C
:10D0D800437913F001031FBFC36803F1FF32C3692B
:10D0E800006A1DBF181A1040C0B21846704743792D
:10D0F80010B513F0010304460DD0FFF7E9FF58B14E
:10D10800236A6269E168D05C0133B3FBF1F201FB89
:10D118001233236210BD184610BDF0B5046D827934
:10D12800A389467923F4005312F0020F4FEA034310
:10D138004FEA13430CBF00214FF4005112F0040FC3
:10D14800A38114BF4FF4806E4FF0000E16F0010F4C
:10D158008768054614BF04200020B307238A48BF08
:10D1680040F008029BB223F4405343EA01032382B0
:10D17800A18948BF90B289B221F4B05121F00C01C5
:10D188004EEA010140EA0102A281A38A87B023F492
:10D1980040731B041B0CA38201A802F0ADFF039B84
:10D1A800049E264A944218BF1E46A3891922724338
:10D1B8001BB2002BB4BF7E00BE00B2FBF6F664279C
:10D1C800B6FBF7F00001010907FB1163A28912B24F
:10D1D800002AB7BFD9001A013231B1FBF7F2A7BF55
:10D1E8003232B2FBF7F302F007021043A8BF03F094
:10D1F8000F03AA79A8BF184380B212F0010F20814B
:10D208002B6D06D00E498B4202BF042001F5484120
:10D21800086112F0080F9A8A0BBF22F0080292B236
:10D22800120442F0080208BF120C9A829A8992B23C
:10D2380042F400529A8107B0F0BD00BF00380140A7
:10D2480000440040417168E7816066E703460A468A
:10D2580090F84602D96A9B7901F0A6BC38B5A0F5CA
:10D2680013746379A579DB0746D594F8383205F04D
:10D278000105F3B1226B1068838DC3F34E038384D9
:10D2880094F83C3223B1B4F842320133A4F8423264
:10D29800917A6A0001F0E7FA012384F83B3200230F
:10D2A80084F8393284F83A3284F83832A4F84032B3
:10D2B80038BD94F83B322046012B04BF94F839322C
:10D2C80084F83A3201F0BAFA94F83B22236B3AB95F
:10D2D800012284F83B221868997A05FA02F207E0DD
:10D2E800002284F83B2295421868997A08BF0222E6
:10D2F800BDE8384001F0B7BA38BD10B5A0F51274D2
:10D3080094F83C22BAB9A36A616A994228D0591C98
:10D31800A069A162C35C2069DBB25B0043F40073BF
:10D328008142A4F83E324FF00A0384F83D3228BF08
:10D33800A262012312E094F93D327BB1B4F83E12A7
:10D3480020464B08A4F83E3201F0010101F09EFA94
:10D3580094F83D32013B84F83D3201E084F83C32D8
:10D3680094F83832002B50D194F839320133DBB2BB
:10D37800092B84F8393204D12046BDE8104001F069
:10D388005DBA0A2B41D194F83B322BB9B4F840323C
:10D3980043F00103A4F840326379D9071CD5B4F8E7
:10D3A8004002820501D4C30705D4B4F844320133DE
:10D3B800A4F8443210E0E36AC0F347000BB1984781
:10D3C8000AE0E3696269D054E369E1680133B3FBB9
:10D3D800F1F201FB1233E361012284F8382294F858
:10D3E8003B220023012A84F839320ED1A27984F82D
:10D3F8003B32236B12F0010F1868997A0CBF022296
:10D408000022BDE8104001F02EBA10BD026D70B5C3
:10D4180015880446ADB2A90613D5036B8BB9C36A48
:10D428001BB1908880B298470BE0E1699288406907
:10D438004E1CD2B2E6614254E169E268914228BFCB
:10D44800E3612B0613D5636AA26A9A42236D0AD058
:10D45800511CA069A162825C9A802369994206D313
:10D468000023A36270BDDA6822F08002DA6070BD22
:10D47800836A8169426B1944D160416A994297BFB6
:10D488000169CB1ACB1A536096BF0023536083629D
:10D498004FF0000380F84430136888BF816243F07E
:10D4A800010313607047436A8269D154436A026971
:10D4B8000133934228BF00234362436B1BB11B68AF
:10D4C800DB0705D4D4E7026DD36843F08003D3604B
:10D4D80070472DE9F0431E46944B8DB0984289461B
:10D4E80090469DF8507051D1914B924A92491A60DA
:10D4F800924AC3F808805A6102F580729A614FF423
:10D508008072DA601A618E4A18651A63A2F5484279
:10D51800543ADA649A6459638A4B9A6942F48042AD
:10D528009A615A6942F001025A6102238DF8033068
:10D538003A074FF40073ADF8003001D51C230FE013
:10D54800B30706D51823804869468DF8023001F0E4
:10D55800F9FAF5070AD54FF48063ADF8003048238F
:10D56800794869468DF8023001F0ECFA0E238DF8FF
:10D5780004300022012301A88DF805308DF806201B
:10D588008DF807306A4C04F04DFC4EE06F4B984222
:10D5980040F0C7806E4B674AC3F808801A604FF4A2
:10D5A8008072DA601A616B4A18655A6102F58072F6
:10D5B8009A61694A3C079A64DA64624BDA6942F410
:10D5C8000032DA615A6942F001025A614FF00203EF
:10D5D8008DF803304FF00403ADF8003001D51C235B
:10D5E8000EE0B00706D51823574869468DF8023073
:10D5F80001F0A8FAF10709D50823ADF8003048234F
:10D60800514869468DF8023001F09CFA26238DF8BE
:10D6180004300022012301A88DF805308DF806207A
:10D628008DF8073004F0FEFB494C0025012384F8EF
:10D6380044302562E561A5626562C4F82C90667184
:10D64800C4F80880A7712046FFF767FDF20731D5B7
:10D65800206B002826D0E36C039501934FF4805388
:10D668000A9380230693E36805950493202309937E
:10D6780063690795029308950B9502F0C5FC01A90B
:10D68800206B02F0A3FC226B216D136843F00103A9
:10D6980013608B8A9BB243F040038B8253689BB222
:10D6A800236407E04FF6DF72236D1A80DA6842F0D0
:10D6B8002002DA60B3072CD5606B28B3A36C002571
:10D6C80001934FF480530A938023069323690295AC
:10D6D80004931023039305950795089509950B95D1
:10D6E80002F092FC606B01A902F070FC636B1A688F
:10D6F80042F002021A60226D5D605D60938A9BB2FF
:10D7080043F08003938204E0226DD36843F08003E2
:10D71800D360226D204693899BB243F400539381D2
:10D7280000E000200DB0BDE8F08300BF00380140E4
:10D7380058140020449D010844000240C8170020E6
:10D748005800024000100240000801400044004018
:10D7580004140020C8190020044400402DE9F04FAB
:10D76800054690F850008DB008910592099318B1BC
:10D778003228A8BF322000E0012005F0A9FC0146AC
:10D78800AA4805F0ADFDAA4B04461888002808BF32
:10D79800012005F09DFCA749069005F0EDFC0190DD
:10D7A8000199204605F0E0FB0146019805F098FD37
:10D7B800A14B07901B889A0724D5A049B1F90030DE
:10D7C800B1F9020083EAE37280EAE071A2EBE37246
:10D7D800A1EBE07191420C46B8BF1446B4F5E17F65
:10D7E80012DA914203DD0028D8BF404203E0002B43
:10D7F800CCBF1846584205F06BFC914905F070FD06
:10D80800064603E0002601E04FF07E564FF000097F
:10D8180003950024CDF8089063000493894B33F9ED
:10D82800140005F055FC884905F0A6FC05F06AFED1
:10D8380005F04EFC854905F09FFC804B824633F984
:10D84800140005F045FC7C4B07461B889B077ED0DF
:10D85800014605F089FB7E4B804633F9140005F03C
:10D8680037FC0146404605F07FFB05F04BFE059B63
:10D878005B42984203DB059B8342A8BF0346754A77
:10D888000499885E099A1B1A32F91400184405F0A5
:10D898001FFC804605F01EF970B16F4B40466F497A
:10D8A80014F8039005F01CFD0146484604F02EFBD1
:10D8B8006A4905F061FC8046287F05F005FC684947
:10D8C80005F05AFC8346287A05F0FEFB01464046DF
:10D8D80005F052FC634905F04FFC05F013FE814644
:10D8E8000BF1004005F00EFE814505DB584605F0BA
:10D8F80009FE4845A8BF484605F0EAFBDFF88891CD
:10D9080002900199404605F037FC59F8241005F0BB
:10D918002BFB55494FEA840B804605F0CBFD38B9FF
:10D928004046524905F0E4FD20B1DFF8408101E0AE
:10D93800DFF8348149F80B80A87C05F0C5FB014667
:10D94800404605F019FC4A4905F016FC81463A4B59
:10D95800B3F800B01BF0010F40F09880394B049ADF
:10D96800DFF81C81D35E002BB8BF5B42B3F5206F94
:10D978004FEA84030A9303DD002348F824302AE0A1
:10D988003C49384605F0F8FB039B0B90587805F0A6
:10D998009BFB0B9A0146104605F0A2FC514605F088
:10D9A800E1FA019905F0E8FB58F8241005F0DCFAD3
:10D9B8003149804605F07EFD38B940462F4905F0CB
:10D9C80097FD20B1DFF8B48001E0DFF8AC802C4A85
:10D9D8000A9B42F80380039BD87A05F075FB284B15
:10D9E80053F8241005F0C8FB264905F0C5FB1BF0C9
:10D9F800020F80464CD03846029905F0B3FA01462A
:10DA0800304605F0B9FB0146029805F0ADFA4946E3
:10DA18000746404605F0A6FA0146304605F0ACFB3D
:10DA28000146484605F0A0FA804631E083F9223ED7
:10DA380004100020BD378635D0110020EC100020DE
:10DA48000000E143281000200000A03ECDCC4C404F
:10DA5800B2300020F8240020F49C01080000204186
:10DA68000000A0406F12033C0000F0C10000F0412C
:10DA78000AD7A33D0000A043000040C30000404374
:10DA8800D01B00200AD7233CC81B0020C846029F91
:10DA98008B4B185D05F01CFB0146504605F06CFBEE
:10DAA800884905F069FB0146384605F05BFA95F8A8
:10DAB800512003463AB18449844B01EBC4011B68E9
:10DAC800FAF7D8FB0346824F504657F824100A93BA
:10DAD80005F048FA019905F003FC47F824A007F17E
:10DAE800080A5AF824B01037594605F03BFA01469F
:10DAF800079805F041FB0146584605F035FA83467C
:10DB08004AF82400385D05F0E3FA0146584605F066
:10DB180033FB704905F030FB07460A9B414618461F
:10DB280005F022FA394605F01DFA09F075F86A4A37
:10DB3800049B0492D0520A9BDFF8C0B1184605F046
:10DB4800E1FC4BF82400404605F0DCFCDFF8B0A10E
:10DB5800DFF8B0814AF8240007F1004005F0D2FC54
:10DB6800039B049A013348F82400039317460CB921
:10DB7800012451E6089A594B9479B3F904306400AA
:10DB880028345C43564B6411B3F9040005F0A0FA3D
:10DB98004FF07A5105F0F0FA09F03EF8201A05F036
:10DBA80097FA002CB8BF6442322C06464D4C02DD71
:10DBB8000023A36025E0069805F0A4FC20F00300EC
:10DBC80005F086FA0190687B05F07EFA014630463A
:10DBD80005F0D2FA019B81464349184605F080FBBF
:10DBE8000146484605F0C8FA05F08CFCA3681844BD
:10DBF8003E4B9842A8BF18463D4B9842ACBFA06028
:10DC0800A360A3686FF0FF005B13B3F5807FA8BF24
:10DC18004FF480739842B8BF184605F059FA044685
:10DC2800304605F06FFCEB785843801105F050FA48
:10DC3800304B06461B78032B12D9B5F84E90B9F530
:10DC4800FA7F0DD205F05EFCC9F10003984203DBB0
:10DC580048450346A8BF4B46184605F039FA06461C
:10DC680095F851206AB1530803D09A42A8BF1A46C2
:10DC780000E00122154B30461F491B68FAF7FAFAF3
:10DC880006462146304605F06FF905F03BFC80B2A8
:10DC9800B88000B205F01CFA08F0BEFFB880304624
:10DCA80005F030FCCBF80800204605F02BFC0023DB
:10DCB800CAF80800C8F808300DB0BDE8F08F00BFFA
:10DCC800DC1B0020A69B443BBC140020D41400207D
:10DCD800E01B0020F7CC923820150020EC10002023
:10DCE80028100020D814002000803B45FEFFFF0FBD
:10DCF800020000F07C150020CC140020281500201C
:10DD080034150020401500202DE9F04F89B0059307
:10DD1800BE4B0026B3F90290B3F90030B9F1000FF9
:10DD2800B8BFC9F10009002BB8BF5B429945B8BF1D
:10DD380099468046B2463446B9F5FA7F0491039273
:10DD4800A8BF4FF4FA79019000960296B04D2B883F
:10DD5800990754D0AD4B610033F91420AD4B33F91A
:10DD6800143003EB4202039B5B429A4203DB039BA2
:10DD78009342A8BF1346A84A8F5E059ADB1B32F967
:10DD880014001F1804F0A6FE90B1A44B384613F8EF
:10DD980004A005F09DF9A24905F0A2FA01465046F3
:10DDA80004F0B4F89E4905F0E7F905F0ABFB074627
:10DDB80098F8083064227B4393FBF2F398F81C2010
:10DDC8006FF0040A0AFB02FA534504DB02EB820AED
:10DDD8009A45A8BF9A4642F21072924B53F8240013
:10DDE80038449042A8BF10468F4A9042B8BF1046A8
:10DDF80043F8240098F812305843031302932D88EF
:10DE080005F00303012B38D0804B884933F91430CF
:10DE1800A6000093019B51F8247093F801E0844B0D
:10DE280033F9140080EAE073A3EBE073B3F5206FD5
:10DE380016DC009A50235A4392FBFEF3042290FB0F
:10DE4800F2F0181A0744B7F57A5F7A4BA8BF4FF477
:10DE58007A579F42ACBF41F8247041F8243002E061
:10DE6800002341F824308B597D2693FBF6F6019B5D
:10DE7800DB7A7343402693FBF6F6AA0712D5009A7D
:10DE880009FB06F509FB02F70298C9F5FA7303FBCB
:10DE98000A7703FB00534FF4FA7297FBF2F193FBF6
:10DEA800F2F505E0EB0755BF354651460099029D4E
:10DEB8005F4B042733F914305F4A93FBF7F3A25CF6
:10DEC8006FF04F07534393FBF7F398F851204FEA4D
:10DED800440BCF1872B13846069205F0F9F8574945
:10DEE800574B01EBC401069A1B68FAF7C3F905F012
:10DEF80009FB07464E4B534A3BF803003BF9021017
:10DF080003B25B1A042193FBF1F102F1040E5EF8EF
:10DF180024302BF802000C3252F8240042F8243046
:10DF280098F8502018444FEA840C08444EF82410FE
:10DF380082B1CDF81CC0069205F0CAF84249404BA0
:10DF480001EBC401069A1B68FAF794F905F0DAFAAE
:10DF5800DDF81CC03D4BDFF810E11B5D7A19584312
:10DF6800202390FBF3F3D21A2BF80E20384A5B4299
:10DF78004CF80230019B3748374901334CF80150BF
:10DF88004CF80070019375460CB90124DEE61F4B6E
:10DF98000427B3F90440049B244E9B79D6F808E083
:10DFA8000F335B006343224C5B11B4F90440002B30
:10DFB80094FBF7F7A3EB0707B8BF5B42322B98F83F
:10DFC8000D400BDC04FB07E4244BA342A8BF234607
:10DFD800234CA342ACBFB360B46001E00023B3603C
:10DFE80098F8034004FB07F31E4C9B112478032C7C
:10DFF8003DD9B8F84E40B4F5FA7F38D26742BB42F3
:10E0080034DBA342A8BF234631E000BFEC10002058
:10E01800D0110020B2300020F8240020F49C010820
:10E0280000002041F41B0020F0D8FFFFD814002086
:10E038002810002080C1FFFFDC1B0020BC1400203A
:10E04800D4140020FC1B002008150020F01B002021
:10E05800401500202815002034150020FEFFFF0F72
:10E06800020000F07C150020201500203B46B46813
:10E078006FF0FF0644F34F34B4F5807FA8BF4FF428
:10E088008074B442B8BF344683601E190023AE8042
:10E098008C60936009B0BDE8F08F2DE9F04F87B030
:10E0A8000393B44B81461D88029105F00205ADB279
:10E0B800019295B1B04BB3F90250B3F90030002D7D
:10E0C800B8BF6D42002BB8BF5B429D42B8BF1D462A
:10E0D800B5F5007FA8BF4FF40075CB460026A64BC8
:10E0E800A64933F91620A64B4FEA460A33F91630EB
:10E0F800520083EAE374A4EBE374B4F5206F4FEAAB
:10E10800860851F8260011DC042493FBF4F3D31A93
:10E118000344B3F57A5F9B48A8BF4FF47A53834210
:10E12800ACBF41F8263041F8260002E0002341F850
:10E13800263051F808709BF80B30FF119BF801400E
:10E148005F438C4B54431B88BF119B074FEAA414B1
:10E1580056D08D4B3AF903301A44019B5B429A42E0
:10E1680003DB019B9342A8BF1346884A3AF9022071
:10E178009B1A039A32F916201A44049204F0AAFC56
:10E18800049A98B1824B10469B5D049304F0A0FF5B
:10E19800804905F0A5F8049B0146184603F0B6FE31
:10E1A8007C4904F0E9FF05F0ADF9024642F210702F
:10E1B800794958F8013013448342A8BF0346774889
:10E1C8008342B8BF034648F8013099F8081099F817
:10E1D8001C004A4300EB8000D21141428A4203DB13
:10E1E8008242A8BF0246114699F81220641A534386
:10E1F8001B13FF1A6F436C4303EB672701EB64247F
:10E208005F4B04223AF9033093FBF2F2644B9B5DB7
:10E21800534399F85120A4EBA31472B120460492F9
:10E2280004F056FF5F49604B01EBC601049A1B6876
:10E23800FAF720F805F066F9044651495B4B3AF8BD
:10E2480001003AF903E002B2CEEB02024FF0040EED
:10E2580092FBFEF22AF803009E440C3358F80EC0D5
:10E2680058F8030048F80E206044104499F85020EC
:10E2780048F803C08C467AB10591049204F028FF4F
:10E288004B49494B01EBC601049A1B68F9F7F2FFA9
:10E2980005F038F9DDF814C0464BDFF834E19B5D32
:10E2A800E21943435B11D21A2AF80E204248434927
:10E2B800434A5B4248F8004048F8017048F8023089
:10E2C8000BF1010B74460EB9012608E72A4B042707
:10E2D800B3F90450029B294E9B79D6F808E00F3316
:10E2E8005B006B43BCF904505B1195FBF7F7002BFF
:10E2F800A3EB0707B8BF5B42322B99F80D500BDC34
:10E3080005FB07E52F4BAB42A8BF2B462E4DAB4272
:10E31800ACBFB360B56001E00023B36099F8035067
:10E3280005FB07F3294D9B112D78032D0CD9B9F85E
:10E338004E50B5F5FA7F07D26F42BB4203DBAB42C2
:10E34800A8BF2B4600E03B46B5686FF0FF0645F3D3
:10E358004F35B5F5807FA8BF4FF48075B542B8BF7B
:10E36800354683605E190023A6808D60936007B0F0
:10E37800BDE8F08FD0110020EC100020D814002048
:10E388002810002080C1FFFFB2300020F8240020B0
:10E39800F49C010800002041F41B0020F0D8FFFF86
:10E3A800DC1B0020BC140020D4140020101C00200A
:10E3B80008150020F01B0020281500203415002027
:10E3C80040150020FEFFFF0F020000F07C15002022
:10E3D800201500202DE9F04F89B00593AE4B00279A
:10E3E800B3F90280B3F90030B8F1000FB8BFC8F133
:10E3F8000008002BB8BF5B429845B8BF98468246D4
:10E40800B946BB463C46B8F5FA7F0492A8BF4FF41C
:10E41800FA7802900397A14D2B88990757D0022CC0
:10E4280055D09D4B610033F914209D4B33F91430BE
:10E4380003EB4202049B5B429A4203DB049B934238
:10E44800A8BF1346974A8E5E059A9B1B32F91400A3
:10E458001E1804F03FFB90B1934B304613F804B0FC
:10E4680004F036FE914904F03BFF0146584603F09C
:10E478004DFD8E4904F080FE05F044F806469AF8F2
:10E4880008306422734393FBF2F39AF81C206FF070
:10E49800040101FB02FB5B4505DB02EB82029342B0
:10E4A800A8BF13469B4642F21072814B53F82400D2
:10E4B80030449042A8BF10467E4A9042B8BF1046EA
:10E4C80043F824009AF81230584303130393298819
:10E4D80001F00303012B01D1022C3DD16E4B764D87
:10E4E80033F91490029BA00093F801E0734B55F8A0
:10E4F800247033F9146086EAE673A3EBE673B3F588
:10E50800206F1CDC022C14D0502303FB09F292FB71
:10E51800FEF3042296FBF2F69E1B3744B7F57A5FAA
:10E52800674BA8BF4FF47A579F42ACBF2F502B5070
:10E5380007E089EAE973A3EBE973642BE4DD0023C0
:10E548002B505D4B7D27C35893FBF7F7029BDB7A73
:10E558007B43402793FBF7F78A0713D5022C11D08A
:10E5680008FB07F508FB09F60398C8F5FA7303FBDF
:10E578000B6603FB00534FF4FA7296FBF2F193FB20
:10E58800F2F508E0CB0704D5022C02D0039D5946CA
:10E5980001E03D46494663000193484B042633F9A0
:10E5A8001430484A93FBF6F3A25C6FF04F065343CE
:10E5B80093FBF6F39AF85120CE18E2B1022C06929A
:10E5C80030460BD104F084FD069A530803D09A42D2
:10E5D800A8BF1A4600E001223B4905E004F078FD97
:10E5E8003A49069A01EBC401394B1B68F9F742FE18
:10E5F80004F088FF0646314B019A0198D15A354BF1
:10E608000AB2C05E4FEA840C121A042092FBF0F2A0
:10E618000198C15203F10801143351F824E053F86A
:10E62800240041F82420704410449AF8502043F8FC
:10E6380024E082B1CDF81CC0069204F049FD2649B9
:10E64800234B01EBC401069A1B68F9F713FE04F08B
:10E6580059FFDDF81CC0214B214A1B5D0199584325
:10E66800202390FBF3F073191B1A8B521D4B404269
:10E678004CF803601C4B01344CF803501B4B032C23
:10E688004CF80300029B03F1010302937FF4C3AE2D
:10E6980009B0BDE8F08F00BFEC100020D0110020B9
:10E6A800B2300020F8240020F49C0108000020412A
:10E6B800F41B0020F0D8FFFFD814002028100020F9
:10E6C80080C1FFFFDC1B0020CC140020BC140020FC
:10E6D800D4140020241C002008150020F01B002062
:10E6E8002015002028150020341500204015002092
:10E6F80010F80A3C0133DBB20A2B84BF10F8131C54
:10E70800044A00F80A3C82BF002322F8113000F8BE
:10E718000A3C7047BC2F0020334A70B5136C9068D0
:10E72800194440F68C23081A98429160D0605160D1
:10E7380013463BD9127893F9451010468A420BD1FB
:10E74800111F082908D893F84610182901D8013153
:10E7580003E083F8442002E0002183F8461093F98F
:10E7680044402149A24219D191F84740B4B10C3133
:10E778000024944206DA51F8046F1C4D25F8146001
:10E788000134F6E70C2805D01849002421F8104078
:10E798000130F7E7164801780131017083F8452008
:10E7A800002201211A7083F8471070BD92F84710B3
:10E7B800C9B140F2DA51A0F2EF248C4208D811789E
:10E7C8000B2905D80B1D0131117042F8230070BDCB
:10E7D800002283F84720074B03F13002002143F859
:10E7E800041F9342FAD170BDF4000020BC2F002012
:10E7F8001C06002000010020024A136C0133194452
:10E8080011647047F4000020024B53F820301B6855
:10E81800198070474C150020074BA1F57A7153F801
:10E8280020301A681B8959434FF47A7391FBF3F12E
:10E8380089B21180704700BF4C15002090F83B3218
:10E8480010B57BB990F83A3290F83942A34209D210
:10E85800B0F8401201229A400A430133A0F840223E
:10E86800DBB2F3E710BD1FB50123ADF80830ADF8F2
:10E878000410002301A9ADF80A30ADF80C30ADF84A
:10E88800062001F09AFC05B05DF804FB8379DB07EC
:10E8980048BFB1FA81F1D0F8343148BF49095A6804
:10E8A8001B8909B113617047536170471FB5012374
:10E8B800ADF808300023ADF80C30ADF80A30094B3C
:10E8C800ADF804101B7801A9012B08BF0323ADF88C
:10E8D800062008BFADF80C3001F06FFC05B05DF8FC
:10E8E80004FB00BFF000002038B510F80E2C0446D9
:10E8F80050F8043C52B9012200F80E2C20F80C1CE8
:10E90800997A18680222BDE83840CFE730F80C2C15
:10E9180020F80A1C891A89B220F8081C074A10F83E
:10E928000F0C002522F8101004F80E5C1868997A6C
:10E938002A46FFF7BBFF04F8065C38BDBC2F002051
:10E94800044B53F820301BB107289CBF1B68198063
:10E95800704700BF1C020020084A13689B020BD5B1
:10E96800074B002119704FF6FE73064908680340EB
:10E978000B604FF400135360704700BF0000024063
:10E98800B93000206C0002402DE9F047664D2B6835
:10E998006649581C0A788E4602F0FF060AB10346FB
:10E9A800F6E737462B60687BAB6895F80C80AA7B46
:10E9B80039B2202900F09C80DFF880C10CEB81037C
:10E9C800DC789B783CF82110C3F1FF039BB2002B45
:10E9D80065D04FF03C0CB1FBFCF9C3F1FF03634376
:10E9E8001B12B9F1050F5DD8DFE809F0030B1A29EE
:10E9F8003A4AE01A4143B1FBFCF0DAB21044C0B223
:10EA080051E0B1FBFCF00CFB101189B2DAB2C1F194
:10EA18003C01E31A4B43B3FBFCFC204694442CE036
:10EA2800B1FBFCF00CFB1011E21A89B24A43B2FBAD
:10EA3800FCF25FFA83F84244D2B2204632E0B1FBDE
:10EA4800FCF90CFB191189B2E01AC1F13C014843E9
:10EA5800B0FBFCF05FFA83F84044C0B2224621E0E4
:10EA6800B1FBFCF80CFB1811D8B289B2E31A01FB10
:10EA780003F2B2FBFCFC224684445FFA8CF412E0F9
:10EA8800B1FBFCF80CFB181189B2D8B2C1F13C01FA
:10EA9800E31A4B43B3FBFCF20244D2B203E0224632
:10EAA800204600E044464FEA042C4CEA004C4CEA6D
:10EAB800020C17234FF0010808FA03F806F11701B2
:10EAC80018EA0C0FA1EB0301DFF8748014BF4FF0B4
:10EAD80011094FF0090989B213F1FF3308F80190C1
:10EAE800E8D218360137B6B2BFB2114BA0465FE77D
:10EAF800AB6001238EF8003040F22A33AA730D4A26
:10EB0800E9800D4985F80C806873AE805360002356
:10EB18008B840B889BB243F001030B80136843F08E
:10EB280001031360BDE8F087441C0020B9300020C1
:10EB3800501C00206C00024000040040920D002090
:10EB4800C5020020F0B5B1F800E000234EFA03F248
:10EB5800D50725D58E784FEAD30CF40648BFCC7874
:10EB680006F00F0203F0070748BF2243BF0050F822
:10EB78002C500F24BC4025EA0404BA402243282E16
:10EB880040F82C2005D1C46801229A4024EA0202E8
:10EB980005E0482E04D1C46801229A402243C2608D
:10EBA8000133102BD2D1F0BD2DE9F04F1E464FF4A2
:10EBB80014734343554D85B005F1100480469146C2
:10EBC800E718A24610B92B44514A03E0012805D1A1
:10EBD800504A2B441A641032C3F844214FF414737A
:10EBE80003FB08F34C48EC180AEB030203F59C738B
:10EBF800343253442061E1636262A36200224FF41D
:10EC080080714FF0010BD4F844310320E161226395
:10EC1800E2622162A263626384F84C2284F848B2FB
:10EC280084F84922A4F85222A4F85422C4F818906F
:10EC38006075A67584F8568258681B8904F5A07219
:10EC48004FF0020CADF80C3003A9102301928DF897
:10EC58000E308DF80FC0CDF800C0FFF773FF236C9E
:10EC6800DDF800C0597B58681B898DF80E1003A980
:10EC7800ADF80C308DF80FC0FFF764FF59463846E1
:10EC8800FFF704FE3220FBF766FC244B019A1B6851
:10EC9800D2F804B01A46B2FBF9F1B1F5803F03D3BC
:10ECA800012AF8D95208F6E71D4A4FF41474B3FB49
:10ECB800F2F204FB08F8584689B2D2B2FCF742FADD
:10ECC80005EB0809174B08F512780AEB080400222F
:10ECD800C9F8583258462146FCF77CFAD9F8405012
:10ECE80016F0010F0CBF022200222868A97AFFF74C
:10ECF800BAFD0D4B2846C9F85C32211D0022FCF7ED
:10ED080069FA384605B0BDE8F08F00BF441C002002
:10ED180080B00108A0B001085C9D010850000020E7
:10ED280040420F0003D3000865D200082DE9F743DD
:10ED38008E460546DFF8A092114699F8B04400685F
:10ED4800164698467246631C89F8B034FCF7A6F953
:10ED58002B8901A9ADF8043018238DF806306868AE
:10ED680002238DF80730FFF7EDFEAB7A09F2B447BE
:10ED7800240127442A6849460C2B00F2F680DFE874
:10ED880013F00D00F400F400F4005100F400F40056
:10ED9800F4008A00F400F400F400C200138CDFF8D9
:10EDA8003CC223F001031B041B0C1384138CB2F820
:10EDB80004E0108B624520F073004FEA00404FEAF0
:10EDC80010409BB21FFA8EFE40F0700014D00CF574
:10EDD800006C624510D00CF5406C62450CD00CF507
:10EDE800806C624508D00CF5806C624504D023F035
:10EDF800020343F0030307E023F00E032EF4407EE2
:10EE080043F003034EF4807EA2F804E01083A2F8D6
:10EE180034801384138B23F008031B041B0C43F06A
:10EE2800080336E0138CDFF8B4C123F010031B0489
:10EE38001B0C1384138CB2F804E0108B624520F489
:10EE4800E6404FEA00404FEA10409BB21FFA8EFEA0
:10EE580040F4E04008D00CF5006C624504D023F083
:10EE6800200343F0300307E023F0E0032EF4406E64
:10EE780043F030034EF4806EA2F804E01083A2F849
:10EE880038801384138B23F400631B041B0C43F496
:10EE98000063138369E0138CDFF840C123F48073A7
:10EEA8001B041B0C1384138CB2F804E0908B62458E
:10EEB80020F073004FEA00404FEA10409BB21FFA5F
:10EEC8008EFE40F0700008D00CF5006C624504D04E
:10EED80023F4007343F4407307E023F460632EF4D3
:10EEE800405E43F440734EF4805EA2F804E09083E1
:10EEF800A2F83C801384938B23F008031B041B0C9B
:10EF080043F0080330E0138CDFF8D0C023F48053BB
:10EF18001B041B0C1384108CB2F804E0938B20F4B0
:10EF2800005023F4E6431B0400041B0C000C62454C
:10EF38001FFA8EFE43F4E04340F4405003D00CF532
:10EF4800006C624503D12EF4804E4EF4804EA2F838
:10EF580004E09383A2F840801084938B23F4006329
:10EF68001B041B0C43F4006393832B7B43B1B2F85F
:10EF780044306FEA43436FEA53439BB2A2F84430EC
:10EF880013889BB243F001031380AB7A0C2B19D87A
:10EF9800DFE803F0071818180B1818180F181818B6
:10EFA80013000B1902F134000AE00B1902F13800C2
:10EFB80006E00B1902F13C0002E00B1902F14000D7
:10EFC800C3F8B40438460C44A4F8BC64C4F8B824A4
:10EFD80003B0BDE8F08300BF441C0020002C0140B2
:10EFE80010B5D420FDF7C5FD8020FDF7C2FDA8208F
:10EFF800FDF7BFFD3F20FDF7BCFDD320FDF7B9FDB0
:10F008000020FDF7B6FD4020FDF7B3FD8D20FDF78C
:10F01800B0FD1420FDF7ADFDA120FDF7AAFDC82025
:10F02800FDF7A7FDDA20FDF7A4FD1220FDF7A1FDED
:10F038008120FDF79EFDCF20FDF79BFDD920FDF730
:10F0480098FDF120FDF795FDDB20FDF792FD4020AE
:10F05800FDF78FFDA420FDF78CFDA620FDF789FDA7
:10F06800AF20FDF786FDA620FDF783FDAE20FDF756
:10F0780080FD2020FDF77DFD0020FDF77AFDB02002
:10F08800FDF777FD4020FDF774FD0020FDF771FDC9
:10F098001020FDF76EFD4FF48064013C0020A4B2FF
:10F0A800FDF762FD002CF8D18120FDF762FDC82034
:10F0B800FDF75FFDAF20FDF75CFD012010BD70B5C9
:10F0C80000EB8000094CA0F1A1059C3825440444BC
:10F0D800074B15F8010F1E787040FDF745FDA54256
:10F0E800F6D13046BDE87040FDF73EBD749D01087D
:10F0F800BD30002010B5441E14F8010F10B1FFF701
:10F10800DEFFF9E710BD08B55038C0B2FDF731FD94
:10F118000020FDF72EFDBDE808401020FDF729BDB1
:10F1280010B504465039C8B2FDF723FD04EB44007E
:10F13800400000F00E00FDF71CFD06206043BDE80E
:10F148001040C0F303101030FDF713BD0028114A1A
:10F15800B8BF404290FBF2F330B50F4C3C2504FB9E
:10F16800030068430D4D90FBF2F22D682D7B25B905
:10F1780003EB830303EB830301E0C3EB031302EB0D
:10F18800830304FB02020B804FF47A7392FBF3F2C1
:10F198004A8030BD80969800806967FFFC10002087
:10F1A800022803D0431E584258417047064B1B683B
:10F1B8001B7823B1054B1868C0F3C0407047044B57
:10F1C8001878C0F380007047F00500200810002070
:10F1D800BA30002010B50A4C5E280146206805D1D7
:10F1E8005D21FBF766FA20683E2105E05D2903D121
:10F1F800FBF75FFA20683D21BDE81040FBF759BADC
:10F20800B821002010B50446C0B2FFF7E3FFC4F3ED
:10F218000720BDE81040DDE7024B5E211868FBF7C8
:10F2280048BA00BFB821002038B50546054C5E2114
:10F238002068FBF73EFA20682946BDE83840FBF70E
:10F2480038BA00BFB821002013B5044601A90068E8
:10F25800FFF77CFF1320FFF7E7FFBDF90400FFF776
:10F26800D1FF1B20FFF7E0FFBDF90600FFF7CAFF3B
:10F278002320FFF7D9FF2368002BB4BF53204E206B
:10F28800FFF7C0FF01A96068FFF760FF1220FFF7D2
:10F29800CBFFBDF90400FFF7B5FF1A20FFF7C4FF45
:10F2A800BDF90600FFF7AEFF2220FFF7BDFF636838
:10F2B800002BB4BF57204520FFF7A4FF02B010BDB4
:10F2C800674B73B51878FFF76BFF664D04462B78CC
:10F2D800834220D0C8B1644B1B68E3B193F90000A6
:10F2E80002230093614B04211B6800225B780033E2
:10F2F80018BF012301934FF41653FBF77AF95C4BBF
:10F30800186040B101232B7005E0594E3068FAF7B8
:10F31800FBFE34602C70574B574D1878FFF740FFB1
:10F328002B780446834218D088B1544B1B68A3B18C
:10F338000022012493F9000008214FF49643009419
:10F348000192FBF756F94E4B186028B905E04C4E70
:10F358003068FAF7D9FE34602C704A4B4A4D187859
:10F36800FFF71EFF2B78044683422E4643D0002821
:10F3780038D0464B1A68002A3DD0D37992F900005C
:10F38800002B4FF00202424C08BF022300920022D9
:10F3980054F8233001921021FBF72BF93D4B054619
:10F3A800186040B33C4C94F84A30022B0BD094F8C8
:10F3B8009620022A01D14C3405E023B1002A04F139
:10F3C8004C0418BF0024354B1C6044B12046002172
:10F3D8004C2207F014FA0223256084F84A300123EE
:10F3E800337008E02B4E306801F0C6FE3068FAF73B
:10F3F8008BFE34602C702A4B2A4D1878FFF7D0FE0C
:10F408002B780446834229D000B3274B1B682BB3C3
:10F41800264A93F900001268032352782021002A13
:10F428000CBF08220922009301924FF46143002285
:10F43800FBF7DFF81E4B186080B11E4A01231370DA
:10F448002B701D4B1A681D4B1A6007E0184E306868
:10F45800FAF75AFE174B34601C702C7002B070BD5E
:10F46800F8050020CC100020F4050020FC10002036
:10F47800B8210020F90500201C110020A01100204F
:10F488009011002004060020A6110020000600208C
:10F4980038A00108A811002038220020AC11002053
:10F4A80010060020BC1100200C06002008060020D1
:10F4B800C0110020C411002024250020C8110020FC
:10F4C800642928BF6421F8B501FB00F5642495FB85
:10F4D800F4F40646E4B20027FBB2A34204D29F200C
:10F4E800FFF7EDFD0137F7E7B4420BD2142195FB86
:10F4F800F1F5C4EB8410663DC4EB80002844C0B22B
:10F50800FFF7DDFD0134E4B2B44201D29A20F7E7F7
:10F51800F8BD2DE9F743FAF7F7FF924C6368C31A71
:10F52800002BC0F2678300F5433303F5A0736360D3
:10F538008D4B1D78237AC5F38005EB1A18BF01237C
:10F5480025724DB1002B00F05583884B5A789A707C
:10F5580001225A701A702BE0844A2BB1D37843F0F9
:10F568000203D37093785370D67806F0020101F045
:10F57800FF0339B97D498968411A002903DB06F080
:10F58800010300E0012303F00107784917707BB1FC
:10F59800F2070DD50A7905230132D2B2B2FBF3F393
:10F5A80003EB8303D31A724ADBB20B71D35C4B7043
:10F5B8006E4EDFF8088233787BB3F37823F00203CA
:10F5C800F3706C4B0344AE20B360FDF7D2FA08B178
:10F5D800FFF706FD88F80000002800F00B83B02034
:10F5E800FDF7C7FA4020FDF7C4FA0020FDF7C1FA7D
:10F5F8001020FDF7BEFA4FF48067013F0020BFB22C
:10F60800FDF7B2FA002FF8D13846FFF77CFD727883
:10F61800594B53F82200FFF76DFD98F80030002B86
:10F6280000F0E8827378062B00F2B282DFE813F06C
:10F638000700B002180078006A018701EC014F4901
:10F648004F4A504B5048F9F740F80120FFF75BFD4F
:10F658004D48FFF74FFD0220FFF755FD4B48ACE141
:10F668004B4F3B689B0735D5DFF854810A23B8F820
:10F678000010DFF85091B1FBF3F203FB121399F875
:10F68800001092B29BB200913F484249F9F71DF829
:10F69800FCF718FE0120FFF736FD3B48FFF72AFD6F
:10F6A8003D4B99F800201868B8F80030067902FB3D
:10F6B800163164234B43C17802208E1B5643B3FB9B
:10F6C800F6F6F6B2FFF71FFD31461520FFF7F8FEF4
:10F6D800032600E001263B681F0540F159822F4BA5
:10F6E8002F491F68642397FBF3F2096803FB127321
:10F6F800009125482B49F8F7E8FFFCF7E3FD304671
:10F70800FFF701FD2048FFF7F5FC00F09BFF0746D7
:10F71800701CFFF7F8FC15203946FFF7D1FE37E2D9
:10F728000120214FFFF7EFFC2048FFF7E3FC3B687F
:10F73800980749D51E4A1448B2F90210B2F90030A8
:10F748000091B2F904201B4901921B4AF8F7BDFF4A
:10F75800FCF7B8FD0220FFF7D6FC0B48FFF7CAFC00
:10F76800032632E0B8210020BA300020D81100204A
:10F778008EBE0108404B4C0018A0010893BE01083A
:10F788009CBE010859B10108C1210020A3BE01088F
:10F7980000250020B1BE0108F4100020001100204F
:10F7A80004110020C9BE010808110020DEBE0108AE
:10F7B800D6100020F4BE010803BF01083D02002056
:10F7C800F81000204400002002263B68D9071AD50B
:10F7D8007B4A7C48B2F90210B2F900300091B2F9C4
:10F7E800042079490192794AF8F76FFF06F1010878
:10F7F800FCF768FD3046FFF786FC5FFA88F8714829
:10F80800FFF778FC46463B681A0718D5704A6D48DA
:10F81800B2F90210B2F900300091B2F904206A4935
:10F8280001926C4AF8F751FF771CFCF74BFD304604
:10F83800FFF769FCFFB26348FFF75CFC3E46664A87
:10F848006149B2F90030B2F902205E480092634A79
:10F85800DFF8B091B2F90020771C0192604AF8F7FE
:10F8680034FFFCF72FFD3046FFF74DFC5548FFF7F6
:10F8780041FC5449D9F80000F8F7C2FD514807F097
:10F8880002F8FFB2C1B2092909D84B1CDBB22144E6
:10F8980020224A720021E21891721946F3E7DFF834
:10F8A8002481D9F804004144F8F7AAFDFCF70AFDC1
:10F8B8003846FFF728FC4046FFF71CFC4146D9F8BC
:10F8C8000800F8F79DFD404606F0DDFF0236F6B267
:10F8D800C7B2092F09D87B1CDBB2274420227A72D1
:10F8E8000021E21891721F46F3E73E4BB3F900007E
:10F8F80003F0EEFB08EB0701F8F782FDFCF7E2FCEA
:10F90800304657E00026384F3B78B34240F24081FA
:10F918000E2E00F03D8170080130FFF7F4FB3046F1
:10F9280002F0ECFC3B78B34206D92020FFF7C7FB76
:10F93800701CC0B202F0E2FC0236F6B2E3E72B4ECE
:10F948002B4996F8AC271F48F8F7BFFE0120FFF7B0
:10F95800DAFB1C48FFF7CEFB264B27491F781948CE
:10F968003A46F8F7B2FE0220FFF7CDFB1548FFF73D
:10F97800C1FB0C2303FB0766204996F8AF2796F8CE
:10F98800AE371048F8F7A1FEFCF79CFC0320FFF700
:10F99800BAFB0C48FFF7AEFB96F8B41796F8B227F7
:10F9A80096F8B337074800911549F8F78EFEFCF72B
:10F9B80089FC0420FFF7A7FB0248FFF79BFBE7E061
:10F9C80028100020C1210020F4BE010807BF01084B
:10F9D8002E10002016CC0108F8240020E410002086
:10F9E8000BBF010864170020D422002060250020E6
:10F9F8000FBF0108AC2400201BBF01082CBF010861
:10FA08003DBF0108581700207C4B1B681B0640F1BE
:10FA1800BB80236A616A7A4A8B421CBF536292F8A0
:10FA280028304FF001011CBF013303F003034FF0EE
:10FA3800000018BF82F82830FFF772FB94F82830CE
:10FA4800704A0026D05CFFF73AFB02200121FFF73D
:10FA580067FB6D4B3620F35C0136C3EBC30393FBA6
:10FA6800F0F0C0B2062828BF06206038C0B2FFF701
:10FA780026FB102EEDD1654B65491B78654813F0C0
:10FA8800020F654B1A7814BF59234E23F8F71DFE51
:10FA9800FCF718FC0220FFF736FB5E48FFF72AFB4D
:10FAA8005E495F4B4E680A685A4892FBF3F25D491B
:10FAB80096FBF3F3F8F709FEFCF704FC0320FFF7C5
:10FAC80022FB5448FFF716FB574B58491A885148F0
:10FAD800F8F7FBFDFCF7E2FB0420FFF714FB4D48A9
:10FAE800FFF708FB524B53491A884A48F8F7EDFDCF
:10FAF800FCF7D4FB04210A20FFF712FB4548FFF767
:10FB0800F9FA4D49E26A4348F8F7DFFD4B4EFCF736
:10FB1800C5FB0520FFF7F7FA3E48FFF7EBFA7268D6
:10FB2800B36847493B48F8F7D0FDFCF7B7FB052118
:10FB38000A20FFF7F5FA3748FFF7DCFA3369F2686D
:10FB48004049D21A3348F8F7C0FDFCF7A7FB062056
:10FB5800FFF7D9FA2F48FFF7CDFAB2683A492D488E
:10FB6800F8F7B3FDFCF79AFB06210A20FFF7D8FA4D
:10FB78002848FFF7BFFA35491522264806F0AEFE99
:10FB8800FCF78CFB072015E7F37843F00203F370CA
:10FB9800002D2FD12E4B00219B791220032B97BFCC
:10FBA8002C4A3F259B181D7FFFF7BAFA2846FFF716
:10FBB80086FA13200021FFF7B3FA274B1B78002B96
:10FBC800264B18BF72201B7808BF2120002B18BFB6
:10FBD8005220FFF774FA14200021FFF7A1FA94F8D5
:10FBE8003050084B585D013505F00305FFF767FAFB
:10FBF80084F8305003B0BDE8F08300BF0025002032
:10FC0800B82100204FBF0108B91000200C110020B6
:10FC180054BF0108C1210020121100201411002036
:10FC28008096980065BF01080E11002072BF010878
:10FC3800701000207ABF010881BF01088C070020DE
:10FC480088BF010891BF010898BF0108B0020020D1
:10FC58001C0E002018A001084B0E0020B00E00203A
:10FC6800084BDA68D10709D4DA68520708D4DB6888
:10FC780013F0100F14BF03200420704701207047B1
:10FC88000220704700200240704770477047037891
:10FC98008B4286BF024B33F811000020704700BF2B
:10FCA800F02100200021062206F0A9BD002106222D
:10FCB80006F0A5BD70B50546FAF726FC324CA369D7
:10FCC800A061C31AB3F5FA5FE36182BF002384F829
:10FCD800203084F8213094F820302BB9A12D02BFB0
:10FCE800294A012182F8211094F82110264A31B1BD
:10FCF800D118EDB2013381F8225082F8203094F8FF
:10FD0800205094F84330AB423CD11F4B93F8443019
:10FD1800052B02D0062B03D02FE0002002F034FE82
:10FD280094F823301E2B28D100200246C1B26B1E46
:10FD380099421ADA214491F822300821DBB283EA89
:10FD48000206F60744BF83F01803C3F3460301F124
:10FD5800FF3154BF5B0843F0800311F0FF01C2F389
:10FD68004702ECD101301A46E0E7234493F82230E9
:10FD78009A4202D1032002F007FE002384F82130C2
:10FD880084F8203070BD00BFF021002010B5044673
:10FD9800B0F9000002F040F8B4F9020002F03CF8B3
:10FDA800B4F90400BDE8104002F036B810B50446B6
:10FDB800006802F031F8606802F02EF8A068BDE82B
:10FDC800104002F029B82DE9F74F0120FAF78AFA16
:10FDD800002488B3012C2FD84FF04C0909FB04FAF2
:10FDE800174E06EB0A0808F19007BD7815B10134E3
:10FDF800E4B2EEE790F9003090F804E01846114BB1
:10FE080003228DE8240001212A4653F82E30FAF700
:10FE1800F0FB834660B106F14800504429464A4643
:10FE280006F0EDFC01231C44C8F848B0BB70E4B2EE
:10FE38000120FAF73DFACCE703B0BDE8F08F00BF28
:10FE4800F021002038A001080021222210B5104816
:10FE580006F0D5FC0F4B002219460F480424105C0D
:10FE6800013283F8F20183F8F74105200024042ABF
:10FE780083F8F60183F8F94183F8F80103F10803E0
:10FE8800EBD10123A1F8F431522381F8F03110BDF0
:10FE98005027002060250020CDBF010870B5064618
:10FEA800441E14F8011F89B1094D284606F0DDFCEF
:10FEB8000028F6D005F1080398423FBF054B401BC8
:10FEC800C018A31B38BF80F88A31EAE770BD00BFAD
:10FED80023CC01086025002007B51C4B03F1E40280
:10FEE800C3F8E0201A4A92F892215AB1012A14D193
:10FEF800032183F8E610072183F8E82083F8E71048
:10FF08000C2208E0022183F8E610032183F8E82098
:10FF180083F8E710072283F8E4200E4A0E4B4020AE
:10FF28001A60FAF7DFF970B10122002390F9000096
:10FF380040218DE80C00094A4FF4E133FAF759FBE8
:10FF4800003018BF012003B05DF804FBF021002049
:10FF5800602500204D27010830000020FD270108FA
:10FF68000120002101F056B9174AF0B5164692F85B
:10FF7800E930D2F8ECE0032B10D85C1C0EEBC3037D
:10FF88009D1CE4B208D09A88D10705D5104203D049
:10FF980008E00131042907D12346ECE786F8E93067
:10FFA8000020F0BD9F7800210C2202FB01F3064DD2
:10FFB80005F1F00C1CF803209742EAD12B4485F890
:10FFC800E940D3F8F400F0BDF02100208A6810B5AC
:10FFD8000C6A036814430A6923F4FF4314434A690B
:10FFE80023F0700314438A691443CA6914434A6AA4
:08FFF80014438A6A22431343FB
:020000040801F1
:100000000360CB6843600B6883604B68C36010BDBE
:100010004FF6FE73026813400360002303604360E1
:100020008360C360284B984201D1284A27E0284BBF
:10003000984201D1254A2AE0264B984201D1234A11
:100040002DE0254B984201D1204A30E0234B9842C5
:1000500001D11E4A33E0224B984204D11B4A536817
:1000600043F470032EE01F4B984204D1174A5368A3
:1000700043F0706326E01C4B984204D11B4A53683E
:1000800043F00F031EE01A4B984204D1174A5368FD
:1000900043F0F00316E0174B984204D1134A53681B
:1000A00043F470630EE0144B984204D10F4A536836
:1000B00043F4704306E0114B984204D10B4A536855
:1000C00043F4702353607047080002400000024070
:1000D0001C00024030000240440002405800024030
:1000E0006C0002408000024008040240000402400C
:1000F0001C04024030040240440402405804024000
:10010000224A10B5536803F00C03042B03D0082BCC
:1001100004D01F4B14E01F4B5B6811E0536851681B
:10012000C3F38343C90303F1020301D41A4906E070
:10013000516811F4003F1749496818BF49084B43FB
:1001400003605368154CC3F30313234493F8201042
:100150000368CB4043605168C1F30221214491F808
:10016000201023FA01F181605168C1F3C2212144BA
:1001700091F82010CB40C3605268C2F38132224410
:1001800092F83020B3FBF2F3036110BD001002407F
:1001900000127A003000002000093D0038A001085C
:1001A00010B50446FFF760FD012806D11CB1FFF72A
:1001B0005BFD013CF8E7052010BD002C08BF0520C1
:1001C00010BD0A88F0B54B888E88B1F808E0CC885D
:1001D000002A3AD1028C43F0010322F001021204FA
:1001E000120C0284058B078CADB225F0F30545EAAD
:1001F0000E1189B241EA06027A49BFB2884212D092
:1002000001F5006188420ED0B0F1804F0BD0A1F50E
:100210009831884207D001F58061884203D001F50A
:100220008061884202D127F0020701E027F00A0727
:100230001F4302830784038B23F00C031B041B0C56
:100240000383038B9BB21C4344E0042A44D1028CF9
:1002500022F010021204120C0284018B058C21F48E
:1002600040721205120D42EA0E325E4992B242EA23
:1002700006228842ADB292B212D001F500618842E6
:100280000ED0B0F1804F0BD0A1F59831884207D045
:1002900001F58061884203D001F58061884207D171
:1002A00025F0200141EA03139BB243F0100304E060
:1002B00025F0A00143F010030B4302830384038B5A
:1002C00023F440631B041B0C0383038B9BB243EAA0
:1002D0000424A4B20483F0BD082A028C3ED122F487
:1002E00080721204120C0284828B3E4D92B222F074
:1002F000F307018C47EA0E1292B2A84289B242EA91
:10030000060212D005F50065A8420ED0B0F1804F6C
:100310000BD0A5F59835A84207D005F58065A84211
:1003200003D005F58065A84207D121F4007141EAA8
:1003300003239BB243F4807304E021F4206143F46F
:1003400080730B4382830384838B23F00C031B0491
:100350001B0C8383838B9BB21C4341E022F48052AD
:100360001204120C0284858B018C25F440752D0536
:100370002D0D45EA062545EA0E321A4D89B2A842EE
:1003800092B212D005F50065A8420ED0B0F1804FB0
:100390000BD0A5F59835A84207D005F58065A84291
:1003A00003D005F58065A84207D121F4005141EA48
:1003B00003339BB243F4805305E047F6FF5543F403
:1003C00080530D402B4382830384838B23F440634B
:1003D0001B041B0C8383838B9BB243EA0424A4B2CB
:1003E0008483F0BD002C0140CA78F0B5D40648BF24
:1003F0008C780D8802F00F0348BF234315F0FF0FE0
:100400001DD0016800240126A64006EA0507B74270
:1004100011D14FEA840E0F2606FA0EF621EA0601E4
:10042000282A03FA0EF641EA060101D1476102E0EB
:10043000482A08BF07610134082CE4D10160FF2D70
:100440001FD94168002404F108070126BE4006EACE
:100450000507B74211D14FEA840E0F2606FA0EF6B1
:1004600021EA0601282A03FA0EF641EA060101D123
:10047000476102E0482A08BF07610134082CE2D135
:100480004160F0BD0F4B1A6842F001021A605968D2
:100490000D4A0A405A601A6822F0847222F48032AF
:1004A0001A601A6822F480221A605A6822F4FE0246
:1004B0005A604FF41F029A60044B4FF000629A603A
:1004C000704700BF001002400000FFF800ED00E0A0
:1004D0002DE9F8435B4C0368013AC4F82031838866
:1004E0000D46A4F82431072A42D8DFE802F0040AB6
:1004F000101822292F35B4F820310B80B4F822319E
:1005000013E0B4F822310B80B4F8203105E0B4F8E0
:1005100020315B420B80B4F822315B4205E0B4F835
:1005200022315B420B80B4F820316B80B4F8243167
:100530001DE0B4F820315B420B80B4F8223112E0A8
:10054000B4F822310B80B4F820310CE0B4F820313B
:100550000B80B4F8223105E0B4F822315B420B8005
:10056000B4F820315B426B80B4F824315B42AB803D
:10057000354B1B7A002B62D1B5F9000002F0ACFDBF
:100580008046B5F9020002F0A7FD0746B5F9040060
:1005900002F0A2FDD4F828110646404602F0F0FD14
:1005A000D4F834118146384602F0EAFD0146484647
:1005B00002F0DEFCD4F840118146304602F0E0FD46
:1005C0000146484602F0D4FC06F02AFBD4F82C1170
:1005D0002880404602F0D4FDD4F8381181463846D0
:1005E00002F0CEFD0146484602F0C2FCD4F84411A8
:1005F0008146304602F0C4FD0146484602F0B8FC90
:1006000006F00EFBD4F830116880404602F0B8FDC9
:10061000D4F83C118046384602F0B2FD014640460F
:1006200002F0A6FCD4F848110746304602F0A8FDB7
:100630000146384602F09CFC06F0F2FAA880BDE8BC
:10064000F88300BFF02100203000002038B50F4BA8
:100650001B689C890E4B186880F31000201A02F06A
:100660003BFD0C4902F08CFD0546204602F034FDAE
:100670000146284602F038FE02F048FF6428A8BF71
:10068000642020EAE070C0B238BD00BFF410002042
:10069000041100200000C84244F6FB71084B1A68A0
:1006A000137803EB431300FB03135078C0EB0030C7
:1006B000B3FBF0F39078B3FBF0F080B2704700BF6B
:1006C000F410002008B50A480A2290F84D3100EBDA
:1006D0004303B3F85C1100F5B47089B220F8041C30
:1006E000FAF7D6FF80B2FFF7D7FF024B188008BD9C
:1006F000F0210020F810002010B54B88DC0641BF27
:100700002F4B14791B6853F8244044BF2D4B43F8FA
:1007100020404B889B0641BF294B54791B6853F8F6
:10072000244044BF274B43F820404B881C070ED57C
:10073000254B0C781B78B3EB141FA1BF204BD4784A
:100740001B6853F82440A4BF1E4B43F820404B883D
:100750009B070ED51D4B0C781B78B3EB141FDFBF26
:10076000174B54781B6853F82440DCBF154B43F8F3
:1007700020404B88DC070FD5154C0B78247803F00C
:100780000F03A342DFBF0E4B14781B6853F82440BD
:10079000DCBF0C4B43F820404B885B070FD50B7830
:1007A0000C4903F00F0309788B42A1BF044B9278E8
:1007B0001B6853F82220A4BF024B43F8202010BD31
:1007C00018120020920D0020AB170020A91700205E
:1007D000A8170020AA170020254A0023F0B51568A5
:1007E0001C461A462348244903700B702E1976883C
:1007F0004EB92F5D3FB9037000230A704B70077824
:100800001C461A460CE0360548BF013204F10404C8
:1008100003F1010348BFD2B2802CDBB2E6D1EAE794
:10082000E0B2B8420CD215F82400013406099E4209
:1008300000F00F00A8BF731C9042A8BF421CEFE756
:100840008A704B70C2F3470102F001020A444C1E49
:100850000A490B480A70C3F3470203F0010313442B
:1008600004700849501E084A08701370F0BD00BF9C
:100870001C120020A0170020E0230020AA1700204F
:10088000A8170020AB170020A9170020924B2DE9D4
:10089000F04FDA68914D1A612A6891B0DA60904A97
:1008A0000295136843F0200313608E4B1A78012AD7
:1008B0000CBF002201221A708B4B1A78910740F16D
:1008C0004D838A490978042940F248838849097888
:1008D00001F0040101F0FF0011B922F001021A70C9
:1008E0001B78DB0702D408B1FAF740FB8149CA78CC
:1008F000531C052293FBF2F202EB82029A1A7E4B02
:10090000CA701F7892000023DFF81082DFF810927F
:1009100058F82310794C91FBF9FE04F1080040F8D7
:1009200023E0774844F8231000FB0E1142F21070C8
:1009300091FBF0F004F1100680B226F813004FF09E
:10094000140C04F114060CFB036C04F13C0A5AF875
:1009500023605CF802504CF80210761B31440526E7
:100960004AF8231091FBF6F109FB0E114434012FD4
:1009700044F823104FEA830B444605D10238B0F502
:10098000797F98BF4BF808100BB90123BCE7594E8B
:10099000029BB2461868336DC01A02F099FB5949A0
:1009A00002F0A2FC029B4FF07E511B6807463365A4
:1009B00002F084FD08B94FF07E574B4BCAF85470D3
:1009C0001B78514E13F00103504D12D00DAA009226
:1009D0004F4B0EAA01920CCB94E80300FAF7DCF916
:1009E0000D9A6421B2FBF1F20E9B328093FBF1F37E
:1009F00000E033802B809AF858303E4D002B35D0E4
:100A0000696D4FF07E5002F06FFC0746EB6D206879
:100A1000C01A02F061FB394602F0B2FB02F076FD2B
:100A20002B6E86B2606836B2C01A02F055FB394BA5
:100A3000196802F0A5FB394602F0A2FB02F066FD40
:100A4000B5F9662000B28118B5F964200220B31808
:100A500091FBF0F193FBF0F389B29BB2A5F86A1019
:100A6000A5F86830A5F86610A5F8643001238AF867
:100A70005830294B61681B88206803F030031D4EF5
:100A8000264DCAF86010CAF85C00002B00F06682A0
:100A900006F17403009306F178030193F26E336F4D
:100AA000FAF77AF96B68306FC01A02F015FB194B30
:100AB000196802F065FB02F029FDF36E2A68C6F89A
:100AC00080009B1AF3670C4B1B78012B2AD0022B5A
:100AD00000F0E68042E200BF8C07002024250020C1
:100AE00008110020721000200C11002012110020AB
:100AF000BA300020E02300201C0F0020E423002057
:100B0000806967FF00007A44861100208811002068
:100B1000741000203C000020D0110020141100208F
:100B200080969800D6F88430D6F8A0400293D6F884
:100B3000943004F100400393D6F89830776D059314
:100B400002F0E4FC8146204602F0E0FCD6F89C303E
:100B5000BB4C0493BB4B06901B684FF0000B0793F4
:100B6000B94E4FEA4B0356F82B80A6F114024046CB
:100B700032F81B50089302F0AFFA029902F000FB22
:100B800002F0C4FC401B1FFA80FA283626F81BA08E
:100B90000FFA8AFA504602F09FFA039902F0F0FA2F
:100BA00002F0B4FC86B20AEB080002F095FA05994F
:100BB00002F0E6FA394602F0E3FA216802F0D8F9C9
:100BC00002F0A4FC484504DB069B9842A8BF1846E7
:100BD00000E0484602F080FA206002F097FC079B94
:100BE000304486B2987802F073FA984902F0C8FA55
:100BF00001464FF07E5002F077FB394602F0B8F91B
:100C00000146384602F070FB09906068D4F808A0ED
:100C1000C0EB080002F060FA394602F065FB51466D
:100C200002F0A4F9099A0146104602F0A9FA014619
:100C3000504602F09DF93135ADB2622D014620617A
:100C4000C4F80480A0600ED9049802F099FA02F06A
:100C50005DFC7F4AB0F5FA6FA8BF4FF4FA6090428E
:100C6000B8BF104600E0002040F6B832064436B265
:100C70009642A8BF1646774A089B9642B8BF1646CA
:100C8000754A54F8140B9E52142202FB0BF273495E
:100C90005050BBF1000F40F061814FF0010B5FE756
:100CA000684BB6F8A8401F68736F3D8902935B08D4
:100CB0009D4228BF1D4623B29D4202DC1FFA85F9E2
:100CC0000AE06749706D02F05BFA02F01FFC2044F5
:100CD0001FFA80F9A6F8A890DAF87860DAF8AC4044
:100CE000341B2046FAF79AF841F293130028D8BF34
:100CF00040429842CCBF0020012078B3204602F049
:100D0000EBF9584902F03CFAF7F727FD0446029840
:100D100002F0DEF90146204602F032FA02F0F6FB5C
:100D200040F6B83380B2AAF8B00000B29842A8BF2B
:100D30001846484B9842ACBF3018F01848F6A0430C
:100D4000984203DDA0F50C40A03804E00028BCBFA9
:100D500000F50C40A030CAF8B40001E0CAF8B46055
:100D6000DAF8B4300026C3F50C502830039302F0B3
:100D7000B3F93C4902F004FA0446F7F761FD0F901D
:100D80002046F7F7EAFCDAF8B830DAF8C440059301
:100D9000DAF8BC300E9004F10040089302F0B6FB84
:100DA0000490204602F0B2FBDAF8C030DAF8548042
:100DB0002A4C09900793730048460A9302F08CF975
:100DC0000EAB53F8261002F0DBF9DFF8A0A00546C1
:100DD0003AF9160002F080F90146284602F0C6F8FA
:100DE00002F094FB05B2204BB5F57A7FA8BF4FF413
:100DF0007A759D42B8BF1D460AF13C0AA8B22AF88E
:100E0000160000B202F068F90599824602F0B8F9BE
:100E100002F07CFB089983B25046069302F0B0F9C9
:100E2000414602F0ADF9216802F0A2F802F06EFB33
:100E3000049B98421CDB099B9842A8BF184618E007
:100E4000580F0020200F00205C240020DB0FC94039
:100E500030F8FFFF48F4FFFF2A0F0020800F00202A
:100E60000000C842D302373918FCFFFF4824002095
:100E7000049802F031F920608346B87802F028F92E
:100E8000384902F07DF901464FF07E5002F02CFA0D
:100E9000414602F06DF80146404602F025FA0B90FB
:100EA0006068D4F808A0281A02F016F9414602F04A
:100EB0001BFA514602F05AF8DDF82CC00146604694
:100EC00002F05EF90146504602F052F865600146B4
:100ED0002061A060079802F053F902F017FB069B0F
:100EE0001434034458469A4602F010FB40F6B832D8
:100EF000504400B29042A8BF10461B4A0A9B904241
:100F0000B8BF1046194A1A4998521422724342F83F
:100F100001B00EB901264EE73B792BB1039A642349
:100F200092FBF3F3134A13803B88029A124C9A42C5
:100F30000DD9D4F8AC30A06FC01AF9F76FFF42F2A8
:100F4000107380EAE072A2EBE0729A4206DD0B4B6E
:100F500001221A70B4F8C820064B1A8011B0BDE8FF
:100F6000F08F00BFDB0FC94048F4FFFF2A0F0020BD
:100F7000580F0020180F0020E02300201C0F002035
:100F800007B5064B06490093064B074A01930748ED
:100F9000074BF7F7B3FB03B05DF804FB84B101081E
:100FA000A3BE010859B101089CBE0108D1BF0108C8
:100FB00078B1010808B5037833B90C4B0C4819789F
:100FC000BDE80840F7F79ABB05F0B6FC02280CD83C
:100FD000064B0C221870074B02FB0030064B063004
:100FE0001860F7F7F3FD0548E5E708BDAC240020DD
:100FF000F1BF0108082D00206C1000207BB401080F
:1010000008B503783BB90B4B0B4893F8AC17BDE818
:101010000840F7F773BB05F08FFC022808D8054B92
:1010200083F8AC07F7F730FDF7F7F4FD0348E8E77E
:1010300008BD00BF60250020F5BF01087BB4010892
:1010400038B5037803BB214B1B6801330F2B07D83E
:101050001F490C2202FB031295681C462DBB00E0C1
:101060001C4601340F2C01DD002400E005D818498E
:101070000C2202FB04129568BDB99C42F1D11548BF
:10108000BDE83840F7F73ABB05F056FC0F28044698
:1010900005D80F4A0C2303FB00239D682DB9214678
:1010A000BDE838400C48F7F729BB084B1C60F9F73E
:1010B000E3F921462A460948F7F720FB0C235C4355
:1010C000034B185DBDE83840F9F7E8B9400000204F
:1010D0006CA0010802C0010818C0010830C0010856
:1010E00073B5037813B9F8F76FFD3DE01F4901AA06
:1010F00005F083FC002401462646254699B134B10B
:10110000012C08D1084605F017FC064603E0084606
:1011100005F012FC05461549002001AA05F06DFCFA
:1011200001340146EAE70B2D02D911480C220BE0ED
:10113000022C10D1A6F57A73B3F57A7F07D90D4842
:101140004FF47A714FF4FA62F8F7BBFC0CE00A4BEB
:1011500003EB45035E80084B084803EB4503294633
:10116000B3F90220F7F7CAFA02B070BDC6B601089B
:10117000DCB601082FBA0108AC24002047C00108E2
:1011800038B50D4C05462368834206D1F8F7C0FFF9
:10119000204600214C2205F036FBE36CAB4209D11E
:1011A0002846F8F7B5FFBDE83840044800214C2236
:1011B00005F029BB38BD00BF382200208422002062
:1011C000034B1A68D379591C1344D171187A7047AC
:1011D000B011002010B5FFF7F3FF84B2FFF7F0FF66
:1011E00004EB002080B210BD10B5FFF7F3FF0446FA
:1011F000FFF7F0FF04EB004010BD10B50446054BAF
:1012000021461868F9F759FA034B1B689879604032
:10121000987110BDB4110020B011002038B50446FB
:101220000D462420FFF7E9FF4D20FFF7E6FF002CD5
:10123000084C14BF21203E20FFF7DFFF2368002267
:1012400028469A71FFF7D9FF236893F84900BDE853
:101250003840D2E7B011002001460020DEE710B58B
:101260000446C0B2FFF7C9FF200ABDE81040C4E73A
:1012700010B5044680B2FFF7F2FF200CBDE8104025
:10128000EDE737B582888368044610060D4641BFF6
:1012900029494FF4CC7091F8AC1700FB0133D1050C
:1012A00042BF26490C20097802F03F0248BF00FBEC
:1012B0000133042A12D006D8012A0DD0022A2FD1D8
:1012C00093F900102DE0102A0AD0202A0AD0082A0B
:1012D00026D1B3F9001024E0197822E0198820E023
:1012E00019681EE069461868F7F78EF80146144839
:1012F000F7F704FAF5B1E06801F0EEFE6946F7F79A
:1013000083F801460F48F7F7F9F9206901F0E4FE88
:101310006946F7F779F801460A48F7F7EFF909E067
:1013200000210948F7F7EAF925B10848E168226980
:10133000F7F7E4F903B030BD60250020AC240020AD
:10134000B9B50108B2B501087EBF010856C0010851
:10135000024B0146D869F9F7B0B900BFAC240020B0
:1013600010B5441E14F8011F21B1034BD869F9F7D9
:10137000A4F9F7E710BD00BFAC240020F7B52A4957
:101380002A4B08782A4D1C682A4B05EB80001A88E6
:10139000D0F8C010284B29481B7800914FF47A717F
:1013A000B4FBF1F1F7F7AAF9254B26481968264B4B
:1013B0000026B1FBF3F1F7F7A1F9244B1F68F3B254
:1013C00005EB8302D2F8D010E9B101249C403C42E5
:1013D00017D0220715D01E4A0B20D25C00FB032336
:1013E000134A1C4802EB8303D3F8F020F7F786F981
:1013F000022C06D1184B93F8281011B11748F7F7B3
:101400007DF90136DBE71648FFF7AAFF154B1648B2
:101410001A88164B92B219884FF4FB6303B0BDE8EB
:10142000F040F7F76BB900BF5811002024250020C9
:101430006CA00108F8100020440000205DC00108E5
:1014400050000020A0C0010840420F0008110020F9
:101450004C000020B0C00108AC240020B8C0010836
:1014600000C1010806100020BCC0010804100020C3
:101470002DE9F0410024804625460F4E4146A759EC
:10148000384605F041FA58B139460C48F7F736F9B5
:1014900030190021FFF7F5FE0948FFF761FF01351C
:1014A00040F6944314349C42E7D11DB9BDE8F041A5
:1014B000044855E7BDE8F0810CA2010831B60108E7
:1014C00000C10108E1B501082DE9F74F824605F09A
:1014D000DEF9054628B1012819D19AF800302A2BE7
:1014E00015D15948FFF73CFF0024584E5848A159E0
:1014F000F7F704F930192946FFF7C3FE5548FFF7FF
:101500002FFF40F6944314349C42EED198E05046AD
:101510003D2105F0AEF9002800F08D8003461D4600
:1015200013F8012D202AFAD0441C204605F004FAB5
:1015300081462046F6F7D2FE0746CAEB05054FF076
:10154000000B142404FB0BF4DFF8208108F5D073A2
:10155000E6580193304605F09AF9844631466246D2
:101560005046CDF800C005F09BF9DDF800C0019BA6
:10157000002856D1EAB2624553D11D194444D4F82B
:10158000AC0101F0A9FD0146384601F0ABFF00288F
:1015900045D0D4F8B00101F09FFD0146384601F076
:1015A00097FF00283BD0B4F8A4319A0658BF4F46A5
:1015B000142202FB0B881C0648BF2748D8F8A82134
:1015C00042BF90F8AC074FF4CC7404FB0022D8055E
:1015D00042BF22480C24007803F03F0348BF04FBBD
:1015E0000022042B39460BD004D8013B012B0CD828
:1015F00017700AE0102B05D0202B05D0082B04D142
:10160000118002E0176000E0176031461448F7F7D8
:1016100075F82846002103B0BDE8F04F31E61148C7
:1016200005E00BF1010BBBF1A10F8AD10E4803B00D
:10163000BDE8F04F94E6504603B0BDE8F04F17E721
:1016400003B0BDE8F08F00BFEEC001080CA2010896
:1016500031B6010800C1010860250020AC2400203B
:1016600003C101080EC10108E1B501086CA0010821
:1016700070B50546284605F00AF9064658B9194BD3
:1016800019485A79194BBDE8704003EB8203D3F82F
:10169000301EF7F733B828461549324605F000F9F1
:1016A00060B91448FFF75CFE134C54F8041F19B1DD
:1016B0001248F7F723F8F8E7114805E00024114B2A
:1016C00053F8241019B91048BDE8704048E6284680
:1016D000324605F0E5F801340028F0D1014B0B4DFE
:1016E0005C71C7E7602500202EC101086CA00108CD
:1016F000D0B501083AC101089CAE0108CCB501087B
:1017000000C10108A0AE0108E1B501087BB40108E1
:1017100008B50748FFF724FE064BD869F8F7B9FF6C
:10172000FAF732F9F7F786F9034A044BDA6008BD95
:101730004DC10108AC2400200400FA0500ED00E0D2
:1017400008B50548FFF70CFE00F036F8F7F79CF9EE
:10175000BDE80840DCE700BF59C1010808B50448EE
:10176000FFF7FEFDF7F790F9BDE80840D0E700BFAE
:101770006FC101080E4B1A78692A15D15A88B2F543
:10178000FB6F11D11A79BE2A0ED193F8D52700200C
:10179000EF2A0BD113F8012B5040064A9342F9D19E
:1017A000B0FA80F04009704700207047704700BFD2
:1017B00000F80308D8FF03082DE9F74FEA4C002191
:1017C0004FF4FB62204605F01EF8E84B04F5397231
:1017D0001A60E74B00221A70E64B04F2AE711960F2
:1017E00069232370032363714FF48073A3604FF464
:1017F0001673A4F86631FA23A4F86831BC23A4F860
:1018000064314FF4FA73A4F86E31012384F8623125
:1018100084F87E3184F88631052384F8233240F23F
:10182000DC53A4F8983140F24C43A4F89A3140F2CA
:101830006C73A4F89C3140F27533A4F89E3140F6E5
:101840004303A4F8A0312346202184F86A116E21B5
:1018500084F87C110A2184F87D112B2184F87F11F2
:10186000212184F88011232184F881114FF4C8715B
:10187000A4F882119918023200254FF01E0A242A7A
:10188000B94C81F8A25181F8A3A1F3D140F27E4175
:10189000A4F8441140F23A71A4F8461140F27E5186
:1018A000A4F84C1140F2EA5140F2DC50A4F84E1179
:1018B00040F2B4514FF4FA63A4F8C831A4F8CC3123
:1018C000A4F8D031A4F8D431052384F8DE31C8233C
:1018D00001264FF47A784FF0320BA4F8E231DFF8AA
:1018E0008C924FF4C8731922A4F8E631A4F84A0187
:1018F000A4F85011A4F8C681A4F8CA81A4F8CE8136
:10190000A4F8D28184F8E06184F8E16184F8E461AC
:10191000A4F84881A4F852B184F895A184F8DF2195
:1019200000920190A4F8543184F8DD6184F8EA61F2
:10193000A4F856B184F8ED61FEF78AFAD9F80030C0
:10194000009A4FF00F0E2674E673A573A58183F8F5
:1019500005E04FF0220E172183F806E0DA714FF010
:101960000E0E21225975997583F810E05A7455218D
:101970004FF0350E53224FF0640C2827D97083F8AE
:101980001AE02D21DA764FF05A0E0A2283F81CC095
:101990004FF0780C83F80BA083F80CA0597383F8F0
:1019A00008E09A7483F80AC01D705F709F70DD753F
:1019B00083F804B09D731D76DD735D765F721975D3
:1019C0004FF4FA71A3F84E106B49DFF8CCC199635C
:1019D000D9636A49C3F82CC0C3F830C09962DFF8F4
:1019E000BCC14FF07E5159634FF07F5A6449019852
:1019F000C3F820A0C3F824A0C3F848C04FF0000AE1
:101A00004FF04B0C83F8502059649E7783F8525066
:101A100083F85170C3F840A083F84CC084F8AEE757
:101A2000A4F8B8074FF0410E042084F8AFE784F81B
:101A3000B0B784F8B15784F8B55784F8B65784F82E
:101A4000B25784F8B35784F8B457009283F85C0017
:101A5000A3F85850A3F85A50A3F856501966152108
:101A600083F8681047494848D966484983F8647044
:101A70001967474983F86570596783F87860FEF7FE
:101A800011FAD9F80030009A18464FF4487183F8DB
:101A9000115183F8125183F8137183F8146183F89C
:101AA0001851A3F8161184F8D821C82284F8D92136
:101AB000A4F8DA810E2202FB05326FF0170482F8D7
:101AC0001941032482F81A416FF02F0482F81B4158
:101AD000072482F81C416FF0230482F81D4105247D
:101AE00082F81E4101355A2480F8204180F82141B6
:101AF0006422FF24082D80F81F2180F822414FF036
:101B0000000100F10E00D5D1C820A3F88A011420ED
:101B100083F88C01A3F890211E204FF4967283F86D
:101B20008D01A3F892210120282283F8891183F8DE
:101B30008E01A3F894210B460B4D5A191033C02B7C
:101B4000C2F814A0F8D105F529700021402204F054
:101B50005AFE00230F4EEA18995904330868382BAF
:101B6000014CC2F8A4021BE06025002044100020B4
:101B7000AC2400206C1000208FC2F53C00002040F7
:101B80000000A0409A99193F1ACC0108F6287C3F22
:101B90003D0A773F64AF0108CDCCCC3E0000404009
:101BA000D8D104F509700021802204F02CFE06F142
:101BB0003801702204F5097004F01AFEFEF70CFEDD
:101BC000D9F8006000230125314604F27C404FF42F
:101BD000CC7284F8D43784F8D25784F8D35704F001
:101BE00007FE04F2146031464FF4CC7204F000FE9C
:101BF0000D4B1B681A68C4F8BA275A68C4F8BE2788
